:1000000000800020BD010000CDC7000085C70000B2
:1000100085C7000085C7000085C7000085C70000B0
:1000200085C7000085C7000085C70000CDC7000058
:10003000CDC7000085C700004DBE000051BF0000C5
:10004000CDC70000CDC70000CDC70000CDC7000060
:10005000CDC70000CDC70000CDC70000CDC7000050
:10006000CDC70000CDC70000CDC70000CDC7000040
:10007000CDC70000CDC70000CDC70000CDC7000030
:10008000CDC70000CDC70000CDC70000CDC7000020
:10009000CDC70000CDC70000CDC70000CDC7000010
:1000A00089A3000095A30000CDC70000CDC70000C4
:1000B000CDC70000CDC70000CDC70000CDC70000F0
:1000C000CDC70000CDC70000CDC70000CDC70000E0
:1000D000CDC70000CDC70000CDC70000CDC70000D0
:1000E000CDC70000CDC70000CDC70000CDC70000C0
:1000F000CDC7000039E80000CDC7000065E9000069
:10010000CDC70000A5D10000CDC70000CDC70000BD
:10011000CDC70000CDC70000CDC70000CDC700008F
:10012000CDC70000CDC70000CDC70000CDC700007F
:10013000CDC70000CDC70000CDC70000CDC700006F
:10014000CDC70000CDC70000CDC70000CDC700005F
:100150003DC0000051C0000065C0000079C0000033
:10016000CDC70000C1D40000CDC70000CDC700003E
:10017000CDC70000CDC70000CDC70000CDC700002F
:10018000CDC70000CDC70000CDC70000CDC700001F
:10019000CDC70000CDC70000CDC70000CDC700000F
:1001A000CDC70000CDC70000CDC70000CDC70000FF
:1001B000CDC70000CDC70000CDC70000564B4CF2A4
:1001C000205210B51A804DF628121A8000BF00BFC9
:1001D0000CF000FB514B4FF010621A60504A9A60CD
:1001E000504ADA60504A136813F4807304D14F49BF
:1001F0000B604FF4A85313604D4B1A78110703D5C9
:100200001A7842F008021A704A4B4B492A221A7097
:100210004A4A4B4B8B4204D252F8040F43F8040B6A
:10022000F8E7484B484900228B4202D243F8042B9E
:10023000FAE74649464A002352F8230041F82300D2
:1002400001336F2BF8D1434B434A802103F8011B44
:100250009342FBD1414B3D4A1A60414B8A221A70AE
:10026000A3F5805324225A70A0221A709A7992071B
:10027000FCD59A79D406FCD43A4A937903F00C035E
:10028000082B384BF9D103221A7140225A719A79FE
:100290009006FCD5334A9179324B4906FBD5324A58
:1002A000324911600221516020221A709A7902F0BD
:1002B0000C020C2AFAD12E4B2E4A1A602E4B2F4AD2
:1002C0001A6000225A60072243F8042C2C4AC3F813
:1002D0000C2D62B60CF02EFE144B1B68DA0705D508
:1002E00028480CF0FBFB284B284A1A60284B1B7847
:1002F0005B0609D5244C254B22689A4204D121483B
:100300000CF0ECFB002323600FF0E6FD0CF068FA24
:100310000CF096F9FEE700BF0E2005403080044047
:10032000823F04000100002B10D0034014D0034092
:1003300002D0074000E00740349BFF1FD436010085
:100340004088FF1F349BFF1F20A3FF1F0082FF1F59
:100350000000000000E400E05FE400E008ED00E0E1
:100360000050064000400640448004400000030165
:1003700004800440C010050014E000E0FF76010096
:1003800000002020A98A195F1CE00340A5C3945AED
:1003900000F00740FFFFFFFFFFFFFFFFFFFFFFFF32
:1003A000FFFFFFFFFFFFFFFFFFFFFFFFFFFFFFFF5D
:1003B000FFFFFFFFFFFFFFFFFFFFFFFFFFFFFFFF4D
:1003C000FFFFFFFFFFFFFFFFFFFFFFFFFFFFFFFF3D
:1003D000FFFFFFFFFFFFFFFFFFFFFFFFFFFFFFFF2D
:1003E000FFFFFFFFFFFFFFFFFFFFFFFFFFFFFFFF1D
:1003F000FFFFFFFFFFFFFFFFFFFFFFFFFFFFFFFF0D
:10040000FFFFFFFFFFFFFFFFFFFFFFFFDEF9FFFF23
:1004100010B5054C237833B9044B13B10448AFF33E
:1004200000800123237010BD349BFF1F00000000DB
:10043000D8360100084B10B51BB108490848AFF386
:1004400000800848036803B910BD074B002BFBD0A0
:10045000BDE81040184700BF00000000389BFF1F98
:10046000D8360100349BFF1F0000000038B5044659
:10047000104621700A491D460FF010FB01464FF04F
:100480007E500FF0BFFB07490FF008FBE56060608E
:10049000256165610CF0DEFCE061204638BD00BFDF
:1004A000DB0FC9400024744938B50446104621705A
:1004B00009491D460FF0F2FA01464FF07E500FF049
:1004C000A1FB06490FF0EAFAE5606060256165610D
:1004D0000CF0C0FCE06138BDDB0FC940002474495A
:1004E00038B503780446032B20D8DFE803F01A1848
:1004F0001002C16840690FF0C7F90D4905466068F0
:100500000FF080FB014628460FF07CFB38BD084900
:1005100040680FF077FBE1680FF0C0FA38BDC068A3
:1005200038BDC16840690FF0AFF938BD002038BD53
:100530000024744970B504460E460CF08BFC054649
:10054000E069281A0FF056FAE3682361E5616661F5
:10055000A061014660680FF055FB0146A06010489D
:100560000FF050FB0EF026FE0EF0C6FA0FF038F931
:10057000054601464FF07E500FF086F961690FF095
:100580008DFA2169064628460FF088FA0146304662
:100590000FF07CF9E0602046BDE87040FFF7A0BF97
:1005A000000080BF08B50E200BF024FF114B1B8804
:1005B000012B19D0104B1B88984213DB40F6FF71BA
:1005C0008842D4BFC3EB0001C3EB0101C1EB013191
:1005D000C3F57F630F33282091FBF3F1BDE808409A
:1005E0000CF08EBA0021F3E70146BDE80840142064
:1005F0000CF086BA609DFF1F009CFF1F10B50446DB
:100600000BF0FAFC204610BD70B44C88A04220D9F3
:1006100001230133DBB21CB2660031F8144084427E
:100620001D46F6D3A04211D005F10045013D965B71
:1006300031F8151032F81530401AF21A00FB02F0AA
:10064000641A90FBF4F4E01870BC7047905B70BCC7
:10065000704702260125E5E700280CDA064A4342E6
:1006600082FB0320DA17C2EB600000EB4000A3EB33
:100670008000C0F10C007047ABAAAA2AF0B40E8823
:1006800086420DD203F10043013B31F813508542FD
:1006900002D9F0BCFFF7B8BF32F81300F0BC7047C6
:1006A0001088F0BC704700BF094B1B880C2B09D881
:1006B000084A80B252F8232028B143F6FE739842CC
:1006C00003D9108C7047108870470349FFF79CBF0F
:1006D000869BFF1FE0110100E4130100374A3849EF
:1006E0001088384AF8B5384B12881B68834248DBBB
:1006F0009342A8BF134698420B60C8BF002342DD57
:10070000101AB0F5804FAABF9B03C3EB83330130AF
:1007100093FBF0F0FFF7C8FF2C4B2D4F1C883B6874
:10072000C0F3C61505FB04F47F2CA8BF7F249D42AF
:10073000064608D0274B1B88002B38D1264B1B8838
:10074000002B30D13D60254D2B689E4205D0214BBA
:100750001B885A1F032A1DD92E60214D2B689C42ED
:100760000ED0204B188848B11A4B1F4A1B88D35C07
:10077000834203D0C0B2E1B207F0B0FF2C60F8BDF5
:10078000F8BD034608609A42D4BFC0EB0203C0EB39
:100790000303B5E7144AD05C2030C0B206F07F01F5
:1007A00007F09CFFD8E7284608F00CF8CAE70E4A85
:1007B0002946D05C07F092FFC0E700BF009CFF1FF6
:1007C000589BFF1FB89DFF1F5C9DFF1F6C9BFF1F69
:1007D000B49BFF1F4A9DFF1FF69BFF1F809BFF1FBF
:1007E000F89BFF1F969DFF1F9889FF1F2DE9F04F73
:1007F000172089B00CF042FDAF4B186016200CF0AA
:100800003DFDAE4BAE4A1B8810600C2B00F03B81C7
:10081000AC4BAD4A19880093AC4B52F821400022F2
:100820001A70AB4BAB4D1B88AB4A2E88013B32F99B
:100830001370002E5CD0A94BA94A1B88A9491278D5
:10084000013B31F91380002A40F0DF8011200CF0C9
:1008500015FDA54B0193D3F800A00646B24540F321
:10086000DF80A24BDFF8A4921B88A14A012BD9F8A4
:100870000030B2F800B09F4A02922046C8EB03084D
:1008800000F09A820FF0B6F8029A52F82B100FF08F
:1008900005F9014600200EF0F7FF0FF0C5FACAEB8C
:1008A0000802B045B8BFB0469042CAEB080880F2D3
:1008B000968200FB0888013298FBF2F08E4BDFF83D
:1008C00050820293D8F80030034403EBD3735B10DB
:1008D000C8F800302B88012B12D1884BDFF834B2D6
:1008E0000393874BDBF8005004934FF0000A47E076
:1008F0007D4B0193DFF814927F4BDFF81482029353
:100900007E4B03931D460F200CF0B8FC2B689842D9
:10091000824641DA754A1288012A00F01D82744A23
:1009200005931288734D049220460FF063F8049AE1
:10093000DFF8E0B155F82210DBF800500FF0AEF808
:10094000014600200EF0A0FF0FF06EFAEF1B059B92
:100950005745A7EB0302B8BF5746FF1A9042BABFEC
:10096000013200FB0777474397FBF2F7D8F80020E6
:10097000634B0493BB1803EBD3735B10C8F80030D0
:10098000604B1B88013B032B00F2B082DFE813F0C1
:100990006301A901C4008601594B04931B68984266
:1009A00040F3C281514A1288012A00F0A682504ABF
:1009B000079311884F4A0691204605920FF01AF8C6
:1009C000059A0699DFF84CB152F82110DBF8005077
:1009D0000FF064F80FF028FA079B2F445745A7EB58
:1009E0000302A8BF5746FF1AD8F800309042BABF9A
:1009F00000FB07770132474397FBF2F73B4403EBD9
:100A0000D3735B10C8F80030BAE715200BF0F2FC86
:100A1000354B0193D3F800A00646B2453FF721AF0E
:100A2000354B0293D3F800A0B24580F289812F4B59
:100A3000DFF8D8901B882E4A012BD9F80030B2F885
:100A400000B02C4A03922046984400F070820EF0C9
:100A5000D1FF039A52F82B100FF020F80FF0E4F9B1
:100A6000B045CAEB0802A8BFB046CAEB08089042DE
:100A7000B6BF00FB088800FB08F8013298FBF2F0D3
:100A8000DFF88C801EE7204B1B78002B3FF4C0AEB4
:100A90000C4B0D4A198800930C4B52F8210001228F
:100AA0001A700EF0A7FF4FF07C510EF0F7FF0FF019
:100AB000BBF90446B5E600BFAC9BFF1F929DFF1F2C
:100AC000D49DFF1FB09BFF1F5889FF1F629BFF1F14
:100AD000A489FF1F049DFF1FCC150100AA89FF1FD9
:100AE000709DFF1FC0130100D89DFF1FE49BFF1FD7
:100AF000A09BFF1FE4150100D89BFF1F849DFF1FD3
:100B0000FC9CFF1F2E89FF1F489DFF1F509BFF1F4E
:100B10009C9DFF1F809DFF1F28460EF06BFFB24972
:100B20000EF0BCFF054650460EF064FFAF490EF0D4
:100B3000B5FF014628460EF0A9FE0FF075F90546EF
:100B4000CBF80050D9F800000EF054FFA6490EF083
:100B5000A5FF074630460EF04DFFA4490EF09EFF5C
:100B6000014638460EF092FE0FF05EF9C9F800001B
:100B70009F4AA04B168819889F4AA04B12681B8871
:100B80009F4FC6EB050E3544039EC6F800E0461A9B
:100B9000084404990D6001990E6002993E8808602E
:100BA0009A4280F289810025C3EB060E954974456F
:100BB0000F6880F27681611C9F4205FB01F50EF102
:100BC000010E95FBFEF5C0F2BE81BE42A8BF3E46B7
:100BD000F61A01FB06F494FBFEF49A4200F3368108
:100BE000BB42C0F23381884C20680EF003FF874976
:100BF0000EF054FF86490EF049FE0FF015F9A0F5EE
:100C0000FF531C3B082B98BF4FF40050D8F800301E
:100C1000184400282060C0F24281B0F5804F80F275
:100C200052817C4B1B781BB1B0F5005F40F05381C3
:100C3000794D2B78002B40F05481784D20682B683B
:100C4000714C984204D080B207F026FE23682B60D6
:100C500009B0BDE8F08F28460EF0CCFE70490EF0CA
:100C60001DFF054650460EF0C5FE6E490EF016FFFC
:100C7000014628460EF00AFE0FF0D6F80546CBF8DE
:100C80000050D9F800000EF0B5FE65490EF006FFE1
:100C9000074630460EF0AEFE62495FE728460EF08A
:100CA000A9FE5A490EF0FAFE054650460EF0A2FE85
:100CB0005D490EF0F3FE014628460EF0E7FD0FF009
:100CC000B3F80546CBF80050D9F800000EF092FEBC
:100CD0004E490EF0E3FE074630460EF08BFE5249B9
:100CE0003CE728460EF086FE50490EF0D7FE05463A
:100CF00050460EF07FFE4E490EF0D0FE01462846CB
:100D00000EF0C4FD0FF090F80546CBF80050D9F86E
:100D100000000EF06FFE45490EF0C0FE074630465B
:100D20000EF068FE424919E7D8F80030DFF810B13C
:100D300003EBD3735B10DBF80050C8F800301FE6FC
:100D4000DFF80081DFF80091D8F8003003EBD373AF
:100D50005B10C8F80030BDE5364A06931188364A64
:100D6000059120460492DFF8D8B00EF043FE049AB5
:100D70000599DBF8005052F821100EF08FFE0FF0AD
:100D800053F8EF1B069B5745A7EB0302B8BF574626
:100D9000FF1AD8F800309042BABF013200FB077743
:100DA000474397FBF2F73B4403EBD373234A049288
:100DB0005B10C8F80030E3E50EF01CFE029A52F812
:100DC0002B100EF06BFE0FF02FF8CAEB0802B045A7
:100DD000B8BFB0468242CAEB08083FF76AAD00FBD5
:100DE00008F898FBF2F069E5CDCC4C3FCDCC4C3EF9
:100DF000A689FF1F2C89FF1FAC9BFF1F5A9DFF1F59
:100E0000989BFF1FD49DFF1F8C89FF1F9A99193F44
:100E1000CDCC4C458A9EFF1FF59BFF1F2089FF1FED
:100E20003333733FCDCC4C3DCDCCCC3E6666663F74
:100E3000CDCCCC3DA09BFF1FE4150100FC9CFF1F07
:100E4000809DFF1F9C9DFF1F509BFF1F009B1B88C9
:100E5000002B3FF4C8AE2B1B002BB8BF5B42092B05
:100E600047DD05F500500130001B0EF0C3FD3B4986
:100E70003B4C0EF013FE054620680EF0BBFD3949D1
:100E80000EF00CFE014628460EF000FD0EF0CCFFE1
:100E9000D8F80030184400282060BFF6BEAE00220B
:100EA00013E09F4205FB04F5B8BF002195FBFEF55A
:100EB0004BDA91FBFEF490E6B242D4BFC3EB0205DD
:100EC000C3EB060570E643F6FF72274B22601B78E2
:100ED000002B3FF4ADAE04F0BDFE244B01221A708E
:100EE000ABE604F0B3FE00232B70A6E6D9F80000B1
:100EF0003EE64FF400501A4C88E61D491D4A069301
:100F000020460D8805920EF075FD059ADFF868B051
:100F100052F82510DBF800500EF0C0FD014600200D
:100F20000EF0B2FC0EF080FF2F44069B56E50EF04B
:100F300061FD039A52F82B100EF0B0FD014600201F
:100F40000EF0A2FC8AE51E4642E6B742D4BFC3EBD0
:100F50000701C3EB060104FB01F1AAE7CDCCCC3EAF
:100F60008C89FF1F9A99193F8A9EFF1FF59BFF1FCF
:100F7000A09BFF1FE4150100809DFF1F08B5244BB7
:100F80001B88FBB1234B1B78FBB1234B1B78E3B1D0
:100F9000224B1B78CBB1224B1B78B3B1214B22489B
:100FA0001A78C2B9214A2249008812880968024485
:100FB000B1EB620F09DD01221A706420BDE8084020
:100FC00004F05CBE174A117801B908BD1370BDE882
:100FD000084007F02BBC154A16490088128809689A
:100FE0000244B1EB620FF0DD00221A7007F01EFC24
:100FF000642004F043FE642004F040FE642004F00A
:101000003DFE4FF41670BDE808400BF045BF00BF31
:10101000069DFF1FE19DFF1FB29DFF1FB39DFF1F98
:10102000B49DFF1F849BFF1F989BFF1F5A9DFF1FAE
:10103000AC9BFF1FD49DFF1F38B5114C2320257892
:101040000BF0D8F90F4A42F82500131F02F1C40033
:10105000002253F8041F83420A44FAD123780A4934
:1010600007480A4C0133DBB2322B81FB025108BF27
:101070000023D217C2EB21120370226038BD00BFDB
:101080006E9BFF1F109CFF1F1F85EB517C9DFF1F58
:101090002DE9F04FB84CB94D2068B94F83B00EF030
:1010A000A9FCB8490EF0FAFC064610200CF0E6F850
:1010B0000EF0A0FCB4490EF0F1FC31460EF0E6FB58
:1010C0000EF0B2FE2988206088423B8843DA9E46B3
:1010D0005B1A7F2B4FF0000247DDD2015E1C92FBB2
:1010E000F6F2AA4EDFF8C882B6F800C0C8F80020B1
:1010F000BCF1190F00F0DF80BCF11A0F00F017816E
:10110000BCF11E0F00F020810126B146A04A1288D2
:10111000002A00F09D808842C0F207817045D4BF4C
:10112000C1EB0000C1EB0E009A42BABF02FB000007
:101130000133504390FBF3F3964A1360964B1888A3
:10114000C0B9964A1288AAB9954B197801B11A709C
:1011500003B0BDE8F08F9842D4BFC1EB0002C1EBF1
:1011600003029E465B1A7F2BB7DCC2EBC21292FBD6
:10117000F3F2B6E72988D4F800E0DFF80082DFF860
:10118000F8A171456CDCDFF818C29CF80020002A39
:101190002ED14FF0010B04288CF800B028D1002E7E
:1011A00040F094817D4B18880028D1D0B9F1000F10
:1011B000CED023682C883A88A34280F26581002330
:1011C000141B7E2C774DD5BFC3EB8313C3EBC31326
:1011D0005B00013493FBF4F42B680134A34203D089
:1011E000C0B2E1B207F07AFA2C6003B0BDE8F08F2C
:1011F000012800F0F680022800F0EB800328D1D10E
:10120000694B1B88092BCDD0002ECBD023682E88AC
:101210003A88B34280F27B810023961B7E2EDFF852
:101220008CA1D5BFC3EB8313C3EBC3135B000136A3
:1012300093FBF6F6DAF800300136B34203D0F1B290
:101240004A2007F04BFACAF80060ABE71646914611
:10125000BCF11E0F7FF472AF0022DFF858817EE0F0
:101260004F4B1A78002A3FF473AF002401281C70FA
:1012700000F0A480022840F00E81002E00F0A38030
:101280004A4D2B68002B00F09E800420214607F079
:1012900025FA424B2C60188800283FF459AFB9F169
:1012A000000F3FF455AFC0B2002107F017FA3D4BD5
:1012B00000221A604CE7DFF8FC8098F80020C2B1E9
:1012C000DFF8D890B9F800A0BAF1000F11D0DFF81C
:1012D000E89099F800B0934578D05FFA8AF07F21C2
:1012E00007F0FCF998F80030B6F800C089F8003033
:1012F00010E0DFF8C49099F800A0924566D0274B23
:101300000021187807F0EAF998F80030B6F800C024
:1013100089F800301E4B1A88002A97D0BCF11E0FA6
:1013200040F006810026B14619E00020FCE6DFF817
:10133000848098F80020002A0BBF012600264FF079
:1013400000094FF00109E1E6DFF86880104B98F8DA
:1013500000601A88B6FA86F676094FF0000998F808
:101360000030002B3FF4E8AE2988B7F800E0206891
:10137000C1EB0E03CFE600BFA49BFF1F0C9DFF1F18
:10138000089DFF1F9A99193FCDCCCC3E929DFF1F1F
:10139000C09DFF1F089CFF1FAA9BFF1FA29DFF1F50
:1013A000999DFF1F8C9BFF1F4A9DFF1F0C9CFF1FD9
:1013B000749DFF1F489DFF1F729BFF1F1EB1614D53
:1013C0002B68002B7BD1604B188865E70026B1465F
:1013D0009CE6002E3FF4E6AEDFF868A1DAF80020C4
:1013E0002EE0002E3FF4DEAEB7F80080F045D4BF0B
:1013F000C1EB0802C1EB0E02C1EB0808B8F17E0F89
:10140000DFF840A1D5BFC2EB8212C2EBC21252007C
:1014100008F1010892FBF8F8DAF8002008F1010859
:10142000424506D05FFA88F10120009307F056F993
:10143000009B1888CAF8008002287FF4DFAE42467D
:101440002168B5F800803888414559DA0021C8EB99
:101450000008B8F17E0FD3BFC1EB8111C1EBC11100
:1014600008F10108490091FBF8F808F101089045DE
:1014700006D05FFA88F10420009307F02FF9009B53
:101480001888CAF80080B9E69342D4BFC4EB0303BE
:10149000C4EB020394E6032827D12C4B1B88092BAD
:1014A00091D0002E8FD0274D2B68002B8BD04A2057
:1014B000214607F013F9244B2C601888ECE62146EE
:1014C00007F00CF9204B2C601888E5E640207F21BE
:1014D0008DE80C0007F002F9019B009A1888584526
:1014E0001CD002287FF48AAE76E704287FF46BAF25
:1014F000002E3FF468AF2146402007F0EFF862E786
:101500008142D4BFC8EB0101C8EB00019FE79342C1
:10151000D4BFC6EB0303C6EB02037EE6B8F80010A7
:10152000DAF800E0B7F800808E45FFF665AF5DE7BA
:101530002988B7F800E020680026C1EB0E03B14609
:10154000E9E500BF0C9CFF1FA29DFF1F4A9DFF1FE6
:1015500008B50F4B1B88022B0FD0032B12D0042B86
:1015600003D00C4B01221A7008BD7F21092007F01F
:10157000B5F8084B01221A7008BD7F21412007F001
:10158000ADF8EEE74021092007F0A8F8E9E700BF31
:10159000049CFF1FC49BFF1F38B51C4B1B881D2BD1
:1015A00026D01B4B1B88012B25D01A4A1A4B1488B6
:1015B0001B681A4AA342128818DB9342D4BFC4EBBB
:1015C0000303C4EB0203141B7F2CC6BFDB010134F1
:1015D000C3EBC31393FBF4F4114D2B689C4203D06F
:1015E000E1B2052007F07AF82C6038BD0023EAE765
:1015F0000C4B1C88F0E70C4B0C4A0D491B68126819
:101600000C689B1A1C1B84F30704E5E7929DFF1FDF
:10161000049DFF1F789DFF1F649BFF1F909DFF1F70
:101620005C9BFF1FA29BFF1FC89DFF1F2889FF1FF8
:10163000109DFF1F10B50F4C23685BB90E4B1B8824
:10164000022B11D0033B012B09D90C4A0023137044
:10165000236010BD0021052007F040F8EEE70021CF
:10166000092007F03BF8F0E70021412007F036F8A9
:10167000EBE700BF5C9BFF1F049CFF1FC49BFF1F89
:1016800008B5274B1B78ABB115200AF0B3FE254AED
:10169000254B128818601D2A15D0244A1288EAB1F9
:1016A000012A25D0224B1B78002B34D0BDE80840FE
:1016B000FFF7C0BF11200BF0E1FD1A4A1A4B128848
:1016C00018601D2AE9D11B4B1B78002BEAD0184B60
:1016D0001B780BB3BDE80840FFF75EBF164A1288BF
:1016E000002ADFD0154A1B6812889A42DADCEEE73E
:1016F0000F200BF0C3FD104B114A1B88106033B153
:10170000104B114A1B6812689B1A9842DFDD084B88
:101710001B78002BCAD108BDFFF71AFFDAE700BF1C
:10172000709DFF1F929DFF1F649BFF1F049DFF1F65
:10173000C49BFF1F489DFF1F049CFF1F789DFF1F38
:10174000109DFF1FC89DFF1F2889FF1F38B510205F
:101750000BF094FDC830B0F5FA7FC0F2C280B0F54E
:101760007A6F0146A8BF4FF47A6101F51673B3F59D
:101770007A6FA8BF4FF47A639BB289B2784A794CEA
:1017800011802220238007F02DF92188764D774C97
:10179000242007F027F90E200AF02CFE40F6FF71F6
:1017A000C8308842A8BF084620EAE07000F5FA6217
:1017B00083B28A42A8BF0A460220194622802B80A3
:1017C00007F010F92188042007F00CF917200BF01E
:1017D00055FD044616200BF051FDA042B8BF20462F
:1017E00000F1C801B1F5FA7F76DBB1F57A6FA8BFD9
:1017F0004FF47A6101F54873B3F57A6FA8BF4FF4DF
:101800007A639BB289B25A4A5A4C11800A202380CB
:1018100007F0E8F80C20218807F0E4F80B200BF023
:1018200005FB002862D011200BF028FD00F1C80153
:10183000B1F52F7F68DA40F214534FF42F714E4AFE
:1018400011804E4C0620238007F0CCF82188082018
:1018500007F0C8F800244FF4AF75E1B2484808F02B
:1018600007FE01348542A8BF05460C2CF5D10120A6
:101870000BF004FD044600200BF000FD323CA0F10B
:10188000320340496FF4957000FB03F300FB04F052
:1018900081FB034281FB0041DB17C017C3EB6223CE
:1018A000C0EB612003F5AF7200F5AF739342A8BFA0
:1018B00013469D42A8BF1D46A5F11401312932DC13
:1018C00040F26C7332213048304A018013602A2084
:1018D000BDE8384007F086B840F214534FF4FA716F
:1018E00091E740F24C434FF4FA7147E715200AF0B4
:1018F00081FD00F59671B1F52F7F9CDB41F25C23F1
:1019000099421FDD19469AE741F25C239942F9DCBE
:10191000194A00F5487089B2B0F52F7F118019DAA5
:101920004FF42F738DE740F23A72A5F5B975184B55
:1019300002FB05F583FB0523ED17A5EB631389B2C5
:101940003233C0E70C4A00F5617089B2B0F52F7FE1
:101950001180E5DB8342A8BF03469BB271E700BF5D
:101960000C9DFF1F089DFF1F009CFF1FB89DFF1FC0
:101970005A9DFF1F989BFF1F789DFF1F909DFF1F83
:10198000F49BFF1F67BBCF46B09DFF1F9489FF1FCD
:10199000B5814E1B2DE9F84F0C200AF0F7FC0C2006
:1019A0000BF0ACF9A14914200BF0B8F9A049A148FB
:1019B00008F0F0F9022103200BF046FA022104207E
:1019C0000BF042FA022105200BF03EFA022106201C
:1019D0000BF03AFA01210A200BF036FA0121092016
:1019E0000BF032FA01210D200BF02EFA01212820F4
:1019F0000BF02AFA012114200BF026FA02210B2009
:101A00000BF022FA01210C200BF01EFA0C20002111
:101A10000BF006FA04200BF009FA70B305200BF066
:101A200005FA044680B300242046834D287005F053
:101A3000F1FB2B78EBB9204606F0FEFF7F4B804987
:101A40001B88804D0988804A2970A3F5AF7140F248
:101A50003A7303FB01F382FB0312DB177B4E7C48D6
:101A6000A3EB621332335A21336008F03DFD90B985
:101A7000FEE7BDE8F84F08F09DB806200BF0D6F958
:101A80000028CBD10124D0E703200BF0CFF9B0FA26
:101A900080F04009C9E76F4A6F481268DFF800B26A
:101AA00000230121FEF700FD0B200BF0BFF9011E02
:101AB0000CBF012300238BF8003002D111200BF062
:101AC000C3F9DFF8A091654FDFF8D881644E002399
:101AD000C9F800303B60C8F800304FF0040A14E049
:101AE0000AF088FC3B68184438600AF0010080F076
:101AF000010004F0B3F83388002B14BF4B20DC2026
:101B00000BF0CAF9BAF1010A1BD00F200BF0B6FB9B
:101B1000D8F8003003440E20C8F800300AF06AFC00
:101B2000D9F800309BF800200344C9F80030152094
:101B3000002AD5D111200BF0A1FB3B681844386076
:101B4000D3E7D8F80030D9F8002046493868DFF8E4
:101B500058E1DFF858C1002BB8BF0333002AB8BFE3
:101B6000033292100A604049404A098812880028CE
:101B7000B8BF03309B10801038605F1A1944CEF84C
:101B80000070CCF80010DFF828E1394F3949C8F867
:101B90000030C2EB000C0244CEF800C03A600B608B
:101BA0000CB1FFF7D3FD33885BB94FF4FA7004F042
:101BB00065F804F04FF805F035FE4FF4AF600BF018
:101BC0006BF92D4B012404201C600BF02FF910B988
:101BD0002A4B28701C702A4B1B881C2B1CD0294CAC
:101BE00004F1C80523200AF005FC44F8040F012085
:101BF0000BF052F9A542F5D1234A244B1078187006
:101C000006F024FE04F022F845F6BF522049214890
:101C1000BDE8F84F0AF0A6B91F4B18880028DED09F
:101C20001E4BC0B2197806F059FDD8E7001B3746A5
:101C300040420F003C90FF1F8A9BFF1FB09DFF1F7B
:101C4000949DFF1FD49BFF1FB5814E1B9489FF1FDE
:101C5000F49BFF1F2489FF1F289DFF1F509BFF1F20
:101C6000569DFF1F689BFF1FA689FF1F2C89FF1F22
:101C7000D89BFF1FC89DFF1F8C9DFF1F769BFF1FDA
:101C8000929DFF1F0C9CFF1F149DFF1FFA9CFF1FBE
:101C9000A5050000A89DFF1FDC9BFF1FA29BFF1F47
:101CA000709DFF1F809DFF1F849DFF1FFC9CFF1FD9
:101CB000D89DFF1F2DE9F04F8BB007ADB54F2C46D7
:101CC0000AAE611BC9B2B44808F0D2FB3B8883421C
:101CD00094BF0020012004F8010BA642F1D1AF48C7
:101CE000AF4A9DF81C70AF4907709DF81E00AE4DBD
:101CF00010709DF820209DF82430AC4EAC4C0A703A
:101D00009DF82210297000253370257073B90029C1
:101D100040F00581A7491AB10B78002B40F0EC8107
:101D2000002800F0BF810223237005E0002A40F064
:101D3000A78005239F492370DFF8D0B2DFF8D08257
:101D40009DF81D209DF82100DFF8C892DFF8C8A299
:101D5000994D9A4F9A4E0B709DF81FC09DF8231015
:101D60009DF827309DF826E08BF8002088F80000C9
:101D70009DF82520297001203A70337089F800C041
:101D80008AF800E00BF07AFA8E4A8F4B116888428D
:101D9000CCBF012200221A7076DD8C4B1B88182BD9
:101DA00072D88B4AB2F800E00C3B0093BEF1000FF2
:101DB00072D1884A9BF800C092F800B098F8008071
:101DC00099F800209AF8009094F800A02C78ABEBDA
:101DD0004C0BC2EB0B0BA8EB880EDE44C9EB897BE6
:101DE000C9EB8B09DFF8F4B1F14497F800E0BBF8D8
:101DF00000B009EB44093478CE4404FB0BEE4FF0FD
:101E00000C09754C19FB0AEEC4F800E0B8F1000F9C
:101E10000BD036784EB1714E3688042E0CBF0EF1C1
:101E2000020E0EF1040EC4F800E06D4CDFF8EC91E8
:101E30002488B9F800A06B4EDFF8E4913688D9F811
:101E40000090009B033C04EB4404CAEBCA0A0EEB6F
:101E500084043444D144644E0C3C56F829601C443C
:101E6000A319BCF1000F28D02C7834B3002A5AD122
:101E7000B8FA88F85D4C4FEA581884F8008023E0DF
:101E8000062323704B4957E7514AB2F800E000237C
:101E90000093BEF1000F8CD0BEF1010F47D0BEF110
:101EA000020F00F0C1804C4C9BF800C099F8002054
:101EB00098F80080D4F800E0A8E74C4C0025257085
:101EC0000AB13A781ABB0022494C8842227049492B
:101ED000C4BF494AC2F800E00A68934213D0474A97
:101EE000474C106805900598206012680692454C92
:101EF000069A24880B60121AA24284BF424A1360D9
:101F00000BB0BDE8F08F3E483C4A0068EDE7BCF1FD
:101F1000000FD8D1B8F1000FD5D10122D4E70423A6
:101F20002370244908E7314A00241470CBE7294A7A
:101F30009BF800C092F800E098F8008099F8002023
:101F400094F800B09AF800902C780194AEEB4C0E07
:101F5000C2EB0E0EA8EB88047444C9EBC909D9443E
:101F6000A31EDFF878A0DFF8BCE0019C97F800B072
:101F70005EF829E0BAF800A096F8009003EB44045C
:101F80005C4409FB0A4909F11809134CCE44C4F812
:101F900000E03BE7B09DFF1FF49BFF1FB29DFF1FBA
:101FA000B39DFF1FB49DFF1FB59DFF1FB69DFF1F73
:101FB000019DFF1F0A9DFF1FE29DFF1FE39DFF1F65
:101FC000989DFF1F9489FF1F489DFF1F929DFF1F33
:101FD000609BFF1FA889FF1F509DFF1FB29BFF1F23
:101FE000649DFF1F709BFF1F14120100C29DFF1F05
:101FF000C39DFF1FBC9BFF1FCC9DFF1FCC9EFF1FDF
:10200000E09BFF1FA09DFF1FD09DFF1FDE9DFF1FB8
:10201000E09DFF1FDF9DFF1FE19DFF1F889DFF1FAC
:10202000089CFF1F94150100374A9BF800C092F8E6
:1020300000B0247899F8002098F800800394ABEB66
:102040004C049AF80090314B95F800A0CDF804A00C
:10205000A8EB880BA41A5C444FF0050B1BFB094B43
:10206000039C97F800A0CDF808A0C9EBC909B3F804
:1020700000A009EB0403BDF80490029C0BF1050BD2
:102080001EFB09BE96F800B0DFF8A490A6440BFB37
:102090000AEE59F823901E4C0EF10C0ECE44C4F8F3
:1020A00000E0B3E65FBB0B78012B2BD9194A2370F4
:1020B0001288002A3FF440AE174A1288013A92B2C1
:1020C000062A3FF639AE154A1278002A3FF434AE9C
:1020D000134A1268012A7FF42FAE1248124A006890
:1020E000124E82FB0025C217C2EB650202EB4202D0
:1020F000A0EB820232801FE6032323701CE601233B
:10210000237019E63B4617E6A889FF1FB29BFF1F05
:10211000509DFF1FDC9DFF1F169DFF1F029CFF1F90
:102120008C9DFF1FD09DFF1FABAAAA2A549DFF1FA5
:10213000BC1701002DE9F04F3A4B1B788BB0002BF8
:102140006AD10E200AF056F90DF054FC01463648CB
:10215000364E374DFEF7EEF93348FEF7C1F90DF074
:1021600063FE80F30C003060FFF7A4FD2C68012CA7
:102170007AD0022C00F0AB82032C00F0B9832D4EF4
:1021800033682D4A2D4E0993099B316812882C4CD7
:10219000591A013A9142236000F29482294E326822
:1021A0009A1A0D2A00F28782274E32689A1A132A49
:1021B00000F27C82254E32689A1A252A1AD9244BBD
:1021C0001B88002B40F06881224B1B78002B40F0CD
:1021D0006381FEF731FF204B1B881B3B9BB2022B18
:1021E00004D81E4B1B78002B40F0598103F058FD9A
:1021F000236833601A4D2A689B1A502B00F2128212
:10220000184B1B88012B00F02A8206F0FBFA06F01F
:1022100029F90BB0BDE8F08F07F054FB0BB0BDE817
:10222000F08F00BF8A9BFF1F289DFF1F5C9DFF1F33
:102230008C9DFF1FCC9EFF1F9089FF1FFC9BFF1FE3
:10224000249DFF1FEC9BFF1FCC9BFF1FD09BFF1FFC
:10225000069DFF1F849BFF1F929DFF1F489DFF1F30
:10226000189DFF1F609DFF1FDFF82893A34AB9F850
:1022700000001378834204D0C3B21846137006F0EE
:10228000FDF9DFF80C839E4AB8F8003011789942C6
:1022900004D09C4F3978002940F0FD869A4A336873
:1022A00012889A4E9A42C0F2FF80994A1278002A08
:1022B00040F0FA80DFF8E0A2BAF8003023B9954B7D
:1022C0001B88002B00F0FC84934A944B11881B88D8
:1022D000934A0B4412685B109342924A126880F250
:1022E0009E8400219342B4BF01230B4604910093C6
:1022F000ACBF4FF0010B8B4605910E200AF07AF827
:10230000894B8A4A1B68176803930133A7F252323C
:10231000002B8446029240F3CF86802BA8BF8023F7
:10232000834A844912780191002A00F0C780097815
:10233000914200F0C380B8F80010DFF854E29942EF
:1023400001F0A7806F49AEF800307B4B4FF0010ED3
:1023500081F800E01978DFF844E2019B8EF8001064
:102360001A70009B002B00F01B81BAF80030002B84
:1023700000F01681714B1B685A1C002A40F3A0869E
:10238000802A00F39C866E4C6E496F482488098829
:1023900000682144B0EB610FC1F2EE82A3F1480264
:1023A0000F2A02D8473BA9F800300E200AF022F885
:1023B0006FF454731F44874202DC644B00221A708E
:1023C00000200AF05BFF624A624B1168624C1B8876
:1023D0008842D4BF002201222270002B00F0168414
:1023E0005E4B1C78944240D088423EDD5C490C78BC
:1023F000002C00F017875B4991F800C0BCF1000F7A
:1024000040F00E87584F0097584F59480297564F43
:10241000007887F800C0554F4FF0010E87F800C0D4
:1024200081F800E0002841F0B48052490978002981
:1024300000F0D887504903910C460978002940F0F4
:10244000CE874E48494F007839700121029721709C
:1024500058B1454843490090002008700099029FF8
:102460000870039901243C7008701A70444B1B8853
:10247000A3F11B02012A40F2E9851D2B7FF480AEF7
:102480003E4F3B78002B41F04B803E4C2378002B95
:1024900040F08984237073E6FEF770FD99E62B689F
:1024A000012B7FF4A3AEA3E63168374A0691069864
:1024B0003649106002220B602A60FBE61E49DFF8F5
:1024C000DCE0097800293FF448AF9EF80000814223
:1024D0003FF443AF03984B2840F3A2871833802B77
:1024E000B8F80000A8BF802398423FF436AF2848D0
:1024F00003800448012303702FE700BFFA9CFF1FED
:10250000D49BFF1F769BFF1F009CFF1FCC9EFF1FCD
:10251000849BFF1FF29BFF1F989BFF1F5A9DFF1F6D
:10252000AC9BFF1FD49DFF1FCC9DFF1F689BFF1F0F
:10253000C29DFF1FB89BFF1FC39DFF1F509DFF1F24
:102540000C9DFF1F089DFF1FA49BFF1F009DFF1FE9
:102550009489FF1F169DFF1F9E9BFF1F549BFF1F0B
:10256000E19DFF1F589DFF1FA49DFF1F029CFF1FA1
:10257000E29DFF1FDE9DFF1F559BFF1F489DFF1F14
:10258000929DFF1F729BFF1FC89BFF1F209DFF1F77
:10259000949DFF1F149DFF1FC09BFF1FB99BFF1F32
:1025A000029B9C45BFF601AF864B1B88002B3FF476
:1025B000FCAEBBF1000F7FF4DDAE834B1B881BB17B
:1025C000059B002B7FF4D6AE049B002B3FF4EDAEB1
:1025D0007E4B1A78002A7FF4E8AEDFF8649299F80F
:1025E000004001221A70002C40F03783784B1B7892
:1025F000002B02F03780774B1B78002B02F0028310
:10260000754B1B78002B7FF4D0AE744B1B78002BDE
:102610003FF4CBAEB8F8003071490A3BA8F800305F
:102620000A70C2E604F03EFE6E4B1B7873B96E4B27
:102630001B785BB96D4B1B7843B96D4B1B782BB97D
:102640006C4B1B7813B903F001FB01E003F00AFBAC
:1026500023682B60684B1B88012B7FF4D6AD674A3B
:10266000674B116867481A78A1F118032A2101FB0A
:1026700003F10160002A00F0B382634C23689942A1
:1026800000F35C8310DA61480278002A40F03E874C
:102690005F4A1068D0F17F0048BF033080100130DE
:1026A0001B1A994242F3428621609BE2FEF7E8FF43
:1026B000236833607EE5FEF799F8FEF7E9FC2368AE
:1026C000336071E5FEF70AF82368336066E5514A26
:1026D00034681188A14204DB464B1B78002B00F0C4
:1026E0005D834D4E4D48336807934D4B079A006804
:1026F0001B88121A9A4200F2A980002B00F0A680D3
:10270000484B1A88002A3FF43BAD474B47481B68AB
:102710000088A342B8BF2346994241F32681444B27
:102720001960DFF8208188F80020344FFDF7D6FFCC
:1027300038687F2840F370853E4B7F3883FB00323A
:10274000C317C3EB620303EB4303A0EB83007330B7
:10275000394B01931B883860002B40F08C86234B4B
:1027600000931B78002B00F0CD83344C2378002B92
:1027700000F0C883DFF8D090DFF8B8A04FF0000B6E
:102780000CE003F17300C0B298F8001005F0CEFF22
:1027900023780BF1010B5B4540F3B4833B6859F898
:1027A000040F1844A0F17F038AFB0321DA17C2EB60
:1027B000610202EB42027F28A3EB8203E1DCFDF71A
:1027C0004BFFE0E7F29BFF1F1C9DFF1F009DFF1FBB
:1027D000DE9DFF1FDF9DFF1FE09DFF1FE19DFF1F8F
:1027E000769BFF1F029CFF1F589DFF1FA49DFF1F8C
:1027F000559BFF1F849BFF1F609DFF1FD09DFF1FE8
:10280000C49BFF1FBC9DFF1F7C9BFF1FA59DFF1F3F
:102810005C9BFF1F009CFF1FCC9EFF1FC89BFF1FE0
:10282000F09BFF1F749BFF1F209DFF1FB89DFF1F84
:10283000589BFF1FABAAAA2AA89BFF1F5489FF1F02
:10284000019DFF1FE69BFF1F2C89FF1F554B564A1A
:102850001B681088554AA342B8BF2346994200F32B
:102860008482534C12888342A8BF03462360002A07
:102870007FF457AF9942C8BF134640F37D82401A98
:10288000B0F5804FAABF9B03C3EB8333013093FBAA
:10289000F0F0FDF709FFC0F3C6100DF0ABF8454BA3
:1028A000044618880DF0A6F84349074620460DF067
:1028B000F5F8014638460DF0F1F821460CF0E6FF38
:1028C0004FF07E5104460DF087FA002841F0318028
:1028D0003A4920460DF09EFA002840F054862046E2
:1028E0000DF0C8FAC0B2DFF8F48088F800001CE7E9
:1028F000334B34681988A14274DD324B1B78002BAE
:1029000070D1DFF8DC9099F800007F2840F3FA8559
:10291000A3F155337F3803F1004383FB0032C31723
:10292000C3EB620303EB4303A0EB83007330264B3E
:1029300001931B88C0B289F80000002B40F0EB87A0
:10294000224B00931B78002B00F09984204C2378B5
:10295000002B00F094841F4FDFF87C804FF0000ABA
:102960000AE003F17300C0B205F008FF23780AF112
:10297000010A534540F3838457F8043F99F8000057
:102980001844A0F17F0388FB0321DA17C2EB610230
:1029900002EB42027F28A3EB8203E2DCFDF75CFE40
:1029A000E1E700BF209DFF1FB89DFF1F749BFF1F25
:1029B000589BFF1FC49DFF1FCDCCCC3D0000FE42A5
:1029C000009CFF1F849BFF1FA89BFF1FA49DFF1F50
:1029D0005489FF1F2C89FF1FABAAAA2AE69BFF1F61
:1029E0004C9DFF1FB84F38687F2840F3CC81B74B10
:1029F0007F3883FB0032C317C3EB620303EB43034F
:102A0000A0EB83007330DFF8249399F800A082458F
:102A100000F01F82AE4B1B88002B43D1AD4AAE485D
:102A200012680088914205DC8242D4BFC1EB0203E8
:102A3000C1EB0003411AB1F5804FA6BF9B030131E2
:102A4000C3EB833393FBF1F0FDF72EFEC0F3C6100A
:102A50000CF0D0FFA14B044618880CF0CBFFA04926
:102A6000804620460DF01AF8014640460DF016F853
:102A700021460CF00BFF4FF07E5104460DF0ACF9EF
:102A8000002840F0C286974920460DF0C3F900287F
:102A900040F0768520460DF0EDF9C0B2DFF8908267
:102AA00088F80000BAF17F0F40F3B2838748AAF19B
:102AB0007F0A80FB0A304FEAEA73C3EB600000EB49
:102AC0004000AAEB80007330874B00931B78C0B2A4
:102AD00089F80000002B40F01283844B03931B788D
:102AE000002B40F0F584824B02931B78002B40F0C2
:102AF0003487804B0193029B1B78FBB17E4B1B8874
:102B0000012B00F00086022B00F05987032B01F007
:102B1000EB80042B01F0EB82052B01F00784062BE0
:102B200001F06085072B01F0D185082B02F02A8087
:102B3000092B02F02F810A2B02F08282009B1B7866
:102B4000002B00F05F84019B6A4C1988002900F07B
:102B5000B58438687F2840F3CF825C4B7F3883FB95
:102B60000032C317C3EB620303EB4303A0EB830004
:102B700073303860002940F06484009B1B78002B80
:102B800000F072815D4C2378002B00F06D81DFF83E
:102B9000A4A1DFF89C814FF0000B0CE003F173005F
:102BA000C0B298F8001005F0C1FD23780BF1010BBD
:102BB0005B4540F359813B685AF8040F434A184477
:102BC000A0F17F0382FB0321DA17C2EB610202EB63
:102BD00042027F28A3EB8203E0DCFDF73DFDDFE747
:102BE000474B1960474B1B68A92202FB03F3002BDC
:102BF000BCBF03F57F533F339B13543B194481F310
:102C00000C01282009F07CFFFFF7FFBA384C3E4842
:102C10003549364A237003700B70137026E49342D3
:102C20004FF0000B80F2B2800123CDF800B0CDF858
:102C300014B00493FFF761BB344B1B78002B7FF477
:102C4000B4AB039B324A243B83F34703D9B25B20E6
:102C5000136005F043FD99F80040032C30D1DFF8F4
:102C6000D88098F80030002B42F02181294F3B7822
:102C7000002B42F00F81254C2378002B42F0FD8081
:102C8000254B1B78002B42F0EB80244A1380244B09
:102C90001B78002B42F017810D4B7F221A8098F889
:102CA00000306BB93B785BB923784BB91D4A7F2163
:102CB0000720138005F012FD7F210B2005F00EFD8B
:102CC000194B1F68FFF771BBD09DFF1FABAAAA2A43
:102CD000749BFF1F589BFF1FB89DFF1FC49DFF1FC4
:102CE000CDCCCC3D0000FE42A49DFF1F559BFF1F95
:102CF000029CFF1FA89BFF1F169DFF1F5489FF1FEB
:102D00007C9BFF1F8C89FF1F589DFF1FE19DFF1FAC
:102D1000949BFF1FE09DFF1FDF9DFF1FF69BFF1F82
:102D2000E29DFF1F4A9DFF1F689BFF1F4C9DFF1FD9
:102D3000E69BFF1F2C89FF1FDE9DFF1FB04A107806
:102D4000002840F04383AF4A1268D2F17F0248BFA7
:102D5000033203EBA202531CAB4A23609942B8BF73
:102D60001160FFF63FAF19463CE7A84B1288196087
:102D7000002A7FF4D6AC0B469842D4BFC1EB0003C7
:102D8000C1EB03037BE5FDF767FC3CE60123CDF8CF
:102D900010B0CDF800B00593FFF7AFBA01232B6058
:102DA0009B4EFFF7EDB99B4B6A20198805F01AFE80
:102DB0003B782370FFF7E4B9029B1B78FBB1964B7D
:102DC0001B88012B00F01884022B00F07686032B61
:102DD00001F00080042B01F0AF81052B01F02A8265
:102DE000062B01F01484072B01F0C085082B01F09D
:102DF0007D86092B01F0EF870A2B02F0B281019B3F
:102E00001B88002B00F02683009B1B783BB9039B9B
:102E10001B7823B9029B1B78002B00F054877F4B53
:102E20001B78002B00F035817D490B78082B00F2D0
:102E300030817C483A6800687B4C0133DBB25F1E0E
:102E4000101A44F827000B70784B3468198889F8F9
:102E500000208C426E4E7FF793A93268744B089223
:102E6000089A1A60FFF78CB9039B1B78002BA3D03C
:102E70003B68A3F10C007F2840F327836D488B3B10
:102E800080FB0320DA17C2EB600000EB4000A3EBED
:102E9000800303F17300DFF8AC81C0B298F8001032
:102EA00005F044FC009B1B78002B85D05C4C2378FC
:102EB000002B81D0DFF890A14FF0000B0CE003F164
:102EC0007300C0B298F8001005F030FC23780BF1C5
:102ED000010B5B457FF770AF3B685AF8040F554A0A
:102EE0001844A0F18B0382FB0321DA17C2EB6102C5
:102EF0000C3802EB42027F28A3EB8203DFDCFDF7F4
:102F0000ABFBDEE7454B1B78002B40F0A9823B680A
:102F1000494A1278002A45D0A3F10C007F2840F3DB
:102F2000EE82444A8B3B82FB0321DA17C2EB61023B
:102F300002EB4202A3EB820303F17300C0B298F8E4
:102F4000001005F0F3FB009B1B7853B3344C23783F
:102F50003BB3DFF8F490DFF8DCA04FF0000B0BE0A0
:102F600003F17300C0B298F8001005F0DFFB23787E
:102F70000BF1010B5B4514DD3B6859F8040F184455
:102F8000A0F18B038AFB0321DA17C2EB61020C3834
:102F900002EB42027F28A3EB8203E1DCFDF75CFB3E
:102FA000E0E73B68254A1278FAB11B4A1288012AE9
:102FB00000F02E84022A00F00186032A00F08387A5
:102FC000042A01F0E080052A01F01882062A01F0A7
:102FD0002A83072A01F01984082A01F05786092A52
:102FE00001F09B860A2A02F08880019A1288002A42
:102FF00000F04882124903220B702A60FFF7C0B824
:10300000A59DFF1F5C9BFF1F7C9BFF1F589BFF1F05
:10301000CC9EFF1FA29BFF1F169DFF1F589DFF1FE9
:103020005489FF1F789BFF1F3089FF1F009CFF1FE3
:10303000749EFF1FABAAAA2A559BFF1F029CFF1F6D
:103040004C9DFF1FE69BFF1F2C89FF1FB04F3B7855
:10305000002B3FF41AAAAF4C207802F071FEAE4B61
:103060001B78002B00F0748223887E2B00F2708284
:10307000AA4A0133108899B22180002800F0788292
:10308000C9B2C0B2A64C05F029FB3B782370FFF70C
:1030900077B83A68D8E6DBB21846137005F0FCFA48
:1030A000A04BA1491A46A14B184600230B703B7058
:1030B00013700370FFF7F2B80123FFF731B98024D2
:1030C0009B499C4B9C4A09881B8812680B44B2EBB5
:1030D000630FBFF66AA98E4B1B78002B40F0DF818F
:1030E000B8F80030954AA3423FF45FA9944B14808E
:1030F00001221A70FFF759B9FDF7AEFA39E5914B85
:1031000001931B88002B42F00B81884B03938E4B5D
:1031100002938E4C23786BB3DFF84082DFF830A245
:103120004FF0000B09E003F17300C0B205F026FB7D
:1031300023780BF1010B5B451CDD58F8043F99F82F
:1031400000001844A0F17F038AFB0321DA17C2EBC9
:10315000610202EB42027F28A3EB8203E3DCFDF76E
:103160007BFAE2E7784B029305F008FB009B1B78A3
:10317000002BCED1039B1B78002B3FF4BCAC99F8FD
:103180000030A3F10C007F2840F3B68170488B3BE0
:1031900080FB0320DA17C2EB600000EB4000A3EBDA
:1031A000800303F17300C0B205F0E8FA009B1B78BE
:1031B000002B00F09681654C2378002B01F04B82A8
:1031C000DFF89881DFF888A14FF0000B0AE003F1E7
:1031D0007300C0B205F0D2FA23780BF1010B5B4506
:1031E0007FF789AC58F8043F99F800001844A0F123
:1031F0008B038AFB0321DA17C2EB61020C3802EB66
:1032000042027F28A3EB8203E1DCFDF725FAE0E729
:103210005046FDF721FA57E4FDF71EFAFFF798BA7A
:10322000002008704B49087840B13E490091097868
:10323000002900F0AB81009F0021397046490978D0
:1032400000297FF4F7A8002C40F0CC80002840F043
:10325000C9802F4C334F94F800E0344C03943A4C1F
:103260000294324C30492070374C00970870387007
:103270002070BEF1000F7FF4EFA8FFF7F6B82B4BDC
:103280001B78002B6CD099F80030A3F10C007F283C
:1032900040F37B832E4A8B3B82FB0321DA17C2EB80
:1032A000610202EB4202A3EB820303F17300C0B29E
:1032B00005F064FA009B1B78002B51D0234C237837
:1032C000002B4DD0254FDFF888804FF0000A09E031
:1032D00003F17300C0B205F051FA23780AF1010A34
:1032E00053453DDD57F8043F99F800001844A0F11C
:1032F0008B0388FB0321DA17C2EB61020C3802EB67
:1033000042027F28A3EB8203E2DCFDF7A5F9E1E7A7
:10331000489DFF1FA29BFF1FE39DFF1FDC9BFF1F1C
:10332000729BFF1FA49DFF1F589DFF1F559BFF1FF2
:103330000C9DFF1F089DFF1FA49BFF1F949DFF1F57
:10334000769BFF1FA89BFF1F029CFF1F5489FF1F36
:10335000ABAAAA2AE29DFF1FDE9DFF1F2C89FF1F3B
:10336000924B1B78FBB1924B1B88012B00F03886E7
:10337000022B00F03287032B01F0AB80042B01F00D
:103380005D81052B01F09783062B01F03084072B1C
:1033900001F0BC85082B01F07B86092B01F08887A2
:1033A0000A2B01F06587019B1B88002B00F0BC8273
:1033B000804B1B78002B40F0B2827F4B7F4A1988EC
:1033C00034680020012310602B6042E50130C0B258
:1033D000022886BF002111701070194602E403987C
:1033E000002101707649097800293FF43EA86F4911
:1033F00002910978002900F01687029800210170D7
:10340000FFF733B8039B1B78002B7FF49CAB029B28
:103410001B78002B7FF497AB019B1988FFF799BBB2
:10342000243B002BB8F8000040F3478498423EF458
:1034300094AF9BB26348A8F8003001230370FEF7F5
:103440008CBFDFF88481C0B298F8001005F06EF9E7
:10345000FFF793BB5C4B3878197805F067F9D3E434
:103460007F21402005F03AF95849594A3B680B60E2
:10347000002111704CE5C0B298F8001005F056F923
:10348000FFF76DB9D8B298F8001005F04FF93B6816
:10349000B0E5504BDFF85CE11978FEF75EBF4B2CCE
:1034A00040F34A821834802CB8F800304A4AA8BF4A
:1034B0008024A3427FF41AAEFEF777BF99F800008C
:1034C00005F05CF92188FFF744BBFDF7C5F8E2E49D
:1034D000424B01931B88002B7FF444AE334B029385
:1034E0004DE6029B1B78002B7FF408AB039B1B78F7
:1034F000002B7FF428AB8FE7FDF7AEF853E6FDF71E
:10350000ABF81BE5FDF7A8F8FFF711BA0132D2B20C
:10351000022A40F23D82002202701946FFF762BB88
:103520002F4C207802F00CFC2E4B1B781BB123880B
:103530007E2B41F23B802C4B1B7823B12388284AF9
:10354000002B41F05880294C3B782370FEF718BEC1
:10355000254B1B78002BF6D02388214A002BF2D074
:103560002349013B088899B2118000287FF488AD77
:10357000C8B21E4C05F026F93B782370FEF700BE5A
:103580007F20FFF78BBA7F20FFF7ADB9074F0949BE
:1035900002974FF0000C81F800C0009F02994FF095
:1035A000010E87F800E081F800C047E6029CFF1F8B
:1035B000169DFF1F589DFF1F009CFF1F589BFF1F5C
:1035C000489DFF1F769BFF1FE69BFF1F789BFF1FF9
:1035D0005489FF1FC39DFF1F949DFF1FA89BFF1FC2
:1035E000A29BFF1FE39DFF1FE29DFF1F729BFF1F1A
:1035F000DC9BFF1FB99BFF1FDFF8B0A33868BAF848
:103600000030E54AE54CC31A82FB031ED917C1EB13
:103610006E0101EB4101A3EB810303EB430354F87B
:10362000233018447F2840F3C9847F3882FB00325E
:10363000C317C3EB620303EB4303A0EB83007330B8
:10364000DFF86C83DFF86CB398F80010C0B205F0B7
:103650006DF8BBF80030022B7FF6D1AB3968BAF8B1
:103660000030CD4ACB1A82FB030ED817C0EB6E0098
:1036700000EB4000A3EB800303EB430304EB830365
:10368000586808447F2840F320877F3882FB003247
:10369000C317C3EB620202EB4202A0EB820073305D
:1036A000C0B298F8001005F041F8BBF80030032BC9
:1036B0007FF6A5AB3968BAF80030B74ACB1A82FB5F
:1036C000030ED817C0EB6E0000EB4000A3EB8003A5
:1036D00003EB430304EB8304A06808447F2840F312
:1036E0006B817F3882FB0032C317C3EB620202EBAF
:1036F0004202A0EB8200733098F80010C0B205F0CF
:1037000015F8FFF77CBBDFF8A4A299F80000BAF81F
:103710000030A14AA14CC31A82FB031ED917C1EB8A
:103720006E0101EB4101A3EB810303EB430354F86A
:10373000233018447F2840F33D847F3882FB0032D9
:10374000C317C3EB620303EB4303A0EB83007330A7
:10375000DFF860B2C0B205F011F8BBF80030022B00
:103760007FF6ECA999F80010BAF800308A4ACB1A13
:1037700082FB030ED817C0EB6E0000EB4000A3EBFA
:10378000800303EB430304EB8303586808447F285A
:1037900040F397867F3882FB0032C317C3EB620287
:1037A00002EB4202A0EB82007330C0B204F0E6FFED
:1037B000BBF80030032B7FF6C1A999F80010BAF8C6
:1037C0000030754ACB1A82FB030ED817C0EB6E008F
:1037D00000EB4000A3EB800303EB430304EB830403
:1037E000A06808447F2840F3CA807F3882FB0032FB
:1037F000C317C3EB620202EB4202A0EB82007330FC
:10380000C0B204F0BBFFFFF799B90120FFF746B93A
:10381000DFF898A16049BAF80020604C9A1A81FB41
:10382000020ED017C0EB6E0000EB4000A2EB80024E
:1038300002EB420254F8220018447F2840F3C2836E
:10384000A0F17F0381FB0321DA17C2EB610000EBDB
:103850004000A3EB80007330DFF858B198F80010F7
:10386000C0B204F063FFBBF80030022B50D93968B6
:10387000BAF80030484ACB1A82FB030ED817C0EBC7
:103880006E0000EB4000A3EB800303EB430304EB6B
:103890008303586808447F2840F37E867F3882FB84
:1038A0000032C317C3EB620202EB4202A0EB8200BC
:1038B0007330C0B298F8001004F038FFBBF8003045
:1038C000032B25D93868BAF80030334AC31A82FB73
:1038D000031ED917C1EB6E0101EB4101A3EB81037C
:1038E00003EB430304EB8304A36818447F2849DDFA
:1038F0007F3882FB0032C317C3EB620202EB420245
:10390000A0EB82007330C0B298F8001004F00EFFF4
:103910003B68FFF76ABB04F031FFFFF711B80021E5
:10392000402004F0DBFE48E599F8000004F026FF93
:103930003EE50120FEF7D7BF243C002CB8F800304C
:1039400040F35685A3423EF430ADA4B2144BA8F820
:10395000004001221A70FEF728BD124B01931B880C
:10396000002B7FF401ACFFF7C6B80F498342A8BF14
:1039700003460B60FEF7D5BE1446FFF7ACBBFCF761
:103980006BFE3DE7FCF768FEBDE7FCF765FE8EE4E5
:1039900002701946FFF726B9ABAAAA2A3013010014
:1039A000769BFF1FA89BFF1F589BFF1F549DFF1F67
:1039B000E69BFF1F889BFF1FFCF74EFE9CE6DFF88F
:1039C0001CA399F80000BAF80030C24AC24CC31ACE
:1039D00082FB031ED917C1EB6E0101EB4101A3EB82
:1039E000810303EB430354F8233018447F2840F34A
:1039F000C7837F3882FB0032C317C3EB620303EB3C
:103A00004303A0EB83007330DFF8D4B2C0B204F0FC
:103A1000B5FEBBF80030022B7FF690A899F8001095
:103A2000BAF80030AB4ACB1A82FB030ED817C0EBB2
:103A30006E0000EB4000A3EB800303EB430304EBB9
:103A40008303586808447F2840F301867F3882FB4F
:103A50000032C317C3EB620303EB4303A0EB830005
:103A60007330C0B204F08AFEBBF80030032B7FF63F
:103A700065A899F80010BAF80030964ACB1A82FB74
:103A8000030ED817C0EB6E0000EB4000A3EB8003E1
:103A900003EB430304EB8304A06808447F287FF70B
:103AA0006EAF7F3882FB0032C317C3EB620303EBB8
:103AB0004303A0EB83007330A2E6DFF820A238684E
:103AC000BAF80030834A844CC31A82FB031ED9170C
:103AD000C1EB6E0101EB4101A3EB810303EB430357
:103AE00054F8233018447F2840F371837F3882FBD9
:103AF0000032C317C3EB620303EB4303A0EB830065
:103B00007330DFF8E081DFF8D8B198F80010C0B268
:103B100004F00CFEBBF80030022B7FF670A9396868
:103B2000BAF800306B4ACB1A82FB030ED817C0EBF1
:103B30006E0000EB4000A3EB800303EB430304EBB8
:103B40008303586808447F2840F374857F3882FBDC
:103B50000032C317C3EB620303EB4303A0EB830004
:103B60007330C0B298F8001004F0E0FDBBF80030EC
:103B7000032B7FF644A93868BAF80030554AC31AB7
:103B800082FB031ED917C1EB6E0101EB4101A3EBD0
:103B9000810303EB430304EB8304A36818447F28E9
:103BA0007FF70AAF7F3882FB0032C317C3EB620393
:103BB00003EB4303A0EB830073309DE5DFF81CA10A
:103BC0004449BAF80020444C9A1A81FB020ED017DF
:103BD000C0EB6E0000EB4000A2EB800202EB420261
:103BE00054F8220018447F2840F3F482A0F17F03A8
:103BF00081FB0321DA17C2EB610000EB4000A3EB6D
:103C000080007330DFF8D8B098F80010C0B204F02C
:103C10008DFDBBF80030022B7FF67AAE3968BAF81A
:103C200000302C4ACB1A82FB030ED817C0EB6E0073
:103C300000EB4000A3EB800303EB430304EB83039F
:103C4000586808447F2840F3EA847F3882FB0032BA
:103C5000C317C3EB620303EB4303A0EB8300733092
:103C6000C0B298F8001004F061FDBBF80030032BDF
:103C70007FF64EAE3868BAF80030164AC31A82FB97
:103C8000031ED917C1EB6E0101EB4101A3EB8103C8
:103C900003EB430304EB8304A36818447F287FF7F6
:103CA00071AE7F3882FB0032C317C3EB620303EBB4
:103CB0004303A0EB8300733025E601283EF44DABAF
:103CC0000123FFF7B7BB99F8000004F057FDFFF799
:103CD000A6B800BFABAAAA2A2C140100549DFF1F4E
:103CE000889BFF1FE69BFF1FDFF8E8A299F8000002
:103CF000BAF80030B54AB64CC31A82FB031ED91776
:103D0000C1EB6E0101EB4101A3EB810303EB430324
:103D100054F8233018447F2840F3DD817F3882FB3C
:103D20000032C317C3EB620202EB4202A0EB820037
:103D30007330DFF8A4B2C0B204F020FDBBF800304D
:103D4000022B7EF6FBAE99F80000BAF800309F4ACD
:103D5000C31A82FB0321DA17C2EB610202EB4202B3
:103D6000A3EB820303EB430304EB83035B68184478
:103D70007F2840F327847F380C2290FBF2F302FB6C
:103D800013007330C0B204F0F9FCBBF80030032B11
:103D90007EF6D4AE99F80000BAF800308B4AC31A08
:103DA00082FB0321DA17C2EB610202EB4202A3EBB2
:103DB000820303EB430304EB8304A36818447F28C6
:103DC0007FF7DDAD7F380C2290FBF2F302FB13008E
:103DD000733015E5DFF8FCA13868BAF800307B4A8B
:103DE0007B4CC31A82FB031ED917C1EB6E0101EB9A
:103DF0004101A3EB810303EB430354F82330184440
:103E00007F2840F365817F3882FB0032C317C3EB04
:103E1000620202EB4202A0EB82007330DFF8BC8149
:103E2000DFF8B4B198F80010C0B204F07FFCBBF822
:103E30000030022B7EF6E3AF3868BAF80030634AF0
:103E4000C31A82FB0321DA17C2EB610202EB4202C2
:103E5000A3EB820303EB430304EB83035B68184487
:103E60007F2840F3A0837F380C2290FBF2F302FB03
:103E700013007330C0B298F8001004F057FCBBF880
:103E80000030032B7EF6BBAF3868BAF800304F4ADB
:103E9000C31A82FB0321DA17C2EB610202EB420272
:103EA000A3EB820303EB430304EB8304A3681844EE
:103EB0007F287FF781AD7F380C2290FBF2F302FB65
:103EC0001300733018E4DFF80CA14049BAF8002061
:103ED0003F4C9A1A81FB020ED017C0EB6E0000EB2C
:103EE0004000A2EB800202EB420254F82200184488
:103EF0007F2840F3F380A0F17F0381FB0321DA17D1
:103F0000C2EB610101EB4101A3EB81007330DFF8EB
:103F1000C8B098F80010C0B204F008FCBBF800303C
:103F2000022B7FF6F5AC3868BAF80030274AC31A7E
:103F300082FB0321DA17C2EB610202EB4202A3EB20
:103F4000820303EB430304EB83035B6818447F287D
:103F500040F345837F380C2290FBF2F302FB130001
:103F60007330C0B298F8001004F0E0FBBBF80030EA
:103F7000032B7FF6CDAC3868BAF80030134AC31A69
:103F800082FB0321DA17C2EB610202EB4202A3EBD0
:103F9000820303EB430304EB8304A36818447F28E4
:103FA0007FF7F0AC7F380C2290FBF2F302FB13009A
:103FB0007330A8E4FCF750FBFFF7CABBFCF74CFBDF
:103FC000FFF73EBBFCF748FB46E400BFABAAAA2ABA
:103FD000BC140100549DFF1F889BFF1FE69BFF1F21
:103FE000DFF83CA399F80000BAF80030C44AC54C89
:103FF000C31A82FB0317D917C1EB670101EB41011B
:10400000A3EB810303EB430354F8233018447F28C8
:104010006ADD7F3882FB0032C317C3EB620202EB1A
:104020004202A0EB82007330DFF8F8B2C0B204F0B5
:10403000A5FBBBF80030022B7FF6B5A999F800006C
:10404000BAF80030AE4AC31A82FB0321DA17C2EB7A
:10405000610202EB4202A3EB820303EB430304EB96
:1040600083035B6818447F2840F3B6827F380C22B4
:1040700090FBF2F302FB13007330C0B204F07EFB3E
:10408000BBF80030032B7FF68EA999F80000BAF830
:1040900000309B4AC31A82FB0321DA17C2EB61028C
:1040A00002EB4202A3EB820303EB430304EB830422
:1040B000A36818447F2814DD7F380C2290FBF2F3AC
:1040C00002FB13007330C0B204F058FBFFF76BB96A
:1040D000FCF7C2FAA2E6FCF7BFFA2AE6FCF7BCFA44
:1040E00015E7FCF7B9FAEEE7FCF7B6FA9CE7DFF85C
:1040F00030A299F80000BAF80030814A824CC31A05
:1041000082FB031ED917C1EB6E0101EB4101A3EB4A
:10411000810303EB430354F8233018447F28DADD8E
:104120007F3882FB0032C317C3EB620303EB430308
:10413000A0EB83007330FCE5DFF8E4A13868BAF83F
:1041400000306F4A704CC31A82FB031ED917C1EBB3
:104150006E0101EB4101A3EB810303EB430354F830
:10416000233018447F28B3DD7F3882FB0032C31729
:10417000C3EB620303EB4303A0EB830073304DE614
:10418000FCF76AFA40E4DFF898A15D49BAF800202C
:104190005D4C9A1A81FB020ED017C0EB6E0000EB4B
:1041A0004000A2EB800202EB420254F822001844C5
:1041B0007F2893DDA0F17F0381FB0321DA17C2EB97
:1041C000610000EB4000A3EB800073309FE6FCF73A
:1041D00043FA96E4FCF740FA14E5DFF844A199F8B5
:1041E0000000BAF80030464A484CC31A82FB031755
:1041F000D917C1EB670101EB4101A3EB810303EB8D
:10420000430354F8233018447F287FF76DAF7F387D
:1042100082FB0032C317C3EB620303EB4303A0EB43
:104220008300733000E73A4800903A483A490390D7
:10423000FEF712B9DFF8E8A03868BAF80030304A63
:10424000364CC31A82FB0321DA17C2EB610202EB80
:104250004202A3EB820303EB430354F823301844D8
:104260007F2840F3B6817F380C2290FBF2F302FBEB
:1042700013007330DFF8B080DFF8A8B098F80010B2
:10428000C0B204F053FABBF80030022B1AD93868D8
:10429000BAF800300C22C11A91FBF2F302FB13139F
:1042A00002FB03435B6818447F2840F367847F3830
:1042B00090FBF2F302FB13007330C0B298F80010C9
:1042C00004F034FABBF80030032B7EF698ADBAF850
:1042D000003038680C22C11A91FBF2F302FB131371
:1042E00002FB0344A36818447F287FF765AB7F383F
:1042F00090FBF2F302FB13007330FFF7FDB900BF30
:10430000ABAAAA2A301301009C1601002C1401004C
:10431000A49DFF1F559BFF1F589DFF1FF417010011
:10432000549DFF1F889BFF1FE69BFF1FDFF894A390
:1043300099F80000BAF80030D84AD94CC31A82FB69
:104340000321DA17C2EB610202EB4202A3EB820304
:1043500003EB430354F8233018447F2840F32081B3
:104360007F380C2290FBF2F302FB13007330DFF86E
:1043700058B3C0B204F002FABBF80030022B19D9CE
:1043800099F80000BAF800300C22C11A91FBF2F340
:1043900002FB131302FB03435B6818447F2840F3BE
:1043A00022847F3890FBF2F302FB13007330C0B21B
:1043B00004F0E4F9BBF80030032B7EF6BFABBAF88B
:1043C000003099F800000C22C11A91FBF2F302FBB5
:1043D000131302FB0344A36818447F287FF7CFAA76
:1043E0007F3890FBF2F302FB13007330FFF708BA3B
:1043F000012B3DF4DAAF0124FFF7A8BADFF8C4A21D
:10440000A649BAF80020A64C9A1A81FB0210D117CF
:10441000C1EB600101EB4101A2EB810202EB420220
:1044200054F8220018447F2840F3D080A0F17F0385
:104430000C2093FBF0F200FB12307330DFF888B2EF
:1044400098F80010C0B204F071F9BBF80030022BEC
:104450001AD93868BAF800300C22C11A91FBF2F36D
:1044600002FB131302FB03435B6818447F2840F3ED
:1044700082837F3890FBF2F302FB13007330C0B2EB
:1044800098F8001004F052F9BBF80030032B7FF6C7
:104490003FAABAF8003038680C22C11A91FBF2F337
:1044A00002FB131302FB0344A36818447F287FF721
:1044B00069AA7F3890FBF2F302FB13007330FFF719
:1044C00022BAFCF7C9F8FFF770B9FCF7C5F8FFF797
:1044D000E7B8DFF8F0A199F80000BAF800306F4AA9
:1044E000704CC31A82FB0321DA17C2EB610202EBA4
:1044F0004202A3EB820303EB430354F82330184436
:104500007F2846DD7F380C2290FBF2F302FB13007C
:104510007330DFF8B4B1C0B204F030F9BBF800304A
:10452000022B19D999F80000BAF800300C22C11AF0
:1045300091FBF2F302FB131302FB03435B68184485
:104540007F2840F3A7807F3890FBF2F302FB130033
:104550007330C0B204F012F9BBF80030032B7EF6C2
:1045600022AFBAF8003099F800000C22C11A91FB72
:10457000F2F302FB131302FB0344A36818447F28E1
:104580007FF7AFAD7F3890FBF2F302FB130073307F
:1045900099E5FCF761F8BCE7FCF75EF8FFF789B92D
:1045A000FCF75AF8E3E6FCF757F863E401339BB2F3
:1045B0002380D9B205203C4C04F090F83B7823705E
:1045C000FDF7DEBDFCF748F8FFF7DCBBFCF744F86D
:1045D00034E7FCF741F84DE6FCF73EF84DE5FCF713
:1045E0003BF8BEE4DFF8DCA099F80000BAF8003030
:1045F0002A4A2E4CA2E6013B9BB2D9B205202A4C96
:10460000138004F06BF83B782370FDF7B9BDDFF839
:10461000B4A03868BAF80030204A244C11E6FCF700
:104620001BF8FFF71DBBDFF89CA01C49BAF800205F
:104630001E4CE9E6FCF710F8FFF793BADFF884A008
:1046400099F80000BAF80030144A194C49E7FCF711
:1046500003F8FFF706BA029B1B78002B7EF44EAAE4
:10466000FEF771BA134B1B78002B00F0DE82124B61
:104670001B78002B7DF499AE104B1B78002B3DF47A
:1046800094AEB8F800300E490A33A8F800300A702A
:10469000FDF78BBEFBF7E0FF5BE700BFABAAAA2AE2
:1046A000F4170100BC140100729BFF1F0C160100DF
:1046B0009C160100DF9DFF1FE09DFF1FE19DFF1F76
:1046C000769BFF1F549DFF1F889BFF1FA14C2388D3
:1046D000002B40F05483DFF890B29F499F4A09882D
:1046E00099F80000B2F800E0DFF87882C1EB000C26
:1046F0000C229CFBF2F102FB11C14FF0900C0CFB61
:104700000EFE02FB01E16FF00B0E58F80110084499
:104710000EFB03007F2840F3EC84A0F17F0393FBA2
:10472000F2F002FB10307330C0B204F027F8BBF88F
:10473000002023881344022B22DD874A874B1188EF
:1047400099F80000B3F800C0DFF818E2411A0C2213
:1047500091FBF2F302FB1311902303FB0CF302FB1A
:10476000013373445B6818447F2840F350857F38D9
:1047700090FBF2F302FB13007330C0B203F0FEFFB4
:10478000BBF8002023881344032B22DD724A734BAD
:10479000118899F80000B3F800C0DFF8C8E1411AA9
:1047A0000C2291FBF2F302FB1311902303FB0CF399
:1047B00002FB013373449B6818447F2840F338851B
:1047C0007F3890FBF2F302FB13007330C0B203F0AA
:1047D000D5FFBBF8002023881344042B7EF7AEA935
:1047E0005F4B1B88012B7EF4A9A999F80020A2F148
:1047F0000C007F287FF7C3A88B3A0C2092FBF0F3C4
:1048000000FB13207330FEF7FBBF524C2288002AB6
:1048100000F018835249DFF850B10988BBF8000056
:104820000331884227DD4C484C490088B1F800E04C
:10483000DFF830C1181A0C2190FBF1F901FB1900C7
:104840004FF0900909FB0EFE01FB00E06FF00B0E2C
:104850005CF8000003440EFB02307F2840F3118413
:104860007F3890FBF1F301FB13007330C0B298F86E
:10487000001003F05BFFBBF8002023881344022BD9
:1048800023DD354B354A38681B88B2F800C0DFF8A5
:10489000D4E0C31A0C2193FBF1F201FB12329023F6
:1048A00003FB0CF301FB023373445B6818447F285D
:1048B00040F3A5847F3890FBF1F301FB13007330C4
:1048C000C0B298F8001003F031FFBBF80020238835
:1048D0001344032B23DD204B204A38681B88B2F891
:1048E00000C0DFF880E0C31A0C2193FBF1F201FB5A
:1048F0001232902303FB0CF301FB023373449B68D9
:1049000018447F2840F37F847F3890FBF1F301FB4C
:1049100013007330C0B298F8001003F007FFBBF823
:10492000002023881344042B7EF7F2AF0C4B1B8826
:10493000012B7EF4EDAF3A68A2F10C007F287FF7DF
:1049400021A88B3A0C2092FBF0F300FB132073306C
:10495000FEF7D9BFE89BFF1F549DFF1F029DFF1F5D
:10496000C29BFF1FA00F0100889BFF1FB84C23882C
:10497000002B40F06A82DFF810B3B649B64A0988C6
:10498000D7F80080B2F800E0B448C1EB080C0C2264
:104990009CFBF2F102FB11C14FF0900C0CFB0EFEE0
:1049A00002FB01E16FF00B0E405880440EFB0380C8
:1049B0007F2840F36A83A0F17F0393FBF2F002FBB0
:1049C00010307330A64BC0B2197803F0AFFEBBF8BD
:1049D000002023881344022B23DD9E4A9E4B11881E
:1049E0003868B3F800C0DFF874E2411A0C2291FB7A
:1049F000F2F302FB1311902303FB0CF302FB0133D0
:104A000073445B6818447F2840F30B847F3890FB25
:104A1000F2F302FB13007330914BC0B2197803F02C
:104A200085FEBBF8002023881344032B23DD894A2D
:104A3000894B11883868B3F800C0DFF820E2411ACA
:104A40000C2291FBF2F302FB1311902303FB0CF3F6
:104A500002FB013373449B6818447F2840F3DE83D4
:104A60007F3890FBF2F302FB130073307C4BC0B233
:104A7000197803F05BFEBBF8002023881344042B55
:104A80007EF7BDA9774B1B88012B7EF4B8A93A6845
:104A9000A2F10C007F2840F3B2808B3A0C2092FBED
:104AA000F0F300FB132073306D4BC0B2197803F0A4
:104AB0003DFEFEF7A4B9DFF89CA199F80000BAF812
:104AC0000030694CC11A0C2291FBF2F302FB131364
:104AD00002FB03F3E35818447F287FF75AAD7F3871
:104AE00090FBF2F302FB1300733012E55F4B1A8860
:104AF000182A13D03B681344A3F118007F2840F311
:104B00007B830C20973B93FBF0F200FB123303F105
:104B10007300534BC0B2197803F008FE544B55494B
:104B20001A78022A94BF013200221A701A7831F8DA
:104B30001200182810D10424022A02F10100C2B286
:104B400088BF002231F81200182804D1013CF3D1AB
:104B50001A70FEF754B91A703B680344A3F11800A9
:104B60007F284CDD0C20973B93FBF0F200FB1233C7
:104B700003F1730098E7FBF76FFD80E4FBF76CFD32
:104B8000FFF79BBB394B1B88182B12D099F80020DC
:104B90001344A3F118007F2840F33D830C20973B7A
:104BA00093FBF0F200FB123303F17300C0B203F089
:104BB000E5FD2F4A2F4B127833F81230182B3DF4B5
:104BC000BDAF99F800201344A3F118007F287EF7A9
:104BD000D6AE0C20973B93FBF0F200FB123303F1AF
:104BE0007300FEF70DBEFBF737FDFFF7E0BBDFF804
:104BF00064A099F80000BAF800301F4C62E7FBF798
:104C00002BFD51E71D4B1B78002B7DF4CEAB1C4BCD
:104C10001B78002B3DF4C9ABB8F800301949013BB3
:104C2000A8F800300A70FDF7C0BB144B1B78002BAE
:104C30007EF402A8124B1B78002B3DF4B6ABB8F8FB
:104C4000003010490133A8F800300A70FDF7ADBB01
:104C5000E89BFF1F549DFF1F029DFF1FA00F010037
:104C6000E69BFF1FC29BFF1FF4170100929BFF1FD3
:104C7000E79BFF1F689DFF1F0C160100E09DFF1FB3
:104C8000E19DFF1F769BFF1F889BFF1F944A1288A0
:104C9000182A12D01344A3F118007F2840F3CC82C5
:104CA0000C20973B93FBF0F200FB123303F17300EF
:104CB000C0B298F8001003F039FD8A4B8A491A787F
:104CC000022A94BF013200221A701A7831F81200B9
:104CD000182811D10424022A02F10100C2B288BFAF
:104CE000002231F81200182805D1013CF3D11A70C6
:104CF0003B68FEF77AB91A703B680344A3F11800C9
:104D00007F287EF73FAE0C20973B93FBF0F200FB31
:104D1000123303F17300FEF7F6BD744A1288182AA5
:104D200012D01344A3F118007F2840F37E820C2098
:104D3000973B93FBF0F200FB123303F17300C0B218
:104D400098F8001003F0F2FC664B69491A78022AC1
:104D500094BF013200221A701A7831F81200182814
:104D6000CAD10424022A02F1010294BFD2B2002265
:104D700031F812001828BED1013CF3D1B7E75D4AE3
:104D8000DFF884B11288BBF80010033291427FF73C
:104D9000CEACA2E4554B1B88182B12D099F80020FA
:104DA0001344A3F118007F2840F323820C20973B83
:104DB00093FBF0F200FB123303F17300C0B203F077
:104DC000DDFC484A4A4B127833F81230182B7FF436
:104DD000F8AEFDF7B3BE454B1A88182A13D03B68CE
:104DE0001344A3F118007F2840F3F2810C20973B75
:104DF00093FBF0F200FB123303F173003E4BC0B2A1
:104E0000197803F093FC374B39491A78022A94BF7A
:104E1000013200221A701A7831F8120018287FF433
:104E20009BAE0424022A02F1010294BFD2B20022F6
:104E300031F8120018287FF48EAE013CF2D11A70BE
:104E4000FDF7DDBFDFF8C0B0EDE42A4ADFF8B8B007
:104E50001288BBF80010033291427FF7B8AD8CE5A1
:104E6000264B01227F2107201A8003F037FC7F2187
:104E70000B2003F033FCFDF70ABF214B04227F21F6
:104E800007201A8003F02AFC00210B2003F026FCE7
:104E9000FDF7F6BE1A4B02227F2107201A8003F08D
:104EA0001DFC7F210B2003F019FCFDF7E4BE144B21
:104EB000002107201C8003F011FC7F210B2003F050
:104EC0000DFCFDF7D3BE0F4B00227F2107201A8077
:104ED00003F004FC7F210B2003F000FCFDF7DFBE94
:104EE000929BFF1FE79BFF1F689DFF1F9A9BFF1F61
:104EF000E89CFF1FC29BFF1FE69BFF1FF69BFF1F47
:104F00004A9DFF1F749BFF1F889BFF1FCC4C23886B
:104F1000002B40F06381DFF854B3CA4999F80000D0
:104F2000C94A09881788DFF824E3411A0C2291FB4B
:104F3000F2FC02FB1C114FF0900C0CFB07F702FB7C
:104F400001716FF00B075EF80110014407FB0310BD
:104F50007F2840F340817F3890FBF2F302FB13007F
:104F60007330C0B203F00AFCBBF80020238813445E
:104F7000022B21DDB34BB44A99F800001B88B2F82C
:104F800000E0B24FC31A0C2193FBF1F201FB123285
:104F9000902303FB0EF301FB02333B445B68184490
:104FA0007F2840F3B1817F3890FBF1F301FB1300C0
:104FB0007330C0B203F0E2FBBBF800202388134437
:104FC000032B21DD9F4BA04A99F800001B88B2F803
:104FD00000E09E4FC31A0C2193FBF1F201FB123249
:104FE000902303FB0EF301FB02333B449B68184400
:104FF0007F2840F386817F3890FBF1F301FB13009B
:105000007330C0B203F0BAFBBBF80020238813440E
:10501000042B7EF7C8A98E4B1B88012B7EF4C3A9F5
:1050200099F80020A2F10C007F287FF75AA88B3A4C
:105030000C2092FBF0F300FB13207330FFF743B812
:10504000844B1B88182B12D099F800201344A3F12D
:1050500018007F2840F35B810C20973B93FBF0F214
:1050600000FB123303F17300C0B203F087FB7A4AEE
:105070007A4B127833F81230182B7FF4A2ADFDF77B
:105080005DBDFBF7E9FAFFF7F1BBFBF7E5FA99E441
:10509000734B1B88182B12D099F800201344A3F1EE
:1050A00018007F2840F339810C20973B93FBF0F2E6
:1050B00000FB123303F17300C0B203F05FFB664ADA
:1050C000684B127833F81230182B3EF46CA999F81B
:1050D00000201344A3F118007F287FF702A80C20BA
:1050E000973B93FBF0F200FB123303F17300FEF7E2
:1050F000EABFFBF7B1FAFFF717BB564A1288182A26
:1051000012D01344A3F118007F2840F303810C2030
:10511000973B93FBF0F200FB123303F17300C0B234
:1051200098F8001003F002FB4B4B4C491A78022A06
:1051300094BF013200221A701A7831F81200182830
:105140007FF4DAAD0424022A02F1010294BFD2B244
:10515000002231F8120018287FF4CDAD013CF2D1C5
:10516000C5E53C4B1A88182A13D03B681344A3F1B9
:1051700018007F2840F3C2800C20973B93FBF0F28D
:1051800000FB123303F17300374BC0B2197803F000
:10519000CDFA314B31491A78022A94BF01320022EC
:1051A0001A701A7831F8120018287FF4D5AC04244C
:1051B000022A02F1010294BFD2B2002231F8120099
:1051C00018287FF4C8AC013CF2D11A70FDF717BE65
:1051D000FBF742FA12E6FBF73FFAC2E61C4ADFF899
:1051E0008CB01288BBF80010033291427FF7BCAE3E
:1051F00093E6FBF731FAE1E5FBF72EFA89E4FBF7DA
:105200002BFAFFF75DBBFBF727FAFFF783BBFBF732
:1052100023FAFFF7B2BAFBF71FFAC7E4FBF71CFA51
:1052200024E4FBF719FAFFF7F7BBFBF715FA86E55D
:10523000FBF712FAFFF7CABAFBF70EFA38E500BF20
:10524000E89BFF1F549DFF1F029DFF1FA00F010041
:10525000C29BFF1F9C9BFF1FE79BFF1FF09CFF1F34
:10526000929BFF1F689DFF1FE69BFF1F889BFF1FF0
:10527000304B1B88182B11D099F800201344A3F150
:1052800018007F2834DD0C20973B93FBF0F200FBE5
:10529000123303F17300C0B203F070FA264A274BB1
:1052A000127833F81230182B7FF411AFFEF77BB869
:1052B000234B1B88182B11D099F800201344A3F11D
:1052C00018007F2817DD0C20973B93FBF0F200FBC2
:1052D000123303F17300C0B203F050FA164A194BAF
:1052E000127833F81230182B7FF4F1AEFEF75BB86A
:1052F000FBF7B2F9CFE7FBF7AFF9ECE7FBF7ACF957
:1053000042E7FBF7A9F97CE6FBF7A6F951E6FBF7C4
:10531000A3F9A9E6FBF7A0F901E7FBF79DF9CBE6B6
:10532000094B0393094B0293FDF71EBF23601946F7
:10533000FDF758BC9C9BFF1FE79BFF1FF09CFF1FC6
:105340009A9BFF1FE89CFF1F559BFF1F029CFF1F9E
:1053500038B507F0EBF80B4805F022F800234FF0C2
:105360007E5201210848FBF781F8084B084A094999
:10537000802400251C7118461D60BDE838400AF0E5
:1053800099BD00BFF49BFF1F289DFF1FA89DFF1F15
:105390001C89FF1FFD05000043682A20198803F0BF
:1053A00021BB00BF10B5044622206368198803F0B2
:1053B00019FBE36824201988BDE8104003F012BBF4
:1053C00010B504460A206368198803F00BFBE368F4
:1053D0000C201988BDE8104003F004BB10B504464A
:1053E00006206368198803F0FDFAE368082019882D
:1053F000BDE8104003F0F6BA10B504460220636819
:10540000198803F0EFFAE36804201988BDE810401A
:1054100003F0E8BA70B50E4C84B0122504220123C3
:1054200006460390029320468DE8240014231021A1
:1054300006F0BAF906220923029303960195204645
:1054400000921423102106F0AFF904B070BD00BF24
:10545000109EFF1F2DE9F041224D82B0012602B2BD
:1054600084B20092284601967823192106F0E2F8CA
:1054700004F10C0212B28DE844002846A7197823E3
:10548000192104F1020806F0D5F83FB20FFA88F8A6
:1054900019233A46284619460196CDF8008006F0B1
:1054A000C9F878233A4628461946CDF80080019677
:1054B00004F10A070B3406F0BDF83FB224B278239A
:1054C0003A46284619468DE8500006F0B3F81923ED
:1054D00000943A4601962846194606F0ABF802B009
:1054E000BDE8F081109EFF1F2DE9F0411E4682B0FD
:1054F0001446002A6AD0099B4D4A00EBC305012CD3
:105500006F8929896868A7EB010382FB03E21A44CB
:105510004FEAE373C3EBA21302887BD0042C38D18B
:1055200012FA83F3994203DC9F423946A8BF194619
:10553000089A0180B6F90030BDF920803D48971DDA
:105540004FF0000E3FB2194642460097CDF804E0F6
:1055500006F070F829896A896B68521A1B885C2AE0
:10556000A3EB010359DD03EB43030132C3EB431308
:1055700093FBF2F303F11B0213B2012032801946B0
:105580004246019000972B4806F054F82A4B00221F
:105590001A702A4B022CB3F9001045D0082C31D1D7
:1055A00000221A8091422DD0089AB6F90030214885
:1055B0000632012412B2009219460194BDF920204E
:1055C00006F038F8204602B0BDE8F0811C4D1D4AB7
:1055D0002B681268CB1A93420F4617D9164A3388A4
:1055E00011781448012918BF01241470089A063252
:1055F0001BB212B28DE814001946BDF9202006F046
:1056000019F82F60012002B0BDE8F081204602B0F9
:10561000BDE8F0819BB2D31A84E75C2101FB03F360
:1056200093FBF2F21B32A7E74A1C12B21A80B9E7C9
:10563000C94216B2109EFF1F899EFF1FF09DFF1FDB
:10564000749EFF1F8027010030B583B000230C46F5
:1056500005B2009326225B231C210C4805F03AFD7D
:10566000294601232622094805F044F8002C24B2DB
:1056700005DB214601232622044805F03BF8044AB5
:10568000044B15801C8003B030BD00BF109EFF1F6F
:10569000AC89FF1FAE89FF1F70B5944C237882B090
:1056A0001BB1934B4FF6FF721A80924BB3F9003047
:1056B000C3B9914A8E4B1068B3F9002080F30C00F7
:1056C0005B2303FB00F000131C3082425AD04FF0E2
:1056D000FF31FFF7B9FF894805F060FD0023237013
:1056E00002B070BD012B32D0022B6AD0032B4FD0F9
:1056F000042BF3D1272200258DE8240076231C21DA
:105700007E487F4E05F096FF17E0B0F5AF7FA8BF4B
:105710004FF4AF70323803FB00F386FB0321DB1735
:10572000C3EB61111C3109B201231D4427227348C8
:1057300004F0E0FF0C2D00F08180E9B2714804F024
:1057400097FE31284FF05B03DFDC1C21ECE76E4B4A
:105750001A68B2F52F7F32DB41F25C239342A8BF77
:105760001346A3F52F735B22684802FB03F380FB0B
:105770000320DB17C3EBA0201C305D4BB3F90030D6
:105780008342A4D1624BB3F9003001339FD1A5E726
:10579000604B1B68B3F5FA7F11DBB3F57A6FA8BFD6
:1057A0004FF47A63A3F5FA725B485B2303FB02F3C1
:1057B00080FB0320DB17C3EB20201C30DDE71C201F
:1057C000DBE7564B1B68B3F5FA7F33DBB3F57A6F33
:1057D000A8BF4FF47A63A3F5FA724F485B2303FB2B
:1057E00002F380FB0320DB17C3EB20201C304C4B63
:1057F0001B68B3F5FA7F1FDBB3F57A6FA8BF4FF4D0
:105800007A63A3F5FA7244495B2303FB02F381FB3D
:105810000321DB17C3EB21211C31354BB3F90030D9
:1058200083427FF456AF3A4BB3F900308B427FF49A
:1058300050AF53E71C20DAE71C21EEE7012007F008
:105840001DFD6FF495733238364A03FB00F082FB7E
:105850000023C017C0EB632303F5AF73312B3ADD90
:10586000B3F5AF7FA8BF4FF4AF735B22323B244D3B
:1058700002FB03F385FB0325DB17C3EB65151C3522
:10588000002007F0FBFC6FF495733238254A03FBC8
:1058900000F082FB0023C017C0EB632303F5AF7356
:1058A000312B1ADDB3F5AF7FA8BF4FF4AF735B2286
:1058B000323B134902FB03F381FB0321DB17C3EBEC
:1058C00061111C310A4BB3F90030AB4207D02846B6
:1058D000FFF7BAFEFFE61C25D2E71C21F2E70C4BCE
:1058E000B3F900308B42F2D1F5E600BFE69DFF1F11
:1058F000AC89FF1FEC9DFF1F5C9DFF1F109EFF1FCB
:105900004B48371BF49BFF1F649BFF1FD30585414A
:10591000AE89FF1FA49BFF1F011FB812AC9BFF1F86
:10592000D49DFF1F67BBCF462DE9F04FDFF8EC8217
:10593000B74CB8F900604D7854F8264087B08246DD
:10594000039305B10D78DFF8FCB2002A34D19BF83F
:1059500000308BBBAF4EB6F90000002800F0CE80BF
:10596000012800F02481012032232A46019000936F
:105970005146A94B2046FFF7B7FD00250746B6F96B
:105980000030022B40F3F48000233380B8F900305C
:10599000A24A002BC0F2F880042BC4BF002313805E
:1059A000039B002B40F0F680002D0CBF38464FF0D3
:1059B000FF3007B0BDE8F08F964EE3682268984844
:1059C00004930027059237808BF8007005F0DAFA0F
:1059D0001120FFF73FFD4FF0010919232821CDF8D1
:1059E00004900091242219468D4805F023FE782367
:1059F00028212422CDF8049000918948194605F009
:105A000019FE4946864806F0ABF90222192184485E
:105A100006F0A2F9DDF8149048460BF011F849465B
:105A200002467F4806F032FB7D4806F045FB3946CA
:105A300014227B4806F090F903227A49784806F050
:105A400025FB774806F038FB39462322744806F0D8
:105A500083F903227449724806F018FB704806F077
:105A60002BFB049B002B72D10123704A1846137044
:105A7000FFF7D0FC208963896768191A5C293A8886
:105A80005BDC131A5C2202FB03F292FBF1F31B3383
:105A9000674A6348138001271BB21A2219468DE812
:105AA0008400142205F0C6FD049BDBB1218A638AC1
:105AB000E768581A5C283A886FDD521A02EB4202F6
:105AC000C2EB4212431C92FBF3F31B33524A54487D
:105AD0001380012738221BB28DE884001946322238
:105AE00005F0A8FD534A544BB6F90000012111708E
:105AF0004FF6FF721A8000287FF432AFDFF848912A
:105B00004E4AD9F800301268C3EB0A0393424CD9CD
:105B1000464B1A78012A18BF012018700127FFF799
:105B200079FCC9F800A0012D4ED0042D59D0022DCA
:105B300060D0082D64D0002521E7121A02EB420242
:105B4000C2EB42124B1C92FBF3F31B33A0E72F2056
:105B5000FFF780FC39463222314806F0FDF8032277
:105B600037492F4806F092FA2D4806F0A5FA7BE750
:105B70007FF40CAFE368002B3FF406AFB8F90030B8
:105B8000264A002BBFF608AF04231380039B002B8B
:105B90003FF40AAFFFF780FD06E7511A5C2202FBD3
:105BA00001F292FBF0F31B3390E70746BBE70027B7
:105BB00014238DE888002A4651461D4B2046FFF7E6
:105BC00093FC3D460746DAE6B8F800308BF8005003
:105BD0000133A8F80030636983B100252046984757
:105BE000CDE6B8F800300122013BA8F800308BF870
:105BF0000020F0E7012333800025C7E61D46BEE6FE
:105C00006369002232804FF0FF35002BE6D1BDE6FC
:105C1000B089FF1FF09DFF1FEA9DFF1FEC9DFF1F36
:105C2000109EFF1FB4180100B8180100899EFF1FC5
:105C3000E89DFF1FE69DFF1FAC89FF1F8027010025
:105C4000BC180100EE9DFF1F749EFF1F01210D2057
:105C500007F0E6B800210D2007F0E2B801460D205C
:105C600007F0DEB808B50D2007F0E0F8B0FA80F1D3
:105C700049090D20BDE8084007F0D2B810B5002151
:105C800044080D2007F0CCF8204607F005F90D2058
:105C9000012107F0C5F82046BDE8104007F0FCB828
:105CA000214A224B10881B68984210B535DA204AE9
:105CB0001288141A9A42A8BF1A46B4F5157F22DA40
:105CC000121A40F2532303FB02F393FBF4F1053164
:105CD0000A2006F015FF174B197801B3164B174928
:105CE0001B6840F2271283F3070302FB03F381FBD7
:105CF00003211944DB17C3EBA11105310920BDE8CD
:105D0000104006F0FDBE131A4FF41572611C02FB21
:105D100003F393FBF1F10531DAE70021D8E709201D
:105D2000BDE8104006F0ECBE009CFF1F589BFF1F13
:105D3000B89DFF1FC49BFF1F5C9BFF1F09040281CE
:105D40007F2838B5A8BF7F200F4C4FF4167202FB96
:105D500000F284FB02311144D2170546C2EBA111B7
:105D60000A2006F0CDFE7F3D4FF4967303FB05F34A
:105D700084FB03211944DB17A3EBA1110920BDE823
:105D8000384006F0BDBE00BF09040281C368B3F904
:105D9000003030B583EAE374A4EBE374002BA0B2C7
:105DA00018DB012300E0134603EB83025200944208
:105DB000F9DA0A4D90FBF3F285FB03E403FB1200D2
:105DC000DB173032D3EBA40380B201F8012BF1D101
:105DD0000B7030BD2D230B700131E2E767666666FC
:105DE00038B5094D8224204602F016FE35F8021B14
:105DF00000B28842204601D002F0F4FD0234A4B281
:105E00008A2CF0D138BD00BFF09CFF1F024B8020D0
:105E1000198802F0E7BD00BF9C9BFF1F38B5094DF4
:105E20007824204602F0F8FD35F8021B00B28842C3
:105E3000204601D002F0D6FD0234A4B2802CF0D16D
:105E400038BD00BFE89CFF1F024B7620198802F086
:105E5000C9BD00BF9A9BFF1F38B5094D4624204697
:105E600002F0DAFD35F8021B00B28842204601D06C
:105E700002F0B8FD0234A4B24E2CF0D138BD00BF00
:105E8000689DFF1F024B4420198802F0ABBD00BF84
:105E9000929BFF1F024B4E20198802F0A3BD00BF4A
:105EA000A89BFF1F024B9A20198802F09BBD00BFE0
:105EB000E89BFF1F024B9820198802F093BD00BF9A
:105EC000C29BFF1F024B8C20198802F08BBD00BFC4
:105ED000029DFF1F024B9C20198802F083BD00BF6A
:105EE000889BFF1F024BA020198802F07BBD00BFDA
:105EF000DC9DFF1F024B9620198802F073BD00BF86
:105F0000549DFF1F024B8A20198802F06BBD00BF11
:105F1000169DFF1F08B5034B1020198802F062FD83
:105F2000012008BD149DFF1F024B1020198802F0AC
:105F300059BD00BF149DFF1F024B2C20198802F091
:105F400051BD00BF869BFF1F024B1E20198802F027
:105F500049BD00BFA09BFF1FC3680E20198802F037
:105F600041BD00BF024B2820198802F03BBD00BF95
:105F7000649DFF1F024B6220198802F033BD00BFF1
:105F8000B29BFF1F024B6420198802F02BBD00BF9B
:105F9000609DFF1F024B5A20198802F023BD00BFED
:105FA0006C9BFF1F024B1620198802F01BBD00BF1F
:105FB000749BFF1F024B2E20198802F013BD00BFF7
:105FC000F09BFF1F024B3020198802F00BBD00BF71
:105FD000C49DFF1F024B9E20198802F003BD00BF25
:105FE0009089FF1F024B1820198802F0FBBC00BFEC
:105FF000049CFF1F024B1A20198802F0F3BC00BF5B
:10600000B09BFF1F024B1C20198802F0EBBC00BFA5
:10601000AA9BFF1F024B6620198802F0E3BC00BF59
:10602000A29DFF1F024B7220198802F0DBBC00BF4B
:10603000C09DFF1F024B2020198802F0D3BC00BF77
:10604000A09DFF1F024B3220198802F0CBBC00BF7D
:10605000929DFF1F024B6820198802F0C3BC00BF4D
:10606000DC9BFF1F024B6C20198802F0BBBC00BFF9
:10607000609BFF1F024B5220198802F0B3BC00BF87
:106080002E89FF1F024B5020198802F0ABBC00BFC5
:10609000A489FF1F024B5420198802F0A3BC00BF43
:1060A000A689FF1F024B5C20198802F09BBC00BF31
:1060B000AA89FF1F024B5E20198802F093BC00BF23
:1060C0002C89FF1F024B6020198802F08BBC00BF97
:1060D000049DFF1F024B5620198802F083BC00BFAD
:1060E000E49BFF1F244B1B880B2B43D8DFE803F0F6
:1060F0000B10151A1F24292E33383D06084604229A
:106100001E490AF05BBD084604221D490AF056BD2F
:10611000084604221B490AF051BD084604221A49C8
:106120000AF04CBD0846042218490AF047BD08464B
:10613000042217490AF042BD0846042215490AF014
:106140003DBD0846042214490AF038BD0846042221
:1061500012490AF033BD0846042211490AF02EBD47
:10616000084604220F490AF029BD084604220E49B8
:106170000AF024BD704700BF549DFF1F1C2401007E
:1061800000220100B4200100D0240100B820010049
:10619000B8240100BC200100C0200100242301001C
:1061A000C420010028240100C8200100064B074A32
:1061B00010B41C88064B0846002C14BF1146194623
:1061C000042210BC0AF0FABCC09BFF1FCC200100C7
:1061D000D0200100064B074A10B41C88064B084625
:1061E000002C14BF11461946042210BC0AF0E6BC6C
:1061F000F29BFF1FCC200100D0200100064B074A74
:1062000010B41C88064B0846002C14BF11461946D2
:10621000042210BC0AF0D2BC069DFF1FCC20010056
:10622000D0200100064B074A10B41C88064B0846D4
:10623000002C14BF11461946042210BC0AF0BEBC43
:106240001C9DFF1FCC200100D0200100064B074AF7
:1062500010B41C88064B0846002C14BF1146194682
:10626000042210BC0AF0AABC569DFF1FCC200100DE
:10627000D0200100064B074A10B41C88064B084684
:10628000002C14BF11461946042210BC0AF096BC1B
:10629000F69BFF1FCC200100D02001001B4B1B8868
:1062A0000A2B0AD8DFE803F00A0E12161A1E22265D
:1062B0002A2E0600164B186808607047154B1868A0
:1062C00008607047144B186808607047134B1868D3
:1062D00008607047124B186808607047114B1868C7
:1062E00008607047104B1868086070470F4B1868BB
:1062F000086070470E4B1868086070470D4B1868AF
:10630000086070470C4B186808607047169DFF1FA7
:10631000F8200100D0200100D4200100D820010085
:10632000DC200100E0200100E4200100E820010061
:10633000EC200100F0200100F4200100F0B52B4E0C
:106340002B4FDFF8C4E005460FCE87B06C460FC474
:1063500096E803003B68274A274F44F8040B40F6B1
:10636000CC308342C8BF3A46BEF800602180012E7F
:1063700011889278ADF80D108DF80F202AD032D305
:1063800040F6CA02022E18BF00229A4226DCA3F66B
:1063900098031A491A4AC3EB031381FB03011944FA
:1063A000DB17C3EB6123243382FB0321DA17C2EB33
:1063B000A10202EB8201A3EB4103303330328DF8AE
:1063C00013308DF811206946284616220AF0F6FB94
:1063D00007B0F0BD40F698029A42D8DD094B186824
:1063E000CDF81100EFE740F6FC02CEE70C210100EA
:1063F0007C9DFF1F00210100FC2001003B773B98A2
:106400006766666604210100F89CFF1FF8B5174C0B
:10641000174E2278174D33782F888E46003218BFDA
:10642000012201467046FFF77FFA0023984233703D
:10643000237015DB14BF012000202B889F420ED053
:1064400040F23A72A3F5AF730B490C4C02FB03F315
:1064500081FB0312DB17A3EB621332332360F8BD19
:106460000749012218460A702270E6E7788AFF1F62
:10647000019EFF1FB09DFF1FB5814E1B9489FF1F1A
:10648000889EFF1F014B187802F044BA709EFF1FD0
:10649000014B187802F058BA2090FF1F134BB3F944
:1064A000003030B583EAE374A4EBE374002BA0B2B0
:1064B00018DB012300E0134603EB830252009442F1
:1064C000F9DA0B4D90FBF3F285FB03E403FB1200BA
:1064D000DB173032D3EBA40380B201F8012BF1D1EA
:1064E0000B7030BD2D230B700131E2E72090FF1FB0
:1064F00067666666144BB3F9003070B583EAE375DE
:10650000A5EBE375002BACB21ADB012300E00346D8
:1065100003EB830040008542F9DA0C4E94FBF3F064
:1065200086FB03E503FB1044DB173030D3EBA503F8
:10653000A4B201F8010BF1D105480B70106070BDD9
:106540002D230B700131E0E76C9BFF1F67666666C9
:1065500024210100134BB3F9003030B583EAE37412
:10656000A4EBE374002BA0B218DB012300E0134678
:1065700003EB830252009442F9DA0B4D90FBF3F2E5
:1065800085FB03E403FB1200DB173032D3EBA403DB
:1065900080B201F8012BF1D10B7030BD2D230B70AF
:1065A0000131E2E79089FF1F67666666134BB3F916
:1065B000003030B583EAE374A4EBE374002BA0B29F
:1065C00018DB012300E0134603EB830252009442E0
:1065D000F9DA0B4D90FBF3F285FB03E403FB1200A9
:1065E000DB173032D3EBA40380B201F8012BF1D1D9
:1065F0000B7030BD2D230B700131E2E72E89FF1F98
:1066000067666666134BB3F9003030B583EAE3740E
:10661000A4EBE374002BA0B218DB012300E01346C7
:1066200003EB830252009442F9DA0B4D90FBF3F234
:1066300085FB03E403FB1200DB173032D3EBA4032A
:1066400080B201F8012BF1D10B7030BD2D230B70FE
:106650000131E2E7A489FF1F67666666134BB3F951
:10666000003030B583EAE374A4EBE374002BA0B2EE
:1066700018DB012300E0134603EB8302520094422F
:10668000F9DA0B4D90FBF3F285FB03E403FB1200F8
:10669000DB173032D3EBA40380B201F8012BF1D128
:1066A0000B7030BD2D230B700131E2E7A689FF1F6F
:1066B00067666666134BB3F9003030B583EAE3745E
:1066C000A4EBE374002BA0B218DB012300E0134617
:1066D00003EB830252009442F9DA0B4D90FBF3F284
:1066E00085FB03E403FB1200DB173032D3EBA4037A
:1066F00080B201F8012BF1D10B7030BD2D230B704E
:106700000131E2E7AA89FF1F67666666134BB3F99A
:10671000003030B583EAE374A4EBE374002BA0B23D
:1067200018DB012300E0134603EB8302520094427E
:10673000F9DA0B4D90FBF3F285FB03E403FB120047
:10674000DB173032D3EBA40380B201F8012BF1D177
:106750000B7030BD2D230B700131E2E72C89FF1F38
:106760006766666608B5702002F056F9044B198812
:10677000884204D07020BDE8084002F033B908BD5B
:10678000F89CFF1F08B5742002F046F9044B1988E5
:10679000884204D07420BDE8084002F023B908BD47
:1067A000889DFF1F054B1B880846042213B9044926
:1067B0000AF004BA03490AF001BA00BFA89BFF1F00
:1067C0002C210100282101000E4B1B88032B17D818
:1067D000DFE803F0110C0702084604220A490AF018
:1067E000EDB90846042209490AF0E8B9084604222E
:1067F00007490AF0E3B90846042206490AF0DEB95F
:10680000704700BF029DFF1F3C210100382101009D
:10681000342101003021010010B40A4B0A4C0A4611
:1068200093E8030083B0238802AC04E9030004EB7F
:106830008303104653F8081C052203B010BC0AF06D
:10684000BDB900BF44190100609DFF1F30B40A4B61
:106850000A4D0C4693E8070084B02B8804AD05E987
:10686000070005EB8303204653F80C1C042204B0F8
:1068700030BC0AF0A3B900BF4C190100F89CFF1FFF
:10688000F0B40C4D0C4F0E460FCD8CB001AC0FC4C4
:106890000FCD0FC495E807003B8884E807000CAAD9
:1068A00002EB8303304653F82C1C04220CB0F0BCDE
:1068B0000AF084B9581901004A9DFF1FF0B40A4D2F
:1068C0000A4F0E460FCD86B001AC0FC42A683B8834
:1068D000226006AA02EB8303304653F8141C0422FC
:1068E00006B0F0BC0AF06AB984190100049CFF1FCD
:1068F000F0B40A4D0A4F0E460FCD86B001AC0FC45E
:106900002A683B88226006AA02EB8303304653F8CC
:10691000141C0C2206B0F0BC0AF050B99819010002
:10692000AA9BFF1FF0B40A4D0A4F0E460FCD86B04A
:1069300001AC0FC42A683B88226006AA02EB8303DD
:10694000304653F8141C042206B0F0BC0AF036B9E5
:10695000AC190100889DFF1F164B1B880BB31BB29F
:1069600083EAE370A0EBE370002B30B584B21DDB4B
:10697000012300E0134603EB830252009042F9DA50
:106980000D4894FBF3F280FB03E503FB1244DB1795
:106990003032D3EBA503A4B201F8012BF1D10B7077
:1069A00030BD0846042205490AF008B92D230B70B2
:1069B0000131DDE7DC9BFF1F676666664021010051
:1069C00030B40A4B0A4D0C4693E8070084B02B887C
:1069D00004AD05E9070005EB8303204653F80C1CC2
:1069E000042204B030BC0AF0E9B800BFC0190100AD
:1069F000609BFF1F054B1B881BB9054B186808607F
:106A000070470846042203490AF0D8B8E89BFF1FE4
:106A1000D0200100CC200100164B1B880BB31BB209
:106A200030B583EAE374A4EBE374002BA0B21CDB63
:106A3000012300E0134603EB830252009442F9DA8B
:106A40000D4D90FBF3F285FB03E403FB1200DB1713
:106A50003032D3EBA40380B201F8012BF1D10B70DB
:106A600030BD064B1868086070472D230B7001314C
:106A7000DEE700BFA09BFF1F67666666D0200100AF
:106A8000164B1B880BB31BB230B583EAE374A4EB3F
:106A9000E374002BA0B21CDB012300E0134603EBE0
:106AA000830252009442F9DA0D4D90FBF3F285FB1C
:106AB00003E403FB1200DB173032D3EBA40380B2F4
:106AC00001F8012BF1D10B7030BD064B186808603E
:106AD00070472D230B700131DEE700BF969DFF1F2D
:106AE00067666666D0200100164B1B880BB31BB28D
:106AF00030B583EAE374A4EBE374002BA0B21CDB93
:106B0000012300E0134603EB830252009442F9DABA
:106B10000D4D90FBF3F285FB03E403FB1200DB1742
:106B20003032D3EBA40380B201F8012BF1D10B700A
:106B300030BD064B1868086070472D230B7001317B
:106B4000DEE700BF749BFF1F676666664421010095
:106B5000174B1B881BB31BB270B583EAE375A5EB1B
:106B6000E375002BACB21EDB012300E0034603EB10
:106B7000830040008542F9DA0E4E94FBF3F086FB69
:106B800003E503FB1044DB173030D3EBA503A4B2BD
:106B900001F8010BF1D108480B70106070BD074B74
:106BA0001868086070472D230B700131DCE700BFC7
:106BB000F09BFF1F6766666648210100D020010038
:106BC000164B1B880BB31BB230B583EAE374A4EBFE
:106BD000E374002BA0B21CDB012300E0134603EB9F
:106BE000830252009442F9DA0D4D90FBF3F285FBDB
:106BF00003E403FB1200DB173032D3EBA40380B2B3
:106C000001F8012BF1D10B7030BD064B18680860FC
:106C100070472D230B700131DEE700BFC49DFF1FBD
:106C200067666666D0200100164B1B880BB31BB24B
:106C300030B583EAE374A4EBE374002BA0B21CDB51
:106C4000012300E0134603EB830252009442F9DA79
:106C50000D4D90FBF3F285FB03E403FB1200DB1701
:106C60003032D3EBA40380B201F8012BF1D10B70C9
:106C700030BD064B1868086070472D230B7001313A
:106C8000DEE700BFA29DFF1F67666666D020010099
:106C9000164B1B880BB31BB230B583EAE374A4EB2D
:106CA000E374002BA0B21CDB012300E0134603EBCE
:106CB000830252009442F9DA0D4D90FBF3F285FB0A
:106CC00003E403FB1200DB173032D3EBA40380B2E2
:106CD00001F8012BF1D10B7030BD064B186808602C
:106CE00070472D230B700131DEE700BFC09DFF1FF1
:106CF00067666666D0200100174B1B881BB31BB26A
:106D000070B583EAE375A5EBE375002BACB21EDB2F
:106D1000012300E0034603EB830040008542F9DADB
:106D20000E4E94FBF3F086FB03E503FB1044DB17E8
:106D30003030D3EBA503A4B201F8010BF1D1084820
:106D40000B70106070BD074B1868086070472D23EA
:106D50000B700131DCE700BFA09DFF1F6766666610
:106D600048210100D0200100074B1B88022B06D0D0
:106D7000012B0CBF054B064B186808607047054B8C
:106D800018680860704700BF049DFF1F5021010074
:106D9000542101004C210100054B1B881BB1054B00
:106DA000186808607047044B18680860704700BF97
:106DB000E49BFF1F5C21010058210100184B1A8839
:106DC00052B3184A128830B50A80B3F90030002B4C
:106DD00083EAE374A4EBE374BCBF2D238B70A0B2F1
:106DE000ACBF02310331012300E0134603EB830201
:106DF00052009442F9DA0C4D90FBF3F285FB03E468
:106E000003FB1200DB173032D3EBA40380B201F88E
:106E1000012BF1D10B7030BD044B1868086070472E
:106E2000B09BFF1F6021010067666666D0200100ED
:106E300070B53C4D2B780646002B35D11C46737837
:106E40000BB9204670BDFAF735FF374A374B384843
:106E5000127831781B78007802EB43034A1E03EB6B
:106E600080030E2AEDD801A050F822F0D56E000064
:106E7000F76E0000436E0000D56E0000436E000008
:106E8000436E0000436E0000C36E0000436E0000BE
:106E9000436E0000436E0000436E0000436E00002E
:106EA000436E0000BF6E0000AE21224803F01AFEC0
:106EB000204804F067F800232B700124BFE706F098
:106EC000FDFAAF211B4803F00DFE1B4A012313708E
:106ED0002B70B6E783B91948038804294FF6FF7170
:106EE00003F1FF320CBF01230B46134403F07F0371
:106EF000013303800FE073B1013B114A32F81330C4
:106F00004BB10E4E0F481049104A33800123002622
:106F100006700B701370084A0221012311702B7048
:106F2000204670BD788AFF1FE29DFF1FE39DFF1F73
:106F3000989DFF1F109EFF1F889EFF1F949DFF1F9F
:106F4000D89CFF1FD49BFF1F769BFF1F8B9EFF1FAC
:106F500010B5064B064C1A882046012101F030FD81
:106F600021884220BDE8104001F03CBDC09BFF1FBE
:106F7000909BFF1F10B5064B064C1A882046022135
:106F800001F01EFD21884220BDE8104001F02ABD1D
:106F9000F29BFF1F909BFF1F10B5064B064C1A88F3
:106FA0002046042101F00CFD21884220BDE810405C
:106FB00001F018BD069DFF1F909BFF1F10B5064BEB
:106FC000064C1A882046062101F0FAFC218842204E
:106FD000BDE8104001F006BD1C9DFF1F909BFF1FE8
:106FE00010B5064B064C1A882046002101F0E8FC3B
:106FF00021884220BDE8104001F0F4BC569DFF1FDF
:10700000909BFF1F08B5122001F006FD054B198863
:10701000884206D0122001F0E5FCBDE8084001F0EE
:10702000F9BB08BD4A9DFF1F08B5582001F0F4FCCC
:10703000054B1988884206D0582001F0D3FCBDE8E2
:10704000084001F0E7BB08BD969DFF1F08B514205E
:1070500001F0E2FC054B1988884206D0142001F0AB
:10706000C1FCBDE8084001F0D5BB08BDF69BFF1F81
:10707000F0B480EAE075A5EBE0750028ACB21FDB48
:107080001DBF2B230B704E1C0E46012300E0134640
:1070900003EB830252009542F9DA0B4F94FBF3F2B3
:1070A00087FB030503FB1244DB173032D3EBA50348
:1070B000A4B206F8012BF1D133700846F0BC70473A
:1070C0002D230B704E1CE0E767666666174B188829
:1070D0000C2813D0192815D01A2817D01B2819D01E
:1070E0001C281BD01D281DD01E2803D00C3800B230
:1070F000FFF7BEBF0E4A1068086070470D4A10685F
:10710000086070470C4A1068086070470B4A1068A6
:10711000086070470A4A106808607047094A10689A
:1071200008607047084A106808607047929DFF1F0A
:1071300080210100682101006C2101007021010003
:1071400074210100782101007C210100034B188883
:10715000A0EB8000400000B2FFF78ABF709EFF1FC7
:10716000024BB3F90000FFF783BF00BFB29BFF1FC4
:10717000024B1888033800B2FFF77ABF649DFF1FE7
:10718000024B18880C3800B2FFF772BF709BFF1FCC
:10719000024B1888183800B2FFF76ABF9C9BFF1F8C
:1071A000024B1888183800B2FFF762BF9A9BFF1F86
:1071B000024B1888183800B2FFF75ABF929BFF1F86
:1071C000C3681888183800B2FFF752BF054B1B88F8
:1071D0001BB9054B1868086070470846042203492C
:1071E00009F0ECBCDC9DFF1FD0200100CC20010089
:1071F000054B1B881BB9054B18680860704708468B
:107200000422034909F0DABCC29BFF1FD020010011
:10721000CC20010030B5134C85B001252B463C2213
:1072200002212046009503F0D3FC204603F0AAFE7D
:1072300000224021802320460191009311460A4BF1
:10724000029504F04DFB204603F0A8FF07480849CB
:10725000084A0023036083800B608B801360938057
:1072600005B030BD109EFF1F0C1A0100F49DFF1FDA
:10727000089EFF1F789EFF1F10B500EBC00000F1B5
:107280000F02D2B293B284B09C1E981C3D2303918E
:107290008DE819003921024804F086FA04B010BDC7
:1072A000109EFF1F014B01221A707047019EFF1FA5
:1072B000F0B5694B694C6A4F6A4E6B4D85B004223C
:1072C0008DE80C0002932046684B4022802103F099
:1072D00087FA2046664A6749674C08F0EBFD674A23
:1072E000674B9761674FD761674F9F61674FDF615A
:1072F000674FB761674FF761674FAF61674FEF61E6
:10730000674FA7616748684FE761684F87616849C1
:10731000684FC761684F8F61684A694FCF61694F95
:107320009761694B694FD761694F9F61694E6A4F99
:10733000DF616A4F6A4DB7616A4FF7616A4F6B4C04
:10734000AF616B4FEF616B4F6B48A7616B4FE761AC
:107350006B4F6C4987616C4FC7616C4F6C4A8F6192
:107360006C4FCF616C4F6D4B97616D4FD7616D4F17
:107370006D4E9F616D4FDF616D4FB7616D4D6E4F0B
:10738000F7616E4FAF616E4C6E4FEF616E4FA7614C
:107390006E486F4FE7616F4F87616F496F4FC761ED
:1073A0006F4F8F616F4A704FCF61704F9761704B15
:1073B000704FD761704F9F61704E714FDF61714F99
:1073C000B761714D714FF761714FAF61714C724F81
:1073D000EF61724FA7617248724FE761724F734954
:1073E0008761734FC761734F734A8F61734FCF616A
:1073F000734F744B9761744FD761744F744E9F6194
:10740000744FDF61744F754DB761754FF761754FFC
:10741000754CAF61754F76487649EF61764F774D81
:10742000A761DFF808E2E561754F764D764C774A43
:10743000774B8761C5618C61764E774F774D784C7D
:10744000C1F81CE0774878499761D5619C61D861A3
:10745000B16005B0F0BD00BF40420F00109EFF1F9D
:1074600081710000F08DFF1FE08BFF1F3C90FF1F1C
:107470001C89FF1F39A80000A48EFF1FE889FF1F89
:10748000808EFF1F595F000071710000655F000072
:10749000AD610000516F0000D5610000756F000004
:1074A000FD6100000C8AFF1F996F000061710000F0
:1074B000708CFF1F755F000025620000008DFF1FAC
:1074C000BD6F0000196800004C8CFF1F855F000035
:1074D0004D620000DC8CFF1FE16F00004D71000069
:1074E000B88CFF1F856400009D6400005C8EFF1F48
:1074F000916400004D680000748BFF1F65670000F9
:1075000081680000108FFF1F05700000816A000075
:10751000288CFF1F29700000F5640000308BFF1FCE
:10752000955F0000756200007C8FFF1F4D700000AA
:10753000E96A0000048CFF1FA55F0000516B00008A
:10754000248DFF1FB55F0000C16B0000BC8BFF1FC7
:10755000C55F000055650000A08AFF1FD55F0000D1
:10756000BD680000948CFF1FE55F0000BD6D00004A
:10757000388EFF1FF55F0000F1680000FC8FFF1FD1
:1075800005600000296C0000CC8DFF1F1560000015
:10759000916C0000C48AFF1F25600000256900006F
:1075A000348FFF1F85670000F96C0000148EFF1FE9
:1075B00035600000CD700000E88AFF1F45600000C4
:1075C000596900007C8AFF1F55600000C1690000F6
:1075D000CC8FFF1F65600000AD650000988BFF1F1A
:1075E0007560000005660000548AFF1F856000007A
:1075F0000C8BFF1FC88EFF1F5D66000095600000AA
:10760000B5660000A56000000D670000308AFF1F0E
:10761000C489FF1FF08FFF1F696D0000C560000067
:10762000996D0000D5600000B57B0000B5600000DA
:10763000F0B5461C83B00D460127032336B22AB2AB
:10764000044631468DE888002448ADB204F042F883
:107650000C23AA1C12B200930197052321B21F48E4
:1076600004F038F81E4A1F4B12881B68BA422AD011
:1076700023D3022A10D11C4CA3F6CA0384FB032493
:107680001C44DB17C3EB24140A2CA8BF0A2424EAE9
:10769000E474A2B223B202E000231A461C460D3560
:1076A000AA1A01200093019012B2314603230B481D
:1076B00003F08EFF204603B0F0BD0C4CA3F6FC0394
:1076C00084FB0324DDE7084CA3F6980384FB032422
:1076D0001C44DB17C3EBE404D6E700BF109EFF1F7A
:1076E000F89CFF1F7C9DFF1F898888881F85EB51B0
:1076F0002DE9F0438FB283B0DFF84C80BD1D461DED
:107700002DB204B236B24FF001090AB22346314617
:1077100040460095CDF8049003F08CFF2A4633468E
:10772000214640468DE8200203F084FF07F10C0259
:107730000095334612B22146CDF80490404603F03E
:1077400079FF03B0BDE8F083109EFF1F2DE9F043E1
:10775000804685B0002956D10121304804F000FB55
:107760002F4998F8062098F8083011F802909945AA
:1077700022DA4FEA89064D460C24D8F80C30274807
:107780009B595F6822B2002104F0E6FA384609F0FE
:1077900057F939460246214804F078FC1F4804F0A6
:1077A0008BFC98F8083001350934AB42A4B206F1DD
:1077B000040601DD422CE0D1B9F1000F13D109F12B
:1077C000060999450CDA3C2301213B2203910293DF
:1077D0000093019239233F223A21104803F0E4FF3D
:1077E00005B0BDE8F0830F2301213B2203910293F2
:1077F0000093019239230C223A21084803F0D4FF68
:1078000098F80830DBE700213423009301913F23EF
:107810000C22024803F0DCFE9EE700BF109EFF1F13
:10782000089EFF1F10B5104C0121204604F09EFA5F
:107830002046012104F094FA20463422552104F018
:107840008BFA20460222094904F020FC204605223A
:10785000074904F01BFC204604F02EFC2046BDE83E
:10786000104003F09BBC00BF109EFF1F842101004D
:107870008821010070B50D46064609F0E1F800EBDD
:1078800040008400002D36D0284609F0D9F800EBDE
:107890004000400023185B1003F16001091A282200
:1078A00009B21748C3F1600404F056FA01211448E4
:1078B00004F056FA284609F0C3F829460246104853
:1078C00004F0E4FB0E4804F0F7FB02210C4804F03E
:1078D00047FA21B221220A4804F03EFA304609F064
:1078E000AFF831460246064804F0D0FB0448BDE834
:1078F000704004F0E1BB6410C4F16004E5E700BF30
:10790000109EFF1F184B70B5B3F9003083EAE37483
:10791000A4EBE374002B82B0A1B21EDB68466D4677
:10792000012300E0134603EB830252009442F9DA8C
:107930000E4E91FBF3F286FB03E403FB1211DB17FF
:107940003032D3EBA40389B205F8012BF1D11946EB
:107950002B70FFF78FFF02B070BD2D238DF8003024
:107960000DF101056846DBE7149DFF1F676666663B
:1079700010B50D4B1B5C51F82340237884B013B134
:10798000012004B010BD04AA01A942F8103D204610
:10799000A3699847A38A9B07F2D401A80099FFF72F
:1079A00069FF012004B010BDF49DFF1F2DE9F04FC9
:1079B0002F4DDFF8CCB0DFF8C4A0DFF8C8900FCDB2
:1079C00091B003AC0FC40FCD0FC40FCD0FC42B6803
:1079D00023600025A8462F462E4600E09846BAF8B8
:1079E000003024495BF8232028461123F8F746FE8F
:1079F00000EBC00400EB840089FB00340444C01792
:107A0000C0EB6434C4F13C00C6F13C0207F1410113
:107A1000012600B208F1410300901BB2019612B298
:107A200009B2154803F006FE08EB060305F211152E
:107A30003C2B2646ADB24746D0D134226B210E48AE
:107A400004F08AF900210C4804F08AF90B4B1B88DA
:107A500010AA02EB830353F8344C204608F0F0FFE1
:107A600002460548214611B0BDE8F04F04F00EBBB8
:107A7000CC190100E4130100109EFF1F869BFF1F1D
:107A8000E01101000900028010B5424C424882B06A
:107A900003F078FA2378C3B906213F4804F060F96F
:107AA0002378012B37D90A22022B11463A486BD092
:107AB00004F052F939490322374804F0E7FA36480E
:107AC00002B0BDE8104004F0F7BA354B1A78012136
:107AD0000523002A35D10191009311462E4803F069
:107AE000F9FD304B1A78002A36D005230122019285
:107AF000009300220A21284803F06AFD2A4B1A78D5
:107B0000002A35D101210523019100931421224837
:107B100003F0E0FDC0E7254C2388092B32D9632B05
:107B20008CBF0A211F210A221B4804F015F9218865
:107B3000194804F011FB184802B0BDE8104004F0E9
:107B4000BBBA0022019100931146134803F040FD97
:107B5000144B1A78002AC8D1052301210191009302
:107B60000A210D4803F0B6FD0F4B1A78002AC9D040
:107B7000012205230192009300221421064803F0FC
:107B800027FD89E73021CEE704F0E6F80322084913
:107B900092E700BF8B9EFF1F109EFF1F94210100E4
:107BA000E29DFF1FE39DFF1F989DFF1F949DFF1FF8
:107BB00090210100F8B56D4D287840B96C4B1B68D9
:107BC00099425CD36B4A012313702B70F8BD0C46AD
:107BD00000266948664F03F0D5F904F6AC533246E7
:107BE00065483B6031212E7004F0B6F801216248EF
:107BF000624D04F0BBF831465F4804F0B1F805224D
:107C00005F495D4804F042FA5B4804F055FA0C22E3
:107C10001021594804F0A0F80B225A49564804F0A4
:107C200035FA05225849544804F030FA524804F015
:107C300043FA564B50481C68A4F69803C3EB031351
:107C400085FB03251D441021DB172022C3EB65258E
:107C500004F082F840F6CC339C4205F124054FF045
:107C600022014FF004000BDCFFF7E2FC484B1C88BC
:107C7000064674B3012C46D0022C41D00120F8BD39
:107C8000FFF736FD092243493B4804F0FFF92A2259
:107C90001021394804F060F83F4C374884FB053424
:107CA000EB17C3EBA404214604F056FA01223B492A
:107CB000314804F0EBF904EB8401A5EB41012E48B7
:107CC00004F04AFA012236492B4804F0DFF901207A
:107CD000F8BD34491022284804F0D8F9264804F0A9
:107CE000EBF92A221021244804F036F831462248C4
:107CF00004F032FA07222C491F4804F0C7F9CBE7F9
:107D00000C222A49E7E70C2229491B4804F0BEF956
:107D1000194804F0D1F92A221021174804F01CF860
:107D2000314615481C4E04F017FA07221E49124826
:107D300004F0ACF986FB0536EB17C3EBA60631461B
:107D40000D4804F009FA224614490B4804F09EF944
:107D500006EB8601A5EB4101074804F0FDF9224638
:107D60000F49054804F092F92046F8BD788AFF1FB4
:107D70008C9EFF1F889EFF1F109EFF1F3B773B9826
:107D800098210100A0210100882101007C9DFF1F96
:107D9000F89CFF1FAC210100676666661029010090
:107DA00088280100B8210100CC210100E421010054
:107DB000D42101002DE9F041754C2278002A0546B6
:107DC0000F4614BF4FF001084FF000084ED1714E1E
:107DD0003368CB1AB3F5FA6F04D86B78A3B9404671
:107DE000BDE8F0816C4B6D486D49DFF8D0E11A7049
:107DF000012303700988237026208EF8002000F0EC
:107E0000F1FD6B78002BEAD03760F9F753FF654A34
:107E1000654B6649127828781B78097802EB430392
:107E2000421E03EB81030E2AD9D801A151F822F09A
:107E3000217F0000ED7E0000DF7D0000217F00003B
:107E4000DF7D0000DF7D0000DF7D0000D57E0000CB
:107E5000DF7D0000877E0000DF7D0000DF7D000009
:107E6000DF7D0000DF7D0000837E0000AF215048F1
:107E7000484E02F037FEFFF707FE002337602370FD
:107E8000ABE705F01BFB4A4803F07CF802214848A9
:107E900003F066FF0F222321454803F05DFF052212
:107EA0004449434804F0F2F8414804F005F91E2221
:107EB00023213F4803F050FF05223F493C4804F08E
:107EC000E5F83B4804F0F8F8394803F067F900F0AA
:107ED000ADFC84E7394D2B78012B50D9304B26204F
:107EE000198800F07FFD00232B7078E7002B3FF40A
:107EF00076AF013B324A32F81330002B3FF46FAFBC
:107F0000274C304825492D4A23804FF00108002393
:107F1000037081F8008082F80080FFF7B5FD5EE70E
:107F200093B1013B264A32F8131019B31C4B254D6F
:107F30001A4C224A19800026012326202E70237015
:107F4000137000F04FFD15E0154C1E4922880B7090
:107F500004284FF6FF7002F1FF310CBF01220246E8
:107F60000A440E4E154D02F07F020132012122809B
:107F700031702B70FFF788FD4FF001082FE706499D
:107F8000064A01230020087013702370A6E700BF83
:107F9000788AFF1F849EFF1F889EFF1F769BFF1F0E
:107FA000949DFF1FE29DFF1FE39DFF1F989DFF1FF4
:107FB000109EFF1FF4210100FC2101008B9EFF1F7A
:107FC000D89CFF1FD49BFF1F2DE9F04F05468BB0B7
:107FD0000F46AD480121164603F0C8FEAA8812F0EC
:107FE000010440F0B080DFF8CC8298F80030002B1C
:107FF0007DD1AB79A54AD15CA1B9DFF8BCA2797873
:108000001AF8039041B339780139072900F2B78093
:10801000DFE811F0F1005401B5006C01B500B500C6
:10802000B500E9007C78002C00F0CA800139EC68CA
:10803000387854F82170FC68411EB4F80080072994
:1080400000F2A780DFE811F074015901A5006C016E
:10805000A500A500A5009F00DFF854A2DAF80020D3
:10806000B21AB2F5967F75D9894A107801281ABFDD
:10807000012010701170874A18BF0146D05CC0EB18
:108080000900C0B2FFF7F8F80124CAF80060AB8815
:108090009B0770D57B78002B6DD0F9F70BFE7E4BDC
:1080A0007E4A7F481B78127839780078022515FBC4
:1080B00002330A2903EB800300F04E810C295AD1C8
:1080C000002B58D003F11900764E774A013B00216E
:1080D000400080B226F813100123157088F8003094
:1080E00000F080FC714B032220461A702FE0664896
:1080F00002F048FF0121644803F032FE6248224644
:10810000214603F029FEAB88580725D42C68204669
:1081100008F096FC214602465B4803F0B7FF5A4838
:1081200003F0CAFF092201238DE80C0000217F2300
:10813000554803F07FFA00212846FFF707FB00238C
:1081400088F8003055E7AB683146384698470BB0A1
:10815000BDE8F08F0846FAE72B6804A8984704A802
:1081600008F06EFC04A90246474803F08FFF46481A
:1081700003F0A2FFD6E720460BB0BDE8F08F002445
:108180000AF8039083E70021D1543846FB699847E9
:10819000FC68A4F80080002725223C238DE8840099
:1081A00041211822384803F013FAE968A879FFF74B
:1081B000DFFB374A3E4B17701E600BB0BDE8F08FF7
:1081C0003B490A68B21AB2F5967FD4D9304F0E6097
:1081D0003E78012E00F0B480E968184601233B7018
:1081E000FFF7C6FBB3E7304AE9791170012288F83E
:1081F00000200024C4E72A7A013A4A45BFDD09F18C
:108200000104E4B2A145BAD0224E16F803B0CBEB7C
:108210000900C0B20021FFF72FF82B7A052BD946B1
:108220001BD9CBEB0402042A40F3AE80A4F1040B6B
:10823000BBF1000FC0F2B080063B5B45A8BF5B46B8
:108240005FFA83F9AA791348B15C994205D000F826
:10825000029001212846FFF779FAC9EB0400C0B269
:1082600001210B4EFFF708F8002134230191009300
:108270000548317040230B223F21A14603F0A8F9A5
:108280000124AB797CE700BF109EFF1F789EFF1F83
:10829000899EFF1F089EFF1FE29DFF1FE39DFF1F9A
:1082A000989DFF1FD89CFF1F889EFF1F8B9EFF1F5E
:1082B000749EFF1F788AFF1FF49DFF1F0FFA89F13C
:1082C000E868604C50F821602168049134785E4978
:1082D00004980860002C71D0012C7FF450AF5B4AE9
:1082E000317A88F800401170002449E7B9F1000F95
:1082F00050D009F1FF34E4B284E7B98A01F00401F7
:1083000089B200293FF440AF3B6A03929847039A31
:1083100000283FF43DAFAB79FC680021D15438E729
:108320007B8A43453CD908F101081FFA88F830E7F9
:108330003B8A43453BD208F1FF381FFA88F828E70B
:1083400025238DE8180042483C703C231822412127
:1083500003F03EF93046FAE6002B3FF40CAF3D4AFD
:108360003D4E1188394A03F11900013B400080B2AB
:1083700026F81310012388F80030157000F032FB46
:10838000364B20461D70E2E6002A3FF755AF04F158
:10839000FF3B4DE74C46F3E64FF000094B4651E7F3
:1083A000BB8ADA077FF5F5AEB7F81080F1E6BB8A35
:1083B000D9077FF5EEAEB7F81280EAE62849C85C27
:1083C000C0EB090009F1010EC0B201214FF0340BDE
:1083D00002F803E0FEF750FFB6681D480194402301
:1083E0000B223F210124CDF800B003F0F1F8402327
:1083F0000B223F211648CDF800B0019403F06AF932
:108400002146134803F0ACFC304608F019FBA0EB02
:10841000800000F15F0109B20F220D4803F09CFCBF
:10842000304608F00DFB31460246094803F02EFEA7
:10843000074803F041FEE968A879FFF799FAAB799C
:108440009EE600BFCC9EFF1F749EFF1F889EFF1FED
:10845000109EFF1F949DFF1FD89CFF1F8B9EFF1F28
:10846000089EFF1F2DE9F047DFF808926D4B99F841
:1084700000601B68DFF800A282B0003601934FF065
:10848000030018BF0126019F9AF8008004F0CEFC7B
:108490000546042004F0CAFC0446052004F0C6FC8E
:1084A000800040EA4404062004F0C0FC2C4364B27F
:1084B0005D4944EAC0000A7880F00F03DBB29A42BB
:1084C0005A4A3CD01760002259480B7003788DF847
:1084D00000808DF8012053B3564A12684EF6602191
:1084E000BA1A8A4219D8022B59D0012B5FD0062B19
:1084F00048D0032B63D0042B69D0052B77D0072BF2
:108500007DD0082B00F08380092B68D016B14A4833
:1085100002F044FE02B0BDE8F087484A484C002310
:108520000121237003701360938089F800103A468C
:1085300069464448FFF748FD3043C6B2E6E7126893
:10854000BA1A1E2A6BD99AF80020934222D0394CCD
:108550003D488AF80030012B276082EA0302076059
:108560009846B1D0042BAFD137480068381AB0F51F
:10857000C87FA9D9354C2068381A3228A4D9276079
:108580001A46A1E73A4669463148FFF71DFD3043D8
:10859000C6B2BBE7012B4FF00002E3D1E4E73A4655
:1085A00069462C48FFF710FD3043C6B2AEE73A46A5
:1085B00069462948FFF708FD3043C6B2A6E73A46A8
:1085C00069462648FFF700FD3043C6B29EE73A46AB
:1085D00069462348FFF7F8FC3043C6B296E73A46AF
:1085E00069462048FFF7F0FC3043C6B28EE73A46B2
:1085F00069461D48FFF7E8FC3043C6B286E73A46B5
:1086000069461A48FFF7E0FC3043C6B27EE73A46B7
:1086100069461748FFF7D8FC3043C6B276E7002218
:1086200052E700BFCC9EFF1F909EFF1FFC9DFF1FC7
:10863000889EFF1F809EFF1F109EFF1F789EFF1FBA
:108640008A9EFF1F08200100949EFF1F049EFF1FAB
:1086500038200100601F0100641E0100DC270100BA
:10866000CC270100541E0100BC1E0100441F010064
:10867000F08FFF1F788AFF1F009EFF1F28B1102870
:10868000044BA8BF102018607047024B01201860EF
:10869000704700BF989EFF1F38B50F4D2B78013BE8
:1086A00001381B02C4B203F47063200443F4404356
:1086B00043F00C0300F4FE00184305F01FFD28688A
:1086C000013860F03F00C0B204F046FD2046BDE82E
:1086D000384004F041BD00BF989EFF1F70B5124D99
:1086E0002B78013B1B0203F47063064643F43043CE
:1086F0000806320400F0FE4043F00B03034302F48B
:10870000FE0018430C4605F0F9FC2868013860F0BB
:108710004F00C0B204F020FD304604F01DFD20469D
:10872000BDE8704004F018BD989EFF1F70B5124D53
:108730002B78013B1B0203F47063064643F410439D
:108740000806320400F0FE4043F00903034302F43C
:10875000FE0018430C4605F0D1FC2868013860F093
:108760006F00C0B204F0F8FC304604F0F5FC20467F
:10877000BDE8704004F0F0BC989EFF1F38B5104D66
:108780002B78013B1B0203F47063044643F410434F
:10879000000443F0090300F4FE00184305F0AEFCAA
:1087A0002868013860F06F00C0B204F0D5FC2046A4
:1087B00004F0D2FC0020BDE8384004F0CDBC00BF7E
:1087C000989EFF1F38B50E4D2B78013B1B0203F41A
:1087D0007063044643F45043000443F00D0300F477
:1087E000FE00184305F08AFC2868013860F02F006D
:1087F000C0B204F0B1FC2046BDE8384004F0ACBC87
:10880000989EFF1F08B5002005F042FD0028FAD110
:1088100008BD00BF08B564210720FFF75FFF7F2177
:108820000B20BDE80840FFF759BF00BF10B500217D
:108830007B20FFF753FF0024E0B2FFF79FFF0134D6
:10884000022004F029FB802CF6D110BD10B504469F
:108850004FF4406004F030FC04F088FC2CB1102C84
:10886000044BA8BF10241C6010BD024B01241C60E7
:1088700010BD00BF989EFF1F10B5044641F0E000F8
:1088800004F06AFC04F07F0004F066FCC4F3C61038
:10889000BDE8104004F060BC38B5134D2B78044699
:1088A00041F6FF72A0F50050824203F1FF33A8BFEA
:1088B00002461B0202F5005203F47063100443F4F5
:1088C000604343F00E0300F4FE005204184302F02C
:1088D000FE42104305F012FC296801392046C9B256
:1088E000BDE83840FFF7C8BF989EFF1F38B5044663
:1088F0000D46F02004F030FC35B1254414F8010B8E
:1089000004F02AFCAC42F9D1F720BDE8384004F06D
:1089100023BC00BF00B50B4B83B002469988186892
:108920000090032AADF8041002D903B05DF804FBEF
:10893000684606218DF80520FFF7D8FF03B05DF8E3
:1089400004FB00BF4828010000B50B4B024683B072
:10895000186899880090131F4C2BADF8041002D9A9
:1089600003B05DF804FB684606218DF80520FFF78B
:10897000BDFF03B05DF804FB50280100030203F4BF
:10898000FE43C0F3C6101843704700BF0378407819
:10899000DB0103F47E5300F07F001843704700BFF3
:1089A00082B002AA114642F8040D002012F8013BE1
:1089B00003F07F03914243EA0020F7D102B07047F1
:1089C000003210B403884FF0010404FA01F418BF18
:1089D000012202FA01F123EA04020A43028010BCD8
:1089E000704700BF70B5CEB20C46054603F0E6FDF9
:1089F000864203D03146284603F0FAFD0135284669
:108A000003F0DCFD240A844205D021462846BDE857
:108A1000704003F0EDBD70BD38B5054603F0CEFDE6
:108A20004FF0000460F30704681C03F0C7FD60F317
:108A30000F24A0B238BD00BFF8B504460020FFF7F0
:108A4000EBFF002C00F051814FF4AF610220FFF7E3
:108A5000C9FF04204FF47A61FFF7C4FF0B2004F034
:108A6000E5F9002840F05E864FF496610620FFF796
:108A7000B9FF4FF4FA610820FFF7B4FF4FF4FA6131
:108A80000A20FFF7AFFF40F6B8310C20FFF7AAFF2E
:108A90004FF42F612220FFF7A5FF40F6AC512420B0
:108AA000FFF7A0FF7D212A20FFF79CFF0C210E205D
:108AB000FFF798FF01211020FFF794FF02211220F9
:108AC000FFF790FF00211420FFF78CFF00211620F4
:108AD000FFF788FF02211820FFF784FF01211A20E9
:108AE000FFF780FF01211C20FFF77CFF04211E20DF
:108AF000FFF778FF14212020FFF774FF01212620C3
:108B0000FFF770FF03212820FFF76CFF04212C20C2
:108B1000FFF768FF14212E20FFF764FF00213020AB
:108B2000FFF760FF0C213220FFF75CFF00213420AB
:108B3000FFF758FF00213620FFF754FF00213820AF
:108B4000FFF750FF00213A20FFF74CFF00213C20A7
:108B5000FFF748FF00213E20FFF744FF002140209F
:108B6000FFF740FF00214220FFF73CFF1F21442078
:108B7000FFF738FF13214620FFF734FF0E2148206E
:108B8000FFF730FF11214A20FFF72CFF0A214C206C
:108B9000FFF728FF00214E20FFF724FF0621502079
:108BA000FFF720FF02215220FFF71CFF0C21542069
:108BB000FFF718FF00215620FFF714FF002158206F
:108BC000FFF710FF01215A20FFF70CFF08215C205E
:108BD000FFF708FF0A215E20FFF704FF0021602055
:108BE000FFF700FF04216220FFF7FCFE0121642053
:108BF000FFF7F8FE00216620FFF7F4FE0B21682046
:108C0000FFF7F0FE7F216A20FFF7ECFE00216C20C9
:108C1000FFF7E8FE00216E20FFF7E4FE0021702040
:108C2000FFF7E0FE00217220FFF7DCFE0021742038
:108C3000FFF7D8FE1F217620FFF7D4FE13217820FE
:108C4000FFF7D0FE0E217A20FFF7CCFE11217C2009
:108C5000FFF7C8FE0A217E20FFF7C4FE1F218020F7
:108C6000FFF7C0FE13218220FFF7BCFE0E218420F7
:108C7000FFF7B8FE11218620FFF7B4FE0A218820F5
:108C8000FFF7B0FE00218A20FFF7ACFE00218C2008
:108C9000FFF7A8FE00219620FFF7A4FE00219820F0
:108CA000FFF7A0FE00219A20FFF79CFE05219C20E3
:108CB000FFF798FE06219E20FFF794FE0021A020DA
:108CC000FFF790FE27210020FFF78CFE0220FFF720
:108CD000A3FEB0F5805F034616D34FF4AF610220C8
:108CE000FFF780FE4FF4AF630EE04FF6FF7398423C
:108CF0003FF4AAAE272840F021850220FFF78CFE22
:108D0000B0F5805F0346E8D2D24A04201380FFF713
:108D100083FEB0F5805F034680F05184CE4A062082
:108D20001380FFF779FEA0F52F739BB2B3F57A6F2E
:108D3000024606D940F628210620FFF753FE40F6EA
:108D40002822C64B08201A80FFF766FEA0F52F7375
:108D50009BB2B3F57A6F024606D940F6E44108208B
:108D6000FFF740FE40F6E442BD4B0A201A80FFF7B1
:108D700053FEA0F5FA739BB240F6AC518B4202460B
:108D800006D94FF4FA610A20FFF72CFE4FF4FA627D
:108D9000B44B0C201A80FFF73FFEA0F5FA739BB28C
:108DA00040F6AC518B42024606D940F6B8310C2051
:108DB000FFF718FE40F6B832AB4B0E201A80FFF7D3
:108DC0002BFE1828034600F21584A84A10201380B1
:108DD000FFF722FE431E9BB20F2B024604D901214E
:108DE0001020FFF7FFFD0122A14B12201A80FFF790
:108DF00013FE0A28034600F2F7839E4A14201380CC
:108E0000FFF70AFE0128034604D900211420FFF7CA
:108E1000E9FD0023984A16201380FFF7FDFD7F2807
:108E2000034600F2DB83954A18201380FFF7F4FD18
:108E30000428034600F2CC83914A1A201380FFF7DE
:108E4000EBFD0C28034600F206848E4A1C2013809A
:108E5000FFF7E2FD0428034600F2F7838A4A1E204A
:108E60001380FFF7D9FD0928034600F2E883874AFB
:108E700020201380FFF7D0FD4628034600F2D98357
:108E8000834A22201380FFF7C7FDA0F5FA739BB237
:108E900040F6AC518B42024606D94FF42F61222096
:108EA000FFF7A0FD4FF42F627A4B24201A80FFF7C2
:108EB000B3FDA0F5FA739BB240F6AC54A342024650
:108EC00004D921462420FFF78DFD2246724B26202F
:108ED0001A80FFF7A1FD7F28034600F2A4836F4AA2
:108EE00028201380FFF798FD0628034600F295839B
:108EF0006B4A2A201380FFF78FFDA0F132039BB24B
:108F0000B3F5967F024604D97D212A20FFF76AFD3A
:108F10007D22644B2C201A80FFF77EFD0C2803462F
:108F200000F27583604A2E201380FFF775FD1E281E
:108F3000034600F266835D4A30201380FFF76CFD24
:108F40000928034600F2E883594A32201380FFF7CC
:108F500063FD1E28034600F2D983564A342013804D
:108F6000FFF75AFD7F28034600F2CA83524C362091
:108F70002380FFF751FD7F28034600F2BB83382092
:108F80006380FFF749FD7F28034600F2AD833A2056
:108F9000A380FFF741FD7F28034600F29F833C201A
:108FA000E380FFF739FD7F28034600F291833E20DE
:108FB0002381FFF731FD7F28034600F283834020A1
:108FC0006381FFF729FD7F28034600F27583422065
:108FD000A381FFF721FD394D28804420FFF71CFDB8
:108FE0003028034600F26283354A46201380FFF79B
:108FF00013FD3028034600F25383324C482023806F
:10900000FFF70AFD3028034600F244834A206380BC
:10901000FFF702FD3028034600F236834C20A38080
:10902000FFF7FAFC3028034600F228834E20E38045
:10903000FFF7F2FC0128034604D900214E20FFF778
:10904000D1FC0023204A50201380FFF7E5FC431E8B
:109050003CE000BF009CFF1FB89DFF1F789DFF1FD5
:10906000909DFF1F5A9DFF1F989BFF1F709BFF1F26
:10907000149DFF1F4A9DFF1FF69BFF1F749BFF1F40
:10908000049CFF1FB09BFF1FAA9BFF1FA09BFF1FFD
:10909000A09DFF1F0C9DFF1F089DFF1F949DFF1F9C
:1090A000649DFF1FB09DFF1F869BFF1FF09BFF1F4E
:1090B000C49DFF1F929DFF1FD89CFF1F909BFF1F09
:1090C000929BFF1F689DFF1FA89BFF1F9BB20B2B4E
:1090D000024604D906215020FFF784FC0622CE4B1D
:1090E00052201A80FFF798FC0428034600F2C08241
:1090F000CA4A54201380FFF78FFC431E9BB21D2BDE
:10910000024604D90C215420FFF76CFC0C22C44BFE
:1091100056201A80FFF780FC0128034604D900215D
:109120005620FFF75FFC0023BE4A58201380FFF74C
:1091300073FC7F28034600F29582BB4A5A201380B5
:10914000FFF76AFC431E9BB2092B024604D901219A
:109150005A20FFF747FC0122B44B5C201A80FFF72E
:109160005BFC431E9BB2102B024604D908215C20F5
:10917000FFF738FC0822AE4B5E201A80FFF74CFC4C
:10918000431E9BB21D2B024604D90A215E20FFF725
:1091900029FC0A22A74B60201A80FFF73DFC022819
:1091A000034600F2FA81A44A64201380FFF734FCDE
:1091B0000128034604D901216420FFF713FC012391
:1091C0009E4A62201380FFF727FCC31E9BB2012B2F
:1091D000024604D904216220FFF704FC0422984BC4
:1091E00066201A80FFF718FC7F28034600F2CF8123
:1091F000944A68201380FFF70FFC7F28034600F293
:10920000C081914A6A201380FFF706FC7F2803463D
:1092100000F2B1818D4A6C201380FFF7FDFB02281C
:10922000034600F2A2818A4A6E201380FFF7F4FB06
:109230001928034600F29381864A70201380FFF7B5
:10924000EBFB0228034600F28481834A72201380DC
:10925000FFF7E2FB0628034600F275817F4A74207F
:109260001380FFF7D9FB0428034600F266817C4A8D
:109270008A201380FFF7D0FB0A28034600F25781AB
:10928000784A8C201380FFF7C7FB0428034600F2BE
:109290004881754A98201380FFF7BEFB01280346DA
:1092A00004D900219820FFF79DFB00236F4A9A20E4
:1092B0001380FFF7B1FB0128034604D900219A204F
:1092C000FFF790FB00236A4A96201380FFF7A4FB68
:1092D0000B28034600F21F81664A9C201380FFF78B
:1092E0009BFB831E9BB2032B024604D905219C20C5
:1092F000FFF778FB0522604B76201A80FFF78CFB86
:109300003028034600F201815C4A78201380FFF781
:1093100083FB3028034600F2F280594C7A202380E8
:10932000FFF77AFB3028034600F2E3807C2063805D
:10933000FFF772FB3028034600F2D5807E20A38021
:10934000FFF76AFB3028034600F2C7808020E380E5
:10935000FFF762FB3028034600F2B980494A8220B9
:109360001380FFF759FB3028034600F2AA80464CD1
:1093700084202380FFF750FB3028034600F29B80B7
:1093800086206380FFF748FB3028034600F21181F6
:109390008820A380FFF740FB3028034600F20381BA
:1093A000A020E380FFF738FB0128034604D9002101
:1093B000A020FFF717FB0023344A9E201380FFF7FD
:1093C0002BFBC31E9BB20C2B04D99E200621FFF75A
:1093D00009FB06202B88DFF8D4E02D4F2D4A2E4DB7
:1093E0002E4E2F4C2F4903F0010CAEF800C0C3F3F2
:1093F000400EA7F800E0C3F380071780C3F3C0074F
:10940000294A2F70C3F30017C3F34015C3F3801329
:10941000378025804CE000BFA489FF1F2E89FF1FE5
:10942000A689FF1FE49BFF1F969DFF1F6C9BFF1FDC
:10943000AA89FF1F2C89FF1F049DFF1F609DFF1F2E
:10944000B29BFF1FA29DFF1FDC9BFF1FA29BFF1F64
:10945000609BFF1FE49DFF1FF89CFF1FC09DFF1F27
:10946000889DFF1F169DFF1F029DFF1FC29BFF1FB0
:10947000E89BFF1F549DFF1F889BFF1F9A9BFF1FA8
:10948000E89CFF1F9C9BFF1FF09CFF1FDC9DFF1FA4
:10949000C09BFF1FF29BFF1FFB9CFF1F069DFF1F32
:1094A000629DFF1F1C9DFF1F9089FF1F569DFF1F80
:1094B0000B801080F8BD0E218420FFF793FA0E2355
:1094C0005EE713218220FFF78DFA13234FE71F2158
:1094D0008020FFF787FA1F2340E70A217E20FFF74D
:1094E00081FA0A2332E711217C20FFF77BFA11234E
:1094F00024E70E217A20FFF775FA0E2316E71321D1
:109500007820FFF76FFA132307E71F217620FFF774
:1095100069FA1F23F8E600219620FFF763FA00237B
:10952000DAE600218C20FFF75DFA0023B1E6002186
:109530008A20FFF757FA0023A2E600217420FFF7E4
:1095400051FA002393E600217220FFF74BFA002323
:1095500084E600217020FFF745FA002375E600211C
:109560006E20FFF73FFA002366E600216C20FFF72C
:1095700039FA002357E67F216A20FFF733FA7F2369
:1095800048E60B216820FFF72DFA0B2339E600216E
:109590006620FFF727FA00232AE600216020FFF764
:1095A00021FA0023FFE50A218820FFF71BFA0A238E
:1095B000F6E611218620FFF715FA1123E8E64FF4AD
:1095C0007A610420FFF70EFA4FF47A63FFF7A6BB27
:1095D00002211820FFF706FA02232DE400211620AD
:1095E000FFF700FA00231EE402211220FFF7FAF928
:1095F000022302E40C210E20FFF7F4F90C23FFF7FD
:10960000E4BB14212E20FFF7EDF9142393E4042189
:109610002C20FFF7E7F9042384E403212820FFF737
:10962000E1F9032364E401212620FFF7DBF901239C
:1096300055E414212020FFF7D5F9142320E4042158
:109640001E20FFF7CFF9042311E401211C20FFF7AE
:10965000C9F9012302E401211A20FFF7C3F901230C
:10966000FFF7F3BB00215820FFF7BCF9002364E5A6
:1096700002215220FFF7B6F9022339E50A214C20D6
:10968000FFF7B0F90A23D1E411214A20FFF7AAF924
:109690001123C3E40E214820FFF7A4F90E23B5E4FB
:1096A00013214620FFF79EF91323A6E41F2144202F
:1096B000FFF798F91F2397E400214020FFF792F964
:1096C000002384E400213E20FFF78CF9002376E498
:1096D00000213C20FFF786F9002368E400213A20AE
:1096E000FFF780F900235AE400213820FFF77AF9C8
:1096F00000234CE400213620FFF774F900233EE4F8
:1097000000213420FFF76EF900232FE40C213220D2
:10971000FFF768F90C2320E400213020FFF762F9FD
:10972000002311E440F628210620FFF75BF940F6FC
:10973000E4410820FFF756F9FFF7A0B917287FF694
:1097400083A919287FF6F2A91B287FF60FAA1C28E7
:109750003FF424AA1E287FF629AA1F283FF42EAA28
:1097600020283FF447AA21283FF450AA22283FF49A
:1097700055AA23283FF45EAA24283FF48FAA25285F
:109780003FF494AA26287FF49DAAFFF793BA00BF5E
:10979000F8B5B32006F0C8FB204B214A054603CBA1
:1097A0001368C5F803001A0CA220C5F807102B8017
:1097B000AA70FFF7E3F82E46002426F80B0FA0B29C
:1097C000FFF72AF9FFF7DAF80234A22C26F8020F85
:1097D000F5D16C1E05F1AE064FF0FF3014F8013FD5
:1097E000082758400F4B40F300017A1E0B4012F03F
:1097F000FF0783EA5000F5D1B442EFD1C043FFF731
:10980000CFF83A46C5F8AF00B321284604F0C4FCAF
:109810002846BDE8F84006F08FBB00BF5C28010079
:10982000582801002083B8EDF0B50E4B0E4C0546CC
:1098300093E8070085B024682E88AD7801AB83E8F3
:109840000700270C184600220B21ADF804408DF8C4
:109850000670ADF80C608DF80E5004F09DFC05B05C
:10986000F0BD00BF6828010058280100F0B5124B78
:10987000124D1E68124F0FCD87B06C460FC495E88D
:10988000030044F8040B38683B79CDF80D00320C26
:10989000272021808DF802208DF81130ADF800606E
:1098A000FFF76CF80022ADF80B001221684604F0B7
:1098B00073FC07B0F0BD00BF5828010074280100F8
:1098C00088210100002004F0E3BC00BF02F02EBE9E
:1098D00070B5124C82B0002540230646294620462A
:1098E000009301958023202201F072FE2022294658
:1098F000204602F031FA2046012102F037FA3046C4
:1099000007F09EF831460246204602F0BFFB204693
:1099100002B0BDE8704001F041BC00BF109EFF1FC7
:10992000F0B5B22983B075D90546441E00F1AE06E4
:109930004FF0FF3014F8012F08275040404A40F301
:1099400000017B1E0A4013F0FF0782EA5000F5D1A8
:10995000B442EFD1C043FFF723F80146D5F8AF007A
:109960000190019A914202D0B2F17F2F0BD105F103
:109970000B00FFF70BF8A2280BD03248FFF7A8FF27
:10998000002003B0F0BD3048FFF7A2FF384603B017
:10999000F0BD05F10D00FEF7F9FF272840D10024A6
:1099A00040F6AC5613E004281AD0062821D0082827
:1099B0001FD00A2828D00C2822D1A1F5FA7292B221
:1099C000B24201D8FFF70EF80234A22C0ED004F1F7
:1099D0000D002844FEF7DAFF022C0146A0B2E2D1C6
:1099E000B1F5805FEED30234A22CF0D1012003B098
:1099F000F0BDA1F52F7292B2B2F57A6FE4D8E1E72B
:109A0000222801D0242811D1A1F5FA7292B2B242D3
:109A1000DAD8D7E70D48FFF75BFF002003B0F0BDB1
:109A20000B48FFF755FF002003B0F0BD2A28C9D12D
:109A3000A1F1320292B2B2F5967FC5D8C2E700BF5B
:109A40002083B8EDB8280100A42801008C2801006B
:109A5000CC28010003290CD970B5461C82B00546FC
:109A60000C46304603222A4907F058F810B102B0DC
:109A700070BD70470B2C05D905222649281D07F01B
:109A80004DF840B12448FFF723FF244802B0BDE859
:109A90007040FFF7C9BE05F10901032201A807F0D4
:109AA0008DF801A803221E4907F038F8D8B1032227
:109AB0001C4901A807F032F808B301A803221A498B
:109AC00007F02CF8B0B91948FFF702FFA11E89B2C0
:109AD0003046FFF725FF0028C9D0154802B0BDE881
:109AE0007040FFF7F5BE1348FFF7F2FEFFF750FE98
:109AF0001148F3E71148FFF7EBFE1148C6E711489C
:109B0000FFF7E6FE02B0BDE87040FFF7AFBE00BF52
:109B10005828010098210100E4280100F8280100DC
:109B2000FC280100242901003C29010040290100F2
:109B300054290100002901001429010068290100AD
:109B40007C290100282901002DE9F043174D2B68DD
:109B500083B081460F469046F3B1154E34880A19FA
:109B600092B218461146328006F05CFD28603A46F3
:109B70004946204402F06CFDB8F1000F09D031884D
:109B80002868FFF767FF286806F0D6F900232B60E6
:109B9000338003B0BDE8F083054E01930846318061
:109BA00006F0C2F9019B28601C46E0E7A09EFF1F5B
:109BB0009C9EFF1F10B51F4C4FF4FA70FCF75EF827
:109BC000204601F0DFF900221146204602F0C4F8D9
:109BD0002046012102F0CAF82046002102F0C0F818
:109BE0000B221549204602F051FA204602F064FA91
:109BF0000F221249204602F049FA204602F05CFA90
:109C00000F490722204602F041FA204602F054FA9A
:109C1000204601F0C3FA0B4B0B4A1A604FF4FA705E
:109C2000FCF72CF8FFF722FE0848BDE81040FFF7CC
:109C30004FBE00BF109EFF1F802901008C2901002C
:109C40009C29010058A0FF1F499B0000A429010086
:109C50000020704790F8392090F83800101A7047AB
:109C600090F8383090F839209A4205D95A1C0344AC
:109C700080F83820187E70474FF0FF30704700BFE3
:109C800090F8383090F839209A4286BF1B18187E19
:109C90004FF0FF30704700BF704700BF38B5054632
:109CA000B0F85E0090B195F85D301446C3F1210222
:109CB00094420CD805F13B001844224602F0C8FC3F
:109CC00095F85D30234485F85D30204638BD01208D
:109CD00014462871EEE700BFB0F85E306BB190F823
:109CE0005D30202B07D8C218013380F85D30012089
:109CF00082F83B107047012303710020704700BFBA
:109D00000023426980F8383080F8393080F85C30C0
:109D100080F85D3080F85E3080F85F3006CA30B47D
:109D20000D68046943662A4383660A60A37042692A
:109D300090F861301649146813441D7A5B7B01EB7F
:109D4000C5051B026D6803F4E06343F064032B60F8
:109D500090F8623013449D7CDB7D01EBC5011B0252
:109D6000496803F4E06343F064030B6021685368BF
:109D7000194205D0036927225A70036904229A7197
:109D8000036920225A71036980229A7030BC70479F
:109D9000D834010043690CCB12681A420CD0094B2D
:109DA00099420AD9084B9942036994BF1A220D229D
:109DB0005A70036904229A717047036927225A7006
:109DC000F7E700BF7F1A06003F420F0010B5026997
:109DD000D378DBB2D90604463DD510215806D170A0
:109DE00038D503F0040303F0FF02002B51D03D49A6
:109DF000626E00230B7084F85D30002A5BD09047C0
:109E000094F85D30002B56D02369D0229A702369D4
:109E100094F83B201A712369012284F85C20022205
:109E2000DA7010BD304B84F860009C424AD02F4B52
:109E30009C4252D094F8391013791F29DBB207D80D
:109E40002848007820B16018013184F83910037671
:109E50000223D37010BD5906C3D4917801F01001CC
:109E600001F0FF000029DDD013F001031ED194F8AA
:109E70005C1094F85D00884281BF4B1C091984F87E
:109E80005C3091F83B3013712369D0229A702269BB
:109E9000DEE7236984F83920C0229A702369114AC9
:109EA0001979012111700222DA7010BDC02393705C
:109EB00022691379CCE70122002384F85D2084F81D
:109EC0003B30A1E7626994F86130094913440322E9
:109ED000187A02F043FD2269ACE7626994F86130B8
:109EE0000449F3E7A49EFF1F3C90FF1FA890FF1FAB
:109EF000559F0000619F00000369DB7803F0200399
:109F000073B190F860300133DBB2012B80F8603020
:109F10001AD9426990F861301344187A02F09ABD58
:109F200070B5426903F0FF0590F8613013440446B0
:109F3000187A02F08FFDA36E5BB184F8385094F864
:109F40003900BDE87040184790F85F30002BE0D032
:109F5000704770BD0148FFF7CFBF00BF3C90FF1FA7
:109F60000148FFF7C9BF00BFA890FF1F2DE9F047C8
:109F7000374FDFF8E0903B68026982B006460093F5
:109F8000DDF800800021A025D3789B065BD53B68D7
:109F90000193019BC8EB03030F2BF5D949B1102B9B
:109FA000F2D000209070336980229A7002B0BDE830
:109FB000F087726996F8613013440521187A02F02F
:109FC00043FF726996F861301344012193F812A09F
:109FD000504602F039FF09240021504602F020FFCC
:109FE0002B46013BFDD10121504602F019FF2B46C3
:109FF000013BFDD1013CEFD1706996F8611001443D
:10A000004FF4A0720C7A4B7B09EBC4011B02496828
:10A0100003F4E06343F064030B6096F8623003449A
:10A02000997CDB7D09EBC1011B02496803F4E06305
:10A0300043F064030B60013AFDD13269D3789B068B
:10A040004FF00101A3D4012002B0BDE8F08700BFAA
:10A05000CC9EFF1FD8340100F0B503691222DA70DC
:10A060000269937803F0200385B004460D46002B67
:10A070005ED0B42393703C4922690B680093009E24
:10A0800005E00B680193019B9B1B042B42D8D378FE
:10A0900003F0200303F0FF00002BF2D094F85D30B2
:10A0A000002B31D04FF0000E4FF0020C04EB0E03EA
:10A0B00093F83B3013710B680393039F206907E00B
:10A0C0009B060DD50B680293029BDB1B052B28D842
:10A0D000C378DBB203F0020202F0FF06002AEFD0E1
:10A0E00080F803C02669F378DBB2DF0632462DD450
:10A0F0009F062BD5DB0731D40EF1010E94F85D30AD
:10A100005FFA8EFE7345D1D800201DBB002384F872
:10A110005E3004E09070236980229A70042005B0BC
:10A12000F0BD86702369802204209A7005B0F0BDCE
:10A1300003F0FF06FFF71AFF10B9042005B0F0BDC9
:10A14000236984F85F60B0229A7094E78023B3702B
:10A150000420DAE726698023B370D7E7BEF1000F49
:10A160000CBF02200320F6E7CC9EFF1F2DE9F04133
:10A1700006690025122780F8385080F83950F770AA
:10A18000D0F810C09CF802E00EF0200E88B0044613
:10A19000884615461E46BEF1000F49D0B4238CF800
:10A1A0000230784B21691A680092DDF800E006E081
:10A1B0001A6801920198CEEB0000042830D8C878C4
:10A1C00000F0200000F0FF070028F1D04FEA48021D
:10A1D00042F00102D2B20A711A680292DDF808E078
:10A1E000206906E01A6803920399CEEB0101052964
:10A1F0002AD8C17801F0020101F0FF070029F1D04F
:10A200004FF0020C80F803C02269D17811F01107D9
:10A2100022D12DBB002E0CBFA0238023937003E01E
:10A220008F70236980229A70384608B0BDE8F081AB
:10A230000EF0FF07FFF79AFE0028F5D0236984F897
:10A240005F70B0229A70ACE787702369802238462D
:10A250009A7008B0BDE8F081802393700027E3E78F
:10A26000012D75D0A021917021690A79BE466746FB
:10A270004FF0A80C1A680492049805E01A68059239
:10A28000059A121A052A4AD8CA7802F0020202F088
:10A29000FF08002AF2D0CF702169CA78D2B212F03A
:10A2A000100F08465AD1920658D5013DEDB2012D46
:10A2B00049D0BEF11F0F3BD90A79012DDAD11A68B6
:10A2C0000692069D05E01A680792079A521B052A16
:10A2D00046D8C27802F0020202F0FF01002AF2D052
:10A2E0000223C3702269D378DBB2D9063AD49B0625
:10A2F00034D5B023BEF11F0F93703FD8226904EB11
:10A300000E0312791A760EF1010E5FFA8EFE16B167
:10A31000236980229A7084F839E0774684E781F8CF
:10A320000280236980229A70774684F839E07BE7BF
:10A3300004EB0E0291F8048082F818800EF1010EF1
:10A340005FFA8EFEB9E781F802C021690846B0E7DE
:10A35000A82191702069BE460279B0E7774663E78D
:10A360008170DEE71021A023D170013BFDD122696D
:10A37000937803F0F7037746937055E723691B79C9
:10A38000C5E700BFCC9EFF1F0148FFF71FBD00BF00
:10A390003C90FF1F0148FFF719BD00BFA890FF1FA9
:10A3A000704700BF38B5144C037801225B000546A6
:10A3B000204684F83B3084F85E2084F85D20FFF767
:10A3C0008BFC20460021FFF747FE0B4C2978012328
:10A3D00020461A46FFF7CAFE0128F6D194F8383015
:10A3E00094F839209A4205D9E218013384F83830BC
:10A3F000107E38BDFF2038BD3C90FF1F38B51B4C88
:10A40000037801225B000546204684F83B3084F83F
:10A410005E2084F85D20FFF75FFC20460021FFF7F7
:10A420001BFE124C2978204601230222FFF79EFED4
:10A430000228F6D194F8382094F839108A420FD2C5
:10A44000531CDBB2A018994284F83830007E0AD938
:10A45000234402321B7E84F8382040EA032038BDB2
:10A460004FF6FF7038BD40F47F4038BD3C90FF1F71
:10A470000C2901D9002070470231490001F0FE018A
:10A48000FFF7BCBF70B50C4C0378164601255B0086
:10A49000204684F83B3084F85E5084F85D50FFF726
:10A4A0001BFC31462046FFF717FC29462046BDE835
:10A4B0007040FFF7D1BD00BF3C90FF1FF8B50546C7
:10A4C0000F461646412421463A462846FFF7DAFF52
:10A4D000611C0234C9B232462846E4B2FFF7D2FF0B
:10A4E000592CF0D1F8BD00BF38B504460D463548AB
:10A4F000FFF706FC6322802120462570FFF7C2FF8C
:10A50000012002F0C9FC204600225E21FFF7BAFFBD
:10A5100020465D21FFF746FF242801D0002038BDEA
:10A52000204606220C21FFF7C9FF204601222B21DD
:10A53000FFF7A8FF204601222C21FFF7A3FF2046AA
:10A540000E222D21FFF79EFF204600222E21FFF72D
:10A5500099FF204601222F21FFF794FF2046052274
:10A560003021FFF78FFF204601223121FFF78AFFBC
:10A57000204600223221FFF785FF204600223321AA
:10A58000FFF780FF204600223421FFF77BFF2046A3
:10A5900000223521FFF776FF204600225B21FFF7DE
:10A5A00071FF204610225C21FFF76CFF204620221D
:10A5B0005D21FFF767FF20468F225E21FFF762FFD4
:10A5C000012038BD3C90FF1F10B4047F4160022C75
:10A5D000C26002D010BC01F0D7BB836810BC184722
:10A5E00090E80C00F0B41C6859682568164F174EA7
:10A5F00029432160164D17491760D6601561116017
:10A60000417A154A5C180A3194F8244053F82150D5
:10A6100002EBC40149680D60017A5C1803EB81010B
:10A62000247ECD6902EBC40149680D60817A581817
:10A6300003EB810390F83000596B02EBC002F0BCD1
:10A6400053681960704700BF01401F0001100038B7
:10A650000110007800001F80D8340100704700BF4F
:10A66000F0B50C1EBDF8146034DBB0F90670191992
:10A67000B942C4BF3B1B1BB2002BA6461CDD002AFF
:10A680001146B8BFD11D02F00705CC10826A012027
:10A6900007FB04E1A840012E0A44C0B21ED00CD32F
:10A6A000022E09D1013B12FA83F3013A12F8011F7D
:10A6B00041409A421170F9D1F0BDC043013B12FAFA
:10A6C00083F3C0B2013A12F8011F014093421170A6
:10A6D000F9D1F0BD23441BB20024C6E7013B12FAB6
:10A6E00083F3013A12F8011F01439A421170F9D124
:10A6F000F0BD00BFF8B50D1E0EDB14461F46064622
:10A7000001F03AFBA84207DD002C05DB304601F0E2
:10A7100037FBA04201DCF8BDF8BD304601F02AFB52
:10A72000022853D003284BD0012806D16540F38876
:10A730006C406540013B5D1B2DB2012F03D02AD335
:10A74000022F14D0F8BD002C2246B6F90630B06AAC
:10A75000B8BFE21D42F3CF0202FB035504F0070429
:10A76000435D012101FA04F41C434455F8BD002C5B
:10A770002246B6F90630B06AB8BFE21D42F3CF02F6
:10A7800002FB035504F00704435D012101FA04F4C0
:10A790005C404455F8BD002C2246B6F90630B06A3C
:10A7A000B8BFE21D42F3CF0202FB035504F00704D9
:10A7B000435D012101FA04F423EA04044455F8BD81
:10A7C0003389013B591B25460CB2B6E7F188328923
:10A7D0000139013A4D1B141B2DB224B2ADE700BF65
:10A7E0002DE9F041079E9DF91880089D04461F46FB
:10A7F00000F0C0FF0D4B0E480E4984F83380FF2255
:10A80000002F08BF1F4684F82F20002384F8302033
:10A8100084F8312084F832202060A665E5656762FF
:10A8200061652362A3622046BDE8F0813C90FF1F72
:10A83000302A01000110013810B50446806A034B2C
:10A84000236008B105F078FB204610BD302A0100D6
:10A85000F8B5436ADBB190F82C200125AA4083F8B3
:10A860003B2083F85E5083F85D500446406A0368DD
:10A870000E461B6800219847606A036831461B68D2
:10A8800098472946606ABDE8F840FFF7E5BBC26B10
:10A89000C56C1368046A23EA050313604CB122688F
:10A8A0004FF00043D3625163D36A002BFCDA936B01
:10A8B000F8BD836B466B0825802410E03768426C36
:10A8C0003A4332601F68826C3A431A601A68876C98
:10A8D000013D22EA07024FEA54041A6007D02142E0
:10A8E000ECD13268476C22EA07023260EAE7F8BD31
:10A8F00070B50446406A0D4600282BD0A16DFFF7C5
:10A9000049FA002D20460CBFA621A721FFF7A0FF82
:10A91000606A20B1E16DBDE87040FFF73BBA216C81
:10A92000226D0868236A02430A6093B1DA7A82B121
:10A93000D00703D5224A99691160DA7A910703D5C5
:10A94000204AD9691160DA7A520702D51E4A1B6A79
:10A95000136070BD236A002B2BD0D97A626DE1B1F0
:10A9600072B6D97ACE0706D51848D968066831403C
:10A9700099610160D97A880706D515481969066872
:10A980003140D9610160D97A4E0705D5114859691E
:10A99000066831401962016062B61B68D96891424D
:10A9A00007D00D4818600D49DA6042F08040186108
:10A9B0001960226C216D136823EA01031360A0E77C
:10A9C00000E100E004E100E008E100E080E100E0F7
:10A9D00084E100E088E100E001403F0000003F80AA
:10A9E000436A2DE9F04105460E469046002B3ED0C5
:10A9F00090F82C100124A14083F83B1083F85E40AE
:10AA000083F85D40406A036800211B6808F1FF3746
:10AA10009847FFB2B8F1000F23D03744A046013E5B
:10AA2000686A16F8011F03681B6898470134B7422B
:10AA3000E4B216D0202CF3D10121686AFFF70CFB99
:10AA400095F82C206B6A520083F83B2083F85E80D7
:10AA500083F85D80686A036800211B6898470124B9
:10AA6000DEE7686A0121BDE8F041FFF7F5BAC26B85
:10AA7000C16C136823EA010306EB080413604FF06E
:10AA80000048A6420ED02B6A16F801EB63B11A6893
:10AA9000C2F82C80C2F834E0D36A002BFCDAA6425C
:10AAA000936BF0D1BDE8F081AB6BD5F834C00820D2
:10AAB0008021DCF800206F6C1EEA010F14BF3A43BE
:10AAC000BA43CCF800201A68AF6C3A431A601A688F
:10AAD000AF6C013822EA07024FEA51011A60E8D14F
:10AAE000CFE700BF70B50446406A0D46002828D065
:10AAF000A16DFFF74FF920462946FFF7A9FE606ACE
:10AB000020B1E16DBDE87040FFF744B9216C226DC2
:10AB10000868236A02430A6093B1DA7A82B1D007E7
:10AB200003D5234A99691160DA7A910703D5214A3E
:10AB3000D9691160DA7A520702D51F4A1B6A13607D
:10AB400070BD236A002B2BD0D97A626DE1B172B649
:10AB5000D97ACE0706D51948D96806683140996177
:10AB60000160D97A880706D5154819690668314009
:10AB7000D9610160D97A4E0705D51248596906682E
:10AB800031401962016062B61B68D968914207D0F2
:10AB90000D4818600D49DA6042F080401861196074
:10ABA000226C216D136823EA01031360A3E700BF41
:10ABB00000E100E004E100E008E100E080E100E005
:10ABC00084E100E088E100E001403F0000003F80B8
:10ABD0002DE9F041044686B0806A9DF830801E461B
:10ABE0000F461546B4F90830002800F04281DA1DFE
:10ABF00048BF03F10E02B4F90630D21003FB02F293
:10AC0000002105F0BDFCB4F90820202A00F3928051
:10AC1000B4F90610A34B0120203A733902EBD2722B
:10AC200001EBD1714FF0200E029073208DE80140AE
:10AC300042F34F0241F34F01204600F051FE606A9B
:10AC400084F82D70002800F04D81002D40F08A809E
:10AC5000B4F90830202B14BF3D253C2584F82C5036
:10AC6000B8F1000F40F0858006B394F93300002856
:10AC700018DBC0B2012102F0E7F8012194F833009B
:10AC800002F0CEF8012002F007F9002194F8330019
:10AC900002F0C6F80A2002F0FFF8012194F8330010
:10ACA00002F0BEF8606A002800F08280A16DFFF714
:10ACB00071F804227C492046FFF792FE217A01397F
:10ACC000C9B22046FFF7C4FD784904222046FFF7A9
:10ACD00087FE94F92D30012B14BF1421102120463A
:10ACE000FFF7B6FD042272492046FFF779FEB4F95A
:10ACF0000630802B00F09280602B00F0A680D921D6
:10AD00002046FFF7A5FD94F92D30012B14BFF1214A
:10AD100022212046FFF79CFD204606226549FFF7C9
:10AD20005FFE606A50B3E16DFFF734F8012006B0B2
:10AD3000BDE8F081B4F906105F4B0120403A52396A
:10AD40004FF0400E029002EBD272522001EBD17113
:10AD50008DE8014042F34F0241F34F01204600F0DD
:10AD6000BFFD6CE76DB284F82C50B8F1000F3FF4D2
:10AD70007BAFFEF7C5FF002E94D076E7216C226DE5
:10AD80000868236A02430A6073B1DA7A62B1D007B5
:10AD900003D54A4A99691160DA7A91077CD452073F
:10ADA00002D5474A1B6A1360012006B0BDE8F08156
:10ADB000236A002B2BD0D97A626DE1B172B6D97AB1
:10ADC000CF0706D53F48D9680568294099610160D9
:10ADD000D97A8E0706D53C48196905682940D9619A
:10ADE0000160D97A4D0705D5384859690568294069
:10ADF0001962016062B61B68D968914207D0344875
:10AE000018603449DA6042F0804018611960226CA1
:10AE1000216D136823EA010313604AE7B4F908308F
:10AE2000202B00F08680402B7FF469AF2A49204612
:10AE30000322FFF7D5FD94F92D30012B14BFCF214C
:10AE40009F212046FFF704FD59E7B4F90830102B85
:10AE50007FF455AF214920460322FFF7C1FD94F945
:10AE60002D30012B14BFAF2110212046FFF7F0FC3D
:10AE700045E7DA1D48BF03F10E02B4F90630D210DF
:10AE800003FB02F21046059205F04EF8A06200287E
:10AE90003FF44DAF059AB3E6114AD9691160DA7AE9
:10AEA0007DE700BF882A0100682C01006C2C01009E
:10AEB000702C0100742C01007C2C010000E100E0EA
:10AEC00008E100E080E100E084E100E088E100E0EA
:10AED00001403F0000003F80842A01003C2F010018
:10AEE00004E100E0012194F83100244F01F0ACFFAF
:10AEF00094F83200012101F0A7FF94F9312094F970
:10AF0000323057F83220E26357F83330206A236436
:10AF10000125E56425651A682A431A6078B1B8F1FD
:10AF2000000F3FF428AFFFF75BFB002E3FF4BAAEF3
:10AF30009BE6042212492046FFF752FDDFE6294630
:10AF400094F82F0001F080FF294694F8300001F0BA
:10AF50007BFF94F92F2094F9303057F83220626348
:10AF600057F833306564A5641A68A36322F00102C0
:10AF70001A60002E3FF496AE77E600BFD834010089
:10AF8000802A0100B0F90820D31D48BF02F10E034A
:10AF9000B0F90620806ADB1002FB03F2002105F005
:10AFA000EFBA00BFF0B50029BDF814502EDBB0F9A0
:10AFB0000660B1422ADA002A59DBB0F9087014465B
:10AFC0001C44BC42C4BFBB1A1BB2002B1EDDD2B254
:10AFD000D408D0F828E016FB041112F00702DBB207
:10AFE0000EEB010421D0C2F10807FAB2374F9342A9
:10AFF000BF5C0CD2C3EB020CFF2646FA0CF6012D07
:10B0000007EA06073FD005D3022D36D0F0BD012D4B
:10B0100039D030D21EF8016026EA07070EF8017019
:10B020009342F3D3B0F906100C449A1AD2B2072A0D
:10B0300010D9022D36D0002D14BFFF26002613464E
:10B040002670083BB0F90610DBB2072B0C44F7D88A
:10B0500002F00702002AD9D01D4B012D9B5C1DD0A8
:10B0600017D3022DD2D1227853402370F0BD134460
:10B070001BB20022A1E7022D25D11EF80160774006
:10B080000EF80170CCE71EF8016037430EF801702E
:10B09000C6E7227822EA03032370F0BD2278134327
:10B0A0002370F0BD11462378DB4323700839B0F9D3
:10B0B0000630C9B207291C44F5D812F00702A5D002
:10B0C000034B9B5CCFE73444AFE700BF202A01006D
:10B0D000102A010070B4C47DBDF80C50022C18D0A9
:10B0E000032C1FD0012C0BD0002A03DBB0F9084041
:10B0F000944201DC70BC7047039570BCFFF7B0BA96
:10B10000C4880395013CA41A0A4621B270BCFFF71B
:10B1100049BF0689C488013E641AB21AE41A12B201
:10B1200021B2E1E704890395E41A641A114622B2B8
:10B1300070BCFFF737BF00BF70B4C57DBDF80C60B1
:10B14000022D1AD0032D12D0012D03D0039670BC0E
:10B15000FFF728BFC488E41AA41A0A4621B2002ABD
:10B1600003DBB0F90840944213DC70BC70470489DB
:10B17000013C641A114622B2F1E7C488058903969E
:10B18000013CAD1AED1A621A11B22AB270BCFFF777
:10B1900009BF039670BCFFF763BA00BF2DE9F843FF
:10B1A0000446406A002863D0A16DFEF7F3FD052236
:10B1B00074492046FFF714FCA1790139C9B2204631
:10B1C000FFF746FBB4F90820E588A66AD31D48BFFF
:10B1D00002F10E03DB10626A15FB03F51FFA85F816
:10B1E000002A7BD094F82C300125AB4082F83B300C
:10B1F00082F85E5082F85D50606A036840211B68E7
:10B2000008F1FF379847BFB2B8F1000F23D0374499
:10B21000A846013E606A16F8011F03681B6898473C
:10B220000135B742EDB216D0202DF3D10121606A6D
:10B23000FEF712FF94F82C20636A520083F83B203B
:10B2400083F85E8083F85D80606A036840211B6834
:10B2500098470125DEE70121606AFEF7FDFE606A7E
:10B26000002800F08D80E16DBDE8F843FEF792BD47
:10B27000236A002B2BD0D97A626DE1B172B6D97AEC
:10B28000CE0706D54048D968056829409961016014
:10B29000D97A8D0706D53D48196905682940D961D5
:10B2A0000160D97A480705D53948596905682940A8
:10B2B0001962016062B61B68D968914207D03548AF
:10B2C00018603549DA6042F0804018611960226CDC
:10B2D000216D136823EA0103136068E7E26BE36CF6
:10B2E0001168276A0B4306EB080913604FF0004E04
:10B2F0004E450DD016F801CB2FB33A68C2F82CE0BA
:10B30000C2F834C0D36A002BFCDA4E45936BF1D1FE
:10B31000226C236D11680B43136097B1FB7A83B1E4
:10B32000D90703D51D4BBA691A60FB7A9A0703D572
:10B330001B4BFA691A60FB7A5B0702D5194B3A6A14
:10B340001A60BDE8F883A36BD4F83480082080210C
:10B35000D8F80020656C1CEA010F14BF2A43AA43E9
:10B36000C8F800201A68A56C2A431A601A68A56CF0
:10B37000013822EA05024FEA51011A60E8D1B7E725
:10B38000276AC5E7182A010080E100E084E100E0B7
:10B3900088E100E001403F0000003F8000E100E064
:10B3A00004E100E008E100E02DE9F04F85B09946A6
:10B3B000BDF93870BDF83CA0BB1AC1EB090B002BDE
:10B3C000B8BF5B42BBF1000FB8BFCBF1000B5B45D0
:10B3D0000D4616460093804648DC4D453A463346B6
:10B3E0004CDC194613460A46C5EB09019B1A89B283
:10B3F000002B0CB2B8BF5B4204EBD474BE42ACBFAE
:10B400004FF0FF3201224D45039102924FEA64044E
:10B4100029DC9BB201930DE0D8F80070BF69B847F2
:10B42000019BE41AA3B21CB20135002C2DB211DB32
:10B43000A94518DB009B5B452A46534631464046EA
:10B44000EADCD8F800205346976929463246404640
:10B45000B847E5E7029A1644039AA94502EB0304AC
:10B4600036B224B2E6DA05B0BDE8F08F4A462B4684
:10B47000B94635464D4517461E46B2DD304629468B
:10B480003E464D4607468946AEE700BF10B4046805
:10B490002469A44610BC604730B40468BDF8085065
:10B4A0000295A46BA44630BC604700BF30B404686A
:10B4B000BDF808500295E46BA44630BC604700BF5D
:10B4C00070B40468BDF90C60BDF810500396049583
:10B4D000246CA44670BC6047704700BF10B582B0B2
:10B4E000B0F90C2001910168009200220C6CB0F9B7
:10B4F0000A301146A04702B010BD00BF704700BF20
:10B5000001F003010129C17506D0032904D0C288C6
:10B5100003894281838170470289C3884281838184
:10B52000704700BF2DE9F0410568134E6F6986B082
:10B53000B7420446BDF8308010D1013B13441BB222
:10B540000093CDF804800B46AD6A2046A8472368D7
:10B55000DB6AB3420AD106B0BDE8F08105930492DC
:10B560000391B84703A925680EC9E6E7204606B04F
:10B57000BDE8F041184700BFD9B400002DE9F04103
:10B580000568124E6F6986B0B7420446BDF8308038
:10B590000FD1013BCDF804800B4400921BB2AD6A81
:10B5A0002046A8472368DB6AB3420AD106B0BDE84B
:10B5B000F081059304920391B84703A925680EC949
:10B5C000E7E7204606B0BDE8F0411847D9B40000CF
:10B5D0002DE9F04F0568DFF858B06F6985B05F4519
:10B5E0000646BDF93890BDF83CA00C46904615D1F2
:10B5F0001F19BC420CDACDF800A0214601342D6A97
:10B600004B464246304624B2A847BC423568F2DB7E
:10B61000EB6A5B4507D105B0BDE8F08F0393B847EF
:10B620003568039BE4E7304605B0BDE8F04F1847A6
:10B63000D9B400002DE9F04387B099420546BDF921
:10B640003840BDF83C6025D0A24212D00768DFF830
:10B650008080D7F81490C14532D18DE8500028463B
:10B66000BC6AA0472B68DB6A434524D107B0BDE81C
:10B67000F083994202DD08461946034628680E9673
:10B68000C46B01335B1A1BB22846A44607B0BDE861
:10B69000F0436047A24202DD134622461C4628685A
:10B6A0000E96631C846B9B1A1BB22846A44607B0F7
:10B6B000BDE8F0436047284607B0BDE8F0431847AF
:10B6C000059304920391C84703A92F680EC9C4E7E4
:10B6D000D9B400002DE9F04FD0F800E0DFF89090E9
:10B6E000DEF814B083B0CB450446BDF93080BDF818
:10B6F00034A00D4617461E4631D1CDF800A0DEF825
:10B7000024B0294633463A462046D8472368CDF828
:10B7100000A008F1FF323A44D3F824B0294612B20F
:10B7200033462046D8472368CDF800A02946D3F8F1
:10B7300020B03A4643462046D8472068CDF800A0BE
:10B74000711E29444346056A09B23A462046A84775
:10B750002368DB6A4B4506D103B0BDE8F08FD847BC
:10B76000D4F800E0C9E7204603B0BDE8F04F184721
:10B77000D9B40000F0B4002401264FF6FF75094F3C
:10B7800007600471C475C48104824476C4618675FF
:10B79000067685824582C180028141818281F0BC2A
:10B7A000704700BF482F01002DE9F04F85B00668B3
:10B7B000BDF84450BDF93880CDF8008004460195AD
:10B7C000D6F848B00392BDF93C60BDF94070894697
:10B7D0009A46D84723680195009742465146D3F8C8
:10B7E000488020463346C0472068039B0E930F9540
:10B7F000856C4B463A4631462046AC4605B0BDE81E
:10B80000F04F60472DE9F04F87B01746BDF9404033
:10B8100000912546E91D059344BF2B4603F10E0117
:10B820000268BDF8486053690294C91003912B491E
:10B83000BDF9444001968B42824645D1002C3CDD47
:10B84000029B3C445E1EB6B24FF0000923B2049343
:10B8500001364D46029B002B28DD059B002403EB9F
:10B86000090806E0EDB22B0604F1010411D4A6424A
:10B870001CD0A1B211F0070F23B24FEA4505F1D158
:10B88000002BB8BF0733DB10013418F803502B0628
:10B89000EDD5009BD2F818B019443A4609B2019B85
:10B8A0005046D847A642DAF80020E2D1039B013780
:10B8B0009944049B3FB2BB42CCD1D36A074A93421E
:10B8C00006D107B0BDE8F08F9847DAF80020B5E759
:10B8D000504607B0BDE8F04F184700BFD9B400008C
:10B8E00070B4BDF90C60BDF91050BDF8144003965A
:10B8F0000495059470BCFFF785BF00BF2DE9F04F9C
:10B9000093B090460591C1691090BDF87000079002
:10B91000BDF874909DF878A00493002900F0CD80C4
:10B920000A7A0AC9894604998A1AD2B203EBC20379
:10B93000BAF1010FDA780B9293F905201E8893F87B
:10B9400002B00F9293F9064079D913B2099323B24A
:10B950000C93109B1A68A94B1193194653698B429B
:10B9600040F0A6800B9B002B55D01FFA88F30021D6
:10B970000D93C8462344DDF8409006910E930F4680
:10B980000C46BBF1000F3FD0BDF818100C9B03977D
:10B990001FFA8AF0CB1813FB00F304900E980144B1
:10B9A0000D98034409B21BB20A910893002505E0E3
:10B9B0000135EBB264009B45E4B222D9039B2B44D2
:10B9C000590703D1731C18F806409EB22306EFD521
:10B9D000099BBDF81000E91811FB00F10598BAF1B8
:10B9E000010F0FFA8AF301441CD0079801900093CD
:10B9F000D26909B217464846089AB847D9F80020D4
:10BA0000D6E7039F5F44FFB2069B0B990133069371
:10BA1000DBB29942B5D8D36A119A934243D113B09D
:10BA2000BDE8F08F0F9B191893690A9A29441F46A5
:10BA300009B2079B4846B847D9F80020B8E7002369
:10BA40000C93099385E70A9A0D9B0132013B52B290
:10BA500013F0FF030A920D936FD1DDF81890079B46
:10BA6000DDF83C80DDF820A04B4517D0BAF1010F7E
:10BA700000F0C8800B9A109DCDF804900BEB8B0161
:10BA80004FEACB030A4400931146DEF81C405346AC
:10BA9000424609B22846A047D5F800E0DEF82C302F
:10BAA000119A9342BBD0109813B0BDE8F04F1847DD
:10BAB000109D284698472A6854E7109A0598B2F9CD
:10BAC0000A308342ABDDB2F90C304345A7DD0623D3
:10BAD00013FB0A03002BA2DD08EBCA03002B9EDD3B
:10BAE000537E2BB9049BAF2B02D90133DBB20493F5
:10BAF000109BD3F800E0414B11931A46DEF8143046
:10BB0000934240F08E801FFA88F30E9308339BB265
:10BB1000BDF81420059305230D9300230A93CDF857
:10BB20003C800FFA8AF3DDF84080CDF818900B9234
:10BB30001FFA8AFBCDF820A099460A9ABDF810009A
:10BB40000B9C0E9D0523194611FB00232C48114622
:10BB5000C75C039702FB0B4214FA81F312B21BB2CB
:10BB600009920C932C462E461CE0089B0999012B48
:10BB70002AB24B4640462DD0079F0197CDF8009042
:10BB8000DEF81CA0D047D8F800E0039B5B08013426
:10BB90000393059BA4B25D445E44A342ADB2B6B22A
:10BBA0003FF451AF039BD807DFD4079B069A93421B
:10BBB000EBD0089B012B16D0069B0193CDF800908B
:10BBC000DEF81CA009994B4632B24046D047D8F85F
:10BBD00000E0DAE7DEF818A0079B0C9922B2D04704
:10BBE000D8F800E0D1E7DEF818A00C9913464046DB
:10BBF00022B2D047D8F800E0C7E700BFD9B40000B0
:10BC0000982F01000B99109DCDF800900531DEF8BA
:10BC1000204009B2424608232846A047D5F800E054
:10BC20003CE7109C20469847D4F800E06BE700BF43
:10BC3000F0B5C36985B004462BB30A2968D00D2935
:10BC40004AD01A7A914247D3587A884244D35D68E1
:10BC50008A1A05EBC205AA78002A50D0E878002895
:10BC60004DD0207E00283AD095F905E0B4F90E00B9
:10BC7000A67DB4F90A70724406FB0202BA4262DC85
:10BC8000B4F9102030E00A2956D00D2924D0027EC4
:10BC9000002A4BD0B0F90E00A57DB4F90A60062247
:10BCA00012FB0502B2423EDD228AE38102EBC502AD
:10BCB00012B218462282A78A668A02950B468DE840
:10BCC000C00001462046FFF719FEA37DE28903EB81
:10BCD000430302EB4303E381012005B0F0BDA67DE1
:10BCE000B4F90E00B4F91020B4F814E0678A029693
:10BCF0000B468DE8804001462046FFF7FFFD29797D
:10BD0000E389A27D012001FB0233E38105B0F0BD90
:10BD10000022C2819A7A817D038A01FB0233038269
:10BD2000012005B0F0BDB4F91020C4E7857DB4F959
:10BD30001020B0F90E00BEE7028A817DC38102EBBC
:10BD4000C1030382C8E70020E0819B7A228A03FBBB
:10BD5000062212B22282C7E7C1810282704700BF69
:10BD6000002908BF01218175704700BF818241828F
:10BD7000704700BFC07D7047B0F90A00704700BF30
:10BD8000B0F90C00704700BF10B4EFF3108272B628
:10BD9000437F33B9017F012907D003290FD0012345
:10BDA000437702B962B610BC7047124C2168A1B14A
:10BDB000114943610B68836108605861EFE70F4CDC
:10BDC000216881B10E4943610B6883610860586145
:10BDD0000C4B4FF080511960E1E7074B41618161E5
:10BDE00020601860DBE7064B4161816120601860CC
:10BDF000EEE700BFB89EFF1FB49EFF1FA89EFF1F67
:10BE0000AC9EFF1F04ED00E070B5EFF3108272B638
:10BE10000C4C206880B10C4E00254369236073B13F
:10BE20009D6102B962B6457783689847EFF3108247
:10BE300072B620680028F0D102B962B670BD3360D6
:10BE4000EFE700BFA89EFF1FAC9EFF1FFFF7DCBF00
:10BE5000184A30B41468002C27D0036821688B423C
:10BE60000ED2CB1A00218460C1602360E0601060B4
:10BE70000223037530BC704711688B42144608D307
:10BE8000A2685B1A0360002AF6D18260C460A060D9
:10BE9000EEE7D268C2608460E060C568CB1A022217
:10BEA000A8602360027530BC70478460C460106075
:10BEB000DEE700BFB09EFF1FF8B5224E34682CB3FA
:10BEC0002368002B3AD1204F1D4604E03468ECB1C2
:10BED0002368002B32D1A36803B1DD602069336091
:10BEE000036825751B68BB4221D1037F4560022B87
:10BEF000C46020D0FFF748FF6368002BE6D02360C2
:10BF00002046FFF7A5FF3468002CE1D1EFF3108342
:10BF100072B60E4A00211068116003B962B628B1EA
:10BF20008468FFF795FF20460028F9D1F8BD224626
:10BF300000219847E0E783689847DDE7013B2360ED
:10BF4000E4E700BFB09EFF1FC9A50000C09EFF1F11
:10BF5000024A136801331360FFF7AEBFCC9EFF1F88
:10BF6000704700BF0368F0B4FBB1002501249D6059
:10BF7000DC601B4C1A601C44241104F144056A1156
:10BF8000032692009E60174F0679174B47F824103E
:10BF900002F1604202F5614205F01F05012000FA3E
:10BFA00005F5E6541560F0BC7047104C236843F467
:10BFB0000003236000BF0E4B0E4DA4F58734A4F59B
:10BFC0009E7401261E60234604609C68002CD0D01D
:10BFD0001033AB420360F8D1002303601846E2E758
:10BFE000008FFCBF1491FF1F44E400E03C8004403C
:10BFF00000700340407103400168A9B10B4BF0B4DD
:10C000000B441B110A4E0B4F0B4D46F8237003F1E6
:10C01000440202F01F0401235211A340002445F8FA
:10C0200022308C600460F0BC704700BF008FFCBF02
:10C030001491FF1F61BF000080E100E0024A034B42
:10C04000012111601B6818470C7103401491FF1FF8
:10C05000024A034B012111605B6818471C710340C1
:10C060001491FF1F024A034B012111609B6818477E
:10C070002C7103401491FF1F024A034B01211160F0
:10C08000DB6818473C7103401491FF1FF8B50E465A
:10C0900071B17AB10746144600253B6816F8011BBA
:10C0A0001B6838469847013C0544F6D12846F8BD40
:10C0B0000846F8BD1046F8BD00B5064A0368128868
:10C0C0005B6883B001A9ADF804200222984703B051
:10C0D0005DF804FB98340100F0B507468BB0002AE8
:10C0E00033D0012A08BF0A2251B3212400E0F4B260
:10C0F000B1FBF2F502FB1511C8B2092900F13001BC
:10C1000098BFC8B20AA988BF3730214488BFC0B2DF
:10C1100001F8240C661E2946002DE8D133B1013CFC
:10C12000E4B20AAB23442D2203F8242C3B6801AA75
:10C1300011195B683846C4F1220298470BB0F0BD74
:10C1400030228DF825202124E8E70368C9B21B6856
:10C1500098470BB0F0BD00BF0029BABF49422D235C
:10C1600000230A22FFF7B8BF374A384913681B0675
:10C17000FCD40B6813F08003F8D172B634490A7806
:10C18000002A5FD0334A3448F0B4344C176806684C
:10C190002568D4680C303E44143200681268304F71
:10C1A00035442C4420440244C2F34E022D4E2E4806
:10C1B0002E4D2F4C42F400423A60376806682D68D5
:10C1C0002C4A24680C303E44006812682A4F3544DB
:10C1D0002C4420440244C2F34E02284E2848294DE4
:10C1E000294C42F400423A60376806682D68274AB5
:10C1F00024680C303E4400681268254F35442C44B6
:10C2000020440244C2F34E02224E2348234D244CC4
:10C2100042F400423A60376806682D68214A246873
:10C220000C303E440068126835442C4420440244DB
:10C23000C2F34E021C4842F4004202600B7062B628
:10C24000F0BC704762B6704724B0034024B00B4086
:10C25000C59EFF1F38B003403CB0034040B00340D0
:10C260002CB0034058B003405CB0034060B00340C2
:10C2700064B003406CB0034030B0034038B00B40B2
:10C280003CB00B4040B00B4044B00B404CB00B40B6
:10C290002CB00B4058B00B405CB00B4060B00B4072
:10C2A00064B00B406CB00B4030B00B4030B4294848
:10C2B000294A2A4B2A4D6024E121047011701B7811
:10C2C000284C082B30D00A2B2748284937D00C2B74
:10C2D0000CBF35223D2212232A60236002600B60CE
:10C2E000234B24491B78244ABBB101230B60136004
:10C2F000224B23491B78234A012B26D9042B0FD923
:10C30000082B1ED9102B94BF862387230B60136044
:10C310001D4B01221A7030BC70470B601360E7E7B9
:10C3200084230B601360F3E700F58E200F4908307B
:10C33000012213232A60236002600B60D0E73922B8
:10C34000F7E785230B601360E2E780230B6013603F
:10C35000DEE700BF00400740014007402491FF1F77
:10C3600008B003400CB0034008B00B400CB00B40C9
:10C37000C89EFF1F20B0034020B00B402591FF1F37
:10C3800024B0034024B00B40C59EFF1F0C2830B4DE
:10C3900017D91023984228BF18461C46104A114D41
:10C3A0001178181A8C42287018D00F4913700B7826
:10C3B00023B10E490E4A00230B60136030BCFFF717
:10C3C00075BF0A2802D90C231C46E7E7082802D9C2
:10C3D0000A231C46E2E708231C46DFE730BC70470F
:10C3E0002491FF1FC49EFF1FC59EFF1F24B0034062
:10C3F00024B00B4028282FD8334B2DE9F0411E5C88
:10C40000FF2E2BD0314B1B78002B2AD132062CD497
:10C4100072B62F4D2F4C2F46012326602B7062B62B
:10C4200072B623681B060CD43B781BB9F4E72B7853
:10C43000002BF1D062B602F09BF972B623681806A1
:10C44000F5D5254B1B6800222A7062B6234A107866
:10C4500043FA00F0BDE8F081002070470020BDE8FD
:10C46000F081FFF781FE3206D2D572B61C4DDFF89F
:10C470007C801C4C06F04007FFB206F03F06D8F85F
:10C480000030DFB123F01003C8F80030012326602C
:10C49000134A2B7062B672B6236819060CD413784F
:10C4A0001BB9ECE72B78002BE9D062B602F060F9FB
:10C4B00072B623681B06F5D50B4BC3E743F0100398
:10C4C000C8F80030E2E700BF9C340100C59EFF1FA2
:10C4D000C79EFF1F00B0034010B00340C49EFF1F63
:10C4E000C69EFF1F00B00B4010B00B400CB00B40BD
:10C4F0000A4A0B49136843F4805313600B7843B91D
:10C50000084BC0221A70084B80F30C0000B2188050
:10C510007047044B80221A70F5E700BF2C8004405E
:10C52000C89EFF1F21C00C4000C00C40F0B51B4B43
:10C530001B4E596818689A68DB6885B06C460FC452
:10C54000337899071DD5174A174C1378174913F0FC
:10C55000700318BF1370164A164B802717700026F9
:10C560003320032226706D4608701A7072B6043CA0
:10C5700045F001052046A84762B6237813F0700302
:10C5800009D10D4B064901E0013B02D00A78D207E0
:10C59000FAD505B0F0BD237005B0F0BDC834010078
:10C5A0000100024000000240040002400B00024073
:10C5B000070002400A000240410D0300B0F5006F81
:10C5C0000AD210B5094B1B78DB07044606D504F1E7
:10C5D000A0500078C0B210BD00207047FFF7A6FF42
:10C5E00004F1A0500078C0B210BD00BF01000240AD
:10C5F000B0F5006F17D238B50F4B1B78DA070D4630
:10C60000044611D504F1A0500378AB420AD00B4A7E
:10C61000137813F0700318BF1370074A057013786E
:10C62000DB07FCD538BD7047FFF780FF04F1A05051
:10C630000378AB42EBD1F5E7010002400000024075
:10C6400008B5F5F7A7F9F5F775FD02F091F8FAE7E7
:10C65000844641EA000313F003036DD1403A41D30D
:10C6600051F8043B40F8043B51F8043B40F8043BCC
:10C6700051F8043B40F8043B51F8043B40F8043BBC
:10C6800051F8043B40F8043B51F8043B40F8043BAC
:10C6900051F8043B40F8043B51F8043B40F8043B9C
:10C6A00051F8043B40F8043B51F8043B40F8043B8C
:10C6B00051F8043B40F8043B51F8043B40F8043B7C
:10C6C00051F8043B40F8043B51F8043B40F8043B6C
:10C6D00051F8043B40F8043B51F8043B40F8043B5C
:10C6E000403ABDD2303211D351F8043B40F8043BFC
:10C6F00051F8043B40F8043B51F8043B40F8043B3C
:10C7000051F8043B40F8043B103AEDD20C3205D30B
:10C7100051F8043B40F8043B043AF9D2043208D003
:10C72000D2071CBF11F8013B00F8013B01D30B8875
:10C7300003806046704700BF082A13D38B078DD053
:10C7400010F003038AD0C3F10403D21ADB071CBF25
:10C7500011F8013B00F8013B80D331F8023B20F88F
:10C76000023B7BE7043AD9D3013A11F8013B00F8C8
:10C77000013BF9D20B7803704B7843708B78837050
:10C780006046704708B5104C08E0236859050DD481
:10C7900023681A050FD42368DB0411D423685803D7
:10C7A000F3D500F08DFE23685905F1D502F044F869
:10C7B00023681A05EFD502F0D5F82368DB04EDD520
:10C7C00000F0F0FCEAE700BF3480044008B5FFF752
:10C7D000D9FF00BF014B10221A807047002005408E
:10C7E000704700BF094908B50B6830B16A46184464
:10C7F000A2F58052904202D20860184608BD03F0AC
:10C8000065FB0C2303604FF0FF3008BD2891FF1F2C
:10C81000FEE700BFEFF3138070B9EFF310836BB93D
:10C82000EFF305825AB94FF48070EFF311832BB107
:10C83000984228BF184670474FF0FF3070470F2AC4
:10C8400001D81846F1E7014BD05CEEE7F0E300E0D9
:10C85000F0B44D1E2E46002400E00134B0FBF2F38C
:10C8600002FB1300092800F130078ABF3730F8B205
:10C87000C0B206F8010F1846002BEED10A1953700A
:10C880004CB1107815F8016F28700133E01A83421B
:10C8900002F80169F5DB0846F0BC7047704700BF3D
:10C8A00010B40F4B53F8302092F880422CB1012382
:10C8B00069B182F8803010BC704703EBC0035B683D
:10C8C0001A6841B922F002021A6010BC704782F85F
:10C8D000003110BC704742F003021A6010BC704770
:10C8E000D83401001C4A02EBC00301295B6811D057
:10C8F00004291BD052F83000002280F8802229B190
:10C90000022920D0032922D01A6070474FF4807288
:10C910001A60704752F830004FF4A27280F880120B
:10C920001A601A6822F020021A60704752F830101C
:10C930004FF4A272012081F880021A601A6842F056
:10C9400020021A60704740F203121A6070474FF4D9
:10C9500081721A60704700BFD8340100212848D87E
:10C96000F8B5042A44D8DFE802F0484B4E034500EE
:10C970004FF410262B4B03EBC0030D465C68216877
:10C9800011F4E06148D0284B284A2949C3F89C217A
:10C9900004F140422748C3F8A411A2F59221264F82
:10C9A000C3F8A0017C292548C3F8A871C3F8AC01DD
:10C9B0002CD9A2F594237C2B2AD9A2F596237C2B83
:10C9C00028D9A2F598237C2B29D9A2F59A227C2A72
:10C9D00027D81B4872B6236823F4702343F0807273
:10C9E000C4F384011643236040F82150266062B6E8
:10C9F000F8BD70474FF43026BCE74FF40026B9E786
:10CA00004FF44026B6E74FF42026B3E70D48E1E7A0
:10CA10000D48DFE70D48DDE7FFF764FFB3E70C489B
:10CA2000D8E7F8BDD83401000082FF1FF188FF1F4E
:10CA30009988FF1FC588FF1F6D88FF1F4188FF1F52
:10CA40000492FF1F2C91FF1F6491FF1FB491FF1FE1
:10CA5000E491FF1F1A4B03EBC00010B4426802F1CF
:10CA60004043A3F592217C2923D9A3F594217C2965
:10CA70000DD9A3F596217C291FD9A3F598217C29EE
:10CA800019D9A3F59A237C2B11D80E4C00E00E4C3B
:10CA900072B613680D4823F08773C2F3840123F440
:10CAA000803343F08073136044F8210062B610BCF9
:10CAB0007047074CECE7074CEAE7074CE8E700BF94
:10CAC000D83401000492FF1F6491FF1F9DC800002D
:10CAD0002C91FF1FE491FF1FB491FF1F30B4054B51
:10CAE000054D064C002210211A602A602060196052
:10CAF00030BC704714D0034004D0034000D0034042
:10CB0000282838B52ED0002904464FDD5F4B1B780E
:10CB1000012505FA03F28A4202D8212837D938BD07
:10CB20000338C2B2012A3AD9202C4AD0192C48D055
:10CB3000574A126802FB011222FA03F31D2800F281
:10CB40009B80DFE800F0928B847D9999766F9999AC
:10CB50009999999999999968615A53994C99999980
:10CB600099999945494B1B780B2B08D90C2B1CBF65
:10CB70000C3B19410846BDE83840FFF7B9BCC3F18A
:10CB80000C0399400846BDE83840FFF7B1BC294680
:10CB9000FFF786FE2946BDE83840FFF7A3BE3D4AB1
:10CBA000126802FB011222FA03F3C7E72128B6D864
:10CBB0000021FFF775FE20460121BDE83840FFF750
:10CBC00091BE354A126802FB011222FA03F3B5E75F
:10CBD0003249334A0B604FF45173136038BD314909
:10CBE000314A0B604FF45173136038BD2F49304AFE
:10CBF0000B6040F24443136038BD2E492E4A0B604F
:10CC000040F24443136038BD2C492D4A0B6040F27A
:10CC10004443136038BD2B492B4A0B6040F2444318
:10CC2000136038BD29492A4A0B6040F2444313601F
:10CC300038BD2849284A0B6040F24443136038BD90
:10CC40002649274A0B6040F24443136038BD25490A
:10CC5000254A0B6040F24443136038BD2349244AFF
:10CC60000B604FF45173136038BD2249224A0B60A8
:10CC70004FF45173136038BD212C3FF650AF7F291C
:10CC8000D4BF00210121204693E700BF0C92FF1F73
:10CC9000088003400890034008800B4010800B4040
:10CCA00048A0044018800B404CA00440188003406A
:10CCB00008B004401080034004B0044040800340AA
:10CCC00018C004403880034014C00440288003404A
:10CCD00010B00440208003400CB00440308003407A
:10CCE00010C00440488003401CC00440189003401A
:10CCF00034900440109003403090044038B1102824
:10CD000028BF1020044AC3B2107813707047024A3B
:10CD100001231078137070470C92FF1F2DE9F84320
:10CD20000E4680463249334D304603F055F847F6FB
:10CD3000122300281ABF1D464FF002094FF00109C7
:10CD4000002425FA04F002F051FE4FF05E51074630
:10CD500002F0A4FE0146304603F052F830B9013427
:10CD6000072CEED1E80902F041FE0746314638466D
:10CD700002F048FF4FF07C5102F086FD03F07AF894
:10CD80004FF6FF729042A8F1030328BF1046012B13
:10CD900029D9B8F1170F17D8174B23FA08F303F066
:10CDA000010383F0010223B9B8F1190F0FD0BDE8D8
:10CDB000F883124B124D13491A6044EAC9042A60E1
:10CDC00008601C60BDE8F883B8F1200FECD10E4B71
:10CDD0000E4D0F49002244EAC9041A602A60086017
:10CDE0001C60BDE8F8830B4B0B4D0C49F2E700BF0C
:10CDF000001BB740006CDC026006F00000800340BE
:10CE0000048003400880034000800B4004800B40F6
:10CE100008800B40009003400490034008900340BA
:10CE2000212801D8FFF73CBD704700BF212806D854
:10CE3000044B53F8303093F80002C0B27047002022
:10CE4000704700BFD8340100212801D8FFF74ABD40
:10CE5000704700BF72B60C490C4B0D4A1B6808683E
:10CE6000126862B6520102D5322B88BF01300949DF
:10CE7000C3F5BB334FF47A72FF33A1FB031302FBFC
:10CE800000F000EB93107047CC9EFF1F18E000E00D
:10CE900004ED00E0ABAAAAAA2DE9F843054672B654
:10CEA000204F214B214A1B683C68126862B6520130
:10CEB00002D5322B88BF013495B3C3F5BB331C4E6A
:10CEC000DFF86490DFF86480FF334FF47A72A6FBDA
:10CED000031302FB04F404EB931472B6D9F80010A8
:10CEE0003A68D8F800E062B6C1F5BB33FF33A6FB61
:10CEF00003031EF0806FC4EB93134FF47A7002D0DB
:10CF0000322988BF013200FB0233B3F57A7F04D3A4
:10CF1000013D05D004F57A74DFE701F029FCDCE778
:10CF2000BDE8F883CC9EFF1F18E000E004ED00E0B0
:10CF3000ABAAAAAAF8B52D4B2D49DFF8D0E0DFF84F
:10CF4000D0C02C4E2C4D2D4C2D4A2E4F4FF40000AE
:10CF500018604FF0807018604FF0007018604FF04C
:10CF6000806018604FF0006018600020086028237F
:10CF70004BF6FF71CCF80010CEF800303360136030
:10CF80002B6023603B60B3629362092245F8242C36
:10CF9000C4F8D80F05F57F65C7F8D41F07F5FF273C
:10CFA00007F5FA67C6F8F83F2B6006F5FF26C4F8C8
:10CFB000D42F05F5FD2504F5FF24386006F2F4763C
:10CFC0001148316005F5FF6504F5FD642B602360B1
:10CFD0000260FFF76BF91920FFF75EFF00F0B6FF64
:10CFE00040F21310BDE8F840FFF756BF08E100E03B
:10CFF0000480034014800340248003402C800340BD
:10D000001C8003403480034000800B400C800340B0
:10D01000088003402DE9F84F214B1B6807460BB1F0
:10D0200001221A70DFF888901E4D99F80040DFF851
:10D0300084801D4E0134272C8ABF4FF0000A5FFA0E
:10D0400084FA5446AB462B78A34216D1FFF7E2FB95
:10D0500040281FDC33791B06F5D59BF800300133DF
:10D06000272B86BF00221346DAB218F80330DBB252
:10D07000F3712A702B78A342E8D00C490A4BFFB217
:10D0800008F804700120AC22087089F800A0DA705A
:10D09000BDE8F88FFF28D6DD01F06AFBD3E700BFBB
:10D0A000449FFF1F419FFF1F00C00640409FFF1F7E
:10D0B000489FFF1FD89EFF1F1C4BDFF894C01A68C3
:10D0C0001B49F0B542F480521A4D1A60DFF884E033
:10D0D000194F1A4E1A4C00238CF800304FF451723D
:10D0E0002B701F2840F213358EF800303B703370E0
:10D0F00025600A6012D819460124124A124D117097
:10D100001248547000212C27402693724FF40034AB
:10D1100091701174D7702E700460F0BDC0F344316B
:10D12000C0F3471400F01F03E7E700BF348004405A
:10D130000CC00440D59EFF1F419FFF1F409FFF1F53
:10D1400008C0044000C0064031E400E004E100E013
:10D15000D49EFF1F489FFF1F034B1B68DB0401D5B4
:10D16000FFF758BF704700BF3480044010B5044C2F
:10D17000237823B101F0FCFA2378002BFAD110BDFB
:10D18000409FFF1F054A064B10781B78C0B2DBB2E8
:10D19000984238BF4030C01A704700BFD49EFF1F6E
:10D1A000D59EFF1F30B42B4B1A7994061FD52A4801
:10D1B000DA790378294901333F2B0978C8BF002366
:10D1C0008B42D2B203D0264CD9B2E2540170254A28
:10D1D000116861B1244A1278D2B2934236BFC2F1CB
:10D1E00040029B1A9B18272BC4BF01230B70194ABE
:10D1F000D378DBB2180611D45A060DD5154B1B791E
:10D200005B0609D5194B1A491B6800220A7003B145
:10D210001A70104B2C22DA7030BC70471179090655
:10D22000EAD5144910480C780178C9B28C420DD067
:10D230004A1C272A84BF00210A460F4D054C98BF7F
:10D24000D1B2AA5CD2B2E2710170D5E76C21D17083
:10D25000D2E700BF00C00640D49EFF1FD59EFF1F2F
:10D26000009FFF1FD09EFF1F419FFF1F449FFF1F76
:10D27000409FFF1F489FFF1FD89EFF1F21282FD8C8
:10D28000184B195CFF292BD0174B184ADFF870C0D8
:10D2900003EBC000F0B54368DFF868E0144F154DAC
:10D2A000154E00241C60DEF80030012043F02003FE
:10D2B0008840CEF8003014604FF4A07338602E60C0
:10D2C000C2F800C0013BFDD113689B05FCD42023AC
:10D2D000013BFDD1094B09B233F8110080B2F0BD1A
:10D2E00000207047E8350100D834010000500440A8
:10D2F0000850044004500440000002030051044060
:10D3000080014A0038800440431E032B14D872B6B3
:10D310000A4951F8230068B170B4094C058834F803
:10D320001320466841F82360521B24F8132062B68C
:10D3300070BC704762B6704700207047A49FFF1F03
:10D34000E8A1FF1F013803280BD872B6074B53F82A
:10D35000203043B100205B680130002BFBD162B666
:10D360007047002070471846F9E700BFF89FFF1F7D
:10D3700030B472B62B4A13781D0706D52A4B196AAA
:10D38000002936D0996A002941D053781C0706D568
:10D39000254B196C00293ED0996C002939D093781F
:10D3A000190705D5204B196E002936D0996E89B121
:10D3B000D3781B0707D51C4BD3F880207AB3D3F85A
:10D3C000882011213AB162B6184B00221A7030BC85
:10D3D00000F04ABE0D21154C154D227843F831500E
:10D3E00003EBC1030830013A5860227062B630BCCA
:10D3F000704704220D4C0F4D217843F8325003EB57
:10D40000C20308304A1E5860227062B6EFE7052159
:10D41000E1E70921DFE70822ECE70C22EAE7102226
:10D42000E8E700BF0C3601000080FF1F21A0FF1FAE
:10D43000C800400088004000431E032B1DD81B4A33
:10D44000400140F0100030B4104472B6184CE25C59
:10D45000032A1BD8DFE802F00212151703220D88F9
:10D46000E25410F0080F14BFC823882343EA054391
:10D4700008310360416062B630BC70470830022258
:10D48000EDE70522EBE708300422E8E7094A52F805
:10D49000230038B1084A52F82300416042F82310B3
:10D4A00062B6E9E742F82310034AF7E70080FF1F5E
:10D4B00030A0FF1FF89FFF1F08A0FF1F00BE70478E
:10D4C0002DE9F04FDFF818B3DFF818A387B044E078
:10D4D000AD4F4FEA930807EBC809013ED9F8042085
:10D4E00003F00803F6B2A2F1080003F0FF04002BDA
:10D4F00040F0018157F838301B0C99B222F8081C13
:10D50000002B00F0EF80A14B22F8064C42F8044CAF
:10D5100053F82620002A00F0CF819D4D55F8263083
:10D5200058609C4C45F8260034F81630194424F80D
:10D53000161000F079FD002800F0C281964A974B42
:10D5400019F0080F00F1080018BF1346C9F80400CD
:10D5500047F8383008238BF800309BF80040E4B2DD
:10D5600065071CD58E4B1B78B3B18E490A7802F043
:10D57000FF0322B1013BDBB20B7003B900BE8A4945
:10D580000A7802F0FF032AB1013BDBB20B70002BDB
:10D5900000F0688100F066FE04238BF8003004F090
:10D5A000080303F0FF02002B00F0C9809AF8003056
:10D5B000DBB21E098CD19A08DFF8CC9159F83210F1
:10D5C00009EBC200C1F38301013940680C2900F264
:10D5D0008580DFE801F07A7A8383838383834683BF
:10D5E000838307000168714D4068714F714E686018
:10D5F000296088B240F281610024674B49F83230DB
:10D600004FF0010E88423C60C9F81040C9F818403C
:10D6100086F800E05C4A00F2E780B0F5D06F80F059
:10D620001B82B0F5817F00F0D98100F269818028EA
:10D6300000F02A82822840F0D781A98801F07F017A
:10D64000042900F2D1815C485C4A890008441470C6
:10D65000547001788C0740F1608382F800E0022169
:10D6600073E1534F3A682AB3554B524E55481988C7
:10D670003478057840298E4645F0020828BF4FF0DF
:10D68000400E002C84F001043470CEEB01010CBF7D
:10D690008824C82409EBC80689B285F0010544EA4C
:10D6A0000E447260198049F83840724405700029B0
:10D6B00065D03A603D4B1A88B2F5A06F0ED10021BB
:10D6C0009A785970404B1A7008E038493F4C0D6801
:10D6D000A54200F09880304949F832103C4A0123B5
:10D6E000137037E72C4A2D4B19F0080F18BF13465B
:10D6F00047F838302EE700F0B7FC364A364952F882
:10D700002630002B00F0E38058688C5D42F826003C
:10D7100003F10802C9F80420032C05D8DFE804F05F
:10D720002C02292602228A551A8819F0080F0CBFEC
:10D730008823C82343EA024347F838300AE7E00762
:10D7400000F19380210600F1D180A20706D5234A7B
:10D75000234913780220DBB213700870E30602D568
:10D760001F4B10221A7007B0BDE8F08F04228A55B3
:10D77000DAE705228A55D7E703228A55D4E7BEF1B6
:10D78000400F18BF002294E70080FF1FA49FFF1FD7
:10D79000509FFF1FE8A1FF1FC80040008800400005
:10D7A0002CA0FF1FB59FFF1FA0A0FF1F18A0FF1FE9
:10D7B0004C9FFF1FB49FFF1FC020074024A0FF1FE6
:10D7C000609FFF1F20A0FF1F982007402109000332
:10D7D00094200740F89FFF1F30A0FF1F88200740BC
:10D7E0008020074090200740B0F5106F00F07C814A
:10D7F00040F2A38040F62112904240F07B82A54A7D
:10D80000012313706AE74C68A3498C427FF463AF2D
:10D810000178A9297FF45FAF417845297FF45BAF98
:10D820008178C2297FF457AFC1786B297FF453AF59
:10D830009A489B4E0178347881F00105002C41F024
:10D84000020105700CBF8820C82084F0010449F84B
:10D85000310009EBC10193483470002505244D6067
:10D86000047038E700F064FF94E68F4B89488B49D9
:10D870001A614FF0020E80F800E08C4F0A708C495C
:10D88000196099608B4E8C4D8C4C9A610D213970CA
:10D89000FF213170DFF84CE229702270884D894AEF
:10D8A0008EF800109F27012406F8047C5D60047048
:10D8B000DA6007B0BDE8F08F43F82600824D30E60D
:10D8C000824A47F8380013780133137042E68B5DC3
:10D8D000032B00F2BA8001A252F823F055D50000C4
:10D8E00055D5000035D900002FD900006F49724B83
:10D8F00080220D2008701A70A2077FF52FAF26E74F
:10D9000040F20232904240F0ED81AA8802F07F029C
:10D91000042A69D86D88002D66D16449CDF804E0E9
:10D92000920011440A7842F002020A70C1E1012318
:10D930008B550FE600238B550CE6B0F5086F53D1DD
:10D940006349644A097811707146ED888D4280F010
:10D95000E88252480478402DAE4644F0020C28BFBD
:10D960004FF0400E02EB0E0309EBCC0102930123B2
:10D970004A604FEA0E48CEEB050101930025C8220C
:10D9800042EA080384F0010249F83C303570027025
:10D99000DFF814C1424BDFF8048149BBBEF1400FF0
:10D9A0007FF42DAF42F0020C09EBCC03029ADFF8B2
:10D9B000F8E05A608DBB0D0445F088059DF80430F1
:10D9C0004EF83C500A4433700470134640297FF4EB
:10D9D00016AF0021404A3B60118010E7AA8802F090
:10D9E0007F02042A40F28B81304A0F23137006E72E
:10D9F0004029D7D942F002020CEBC200029E4660D9
:10DA0000BDB19DF8045035481D703346403988F843
:10DA1000004040334CF83200DCE79DF804303370AE
:10DA20000D04029B047045F0C8050B444EF83C50B1
:10DA3000CCE79DF804501D70029B1D4888F80040FB
:10DA4000403940334CF83200C4E719F0080F0CBFDE
:10DA5000022303238B557DE521494A68002AC3D060
:10DA60006C88B5F804E003E00C314A68002ABBD0AA
:10DA70000B88A342F8D14B887345F5D1240A032CB7
:10DA80000CBF1178098960E7124A022114705470A2
:10DA90005BE700BF942007400100040020A0FF1FA7
:10DAA000B49FFF1FB59FFF1F0080FF1FC0200740CE
:10DAB00088004000882007408020074098200740C9
:10DAC000649FFF1FB89FFF1F509FFF1F21A0FF1FD4
:10DAD0002CA0FF1F24A0FF1F609FFF1FC800400055
:10DAE000103601008C200740B248116AAC780470EF
:10DAF0000C0600F19881D9F82820AF49100600F1F2
:10DB0000DB81D9F83020AC49120600F1D081D9F878
:10DB10003820A949130600F1C581D9F84020A6494B
:10DB2000150600F1BA81D9F84820A349140600F17E
:10DB3000AF81D9F85020A049100600F1A481D9F88E
:10DB400058209D49120600F19981D9F860209A4920
:10DB5000130600F18E81D9F868209749150600F167
:10DB60008381D9F870209449140600F17881D9F89E
:10DB700078209149100600F16D81D9F880208E49F6
:10DB8000120600F16181D9F888208B49130600F153
:10DB90005581D9F890208849150600F14981D9F8B6
:10DBA00098208549140600F1FF808448844A8549FD
:10DBB00001908548854D864C049700230596029573
:10DBC00080460F4616461D460394306828B14468C7
:10DBD00000F04AFA2046002CF9D100233360029B62
:10DBE00038681A46002342F8253028B1446800F00E
:10DBF0003BFA2046002CF9D100223A60019A98F8AD
:10DC000000301146002241F8042B039A0191023B97
:10DC10004FF0000122F81510032B07D8DFE803F0BE
:10DC20005D025D024FF0010388F800300135042DDC
:10DC300006F1040607F1040708F10108C5D1654C97
:10DC4000654D2278654B049F059E002110072970C1
:10DC50001A7000F19280624962780A700021C9F856
:10DC60003010C9F838101107DFF84C816ED4A27853
:10DC70005C49DFF844810A7000211207C9F850108E
:10DC8000C9F858104BD4E27857494B4C0A70130727
:10DC90004FF00001C9F87010C9F8781000F1AE809B
:10DCA00033780193002283F00105C9F89020C9F868
:10DCB00098200021029188468E460A464B480478F7
:10DCC00044F0020C09EBCC030393019B002B039B54
:10DCD0005A600CBF8822C82252E64FF0000388F831
:10DCE0000030A3E7B0F5A06F7FF47EAE01230025DE
:10DCF0000193DEE740F621229042F7D074E66D886A
:10DD0000002D7FF471AE3A49CDF804E09200114441
:10DD10000A7822F002020A70CBE7022115E600F031
:10DD200083F9002800F0EB800830324AC8F864001C
:10DD3000C8F8602000F078F9002800F0DA80083098
:10DD40002D4AC9F86C00C9F868209CE700F06CF90E
:10DD5000002800F0E0800830264AC8F84400C8F8DF
:10DD6000402000F061F9002800F0CF800830224AFE
:10DD7000C9F84C00C9F8482079E700F055F90028A7
:10DD800000F0A58008301B4AC9F82400C9F82020FB
:10DD900000F04AF9002800F094800830164AC9F8CB
:10DDA0002C00C9F8282056E7D1F89C00083800F06C
:10DDB0005BF9FAE62CA0FF1F0080FF1F08A0FF1FE1
:10DDC000A49FFF1FF89FFF1F30A0FF1F509FFF1F42
:10DDD000E8A1FF1F0C36010021A0FF1FC42007404F
:10DDE000C8200740CC200740D020074020A0FF1FBC
:10DDF000C020074088004000C800400000F014F92F
:10DE0000002870D008304F4AC4F88400C4F880203D
:10DE100000F00AF9002860D008304B4AC9F88C009D
:10DE2000C9F888203CE7506A083800F01DF962E61E
:10DE3000D1F89400083800F017F9B0E6D1F88C005A
:10DE4000083800F011F9A4E6D1F88400083800F091
:10DE50000BF998E6C86F083800F006F98DE6486FB0
:10DE6000083800F001F982E6C86E083800F0FCF8C6
:10DE700077E6486E083800F0F7F86CE6C86D0838A9
:10DE800000F0F2F861E6486D083800F0EDF856E66B
:10DE9000C86C083800F0E8F84BE6486C083800F029
:10DEA000E3F840E6C86B083800F0DEF835E6486B6A
:10DEB000083800F0D9F82AE6C86A083800F0D4F823
:10DEC0001FE62A78C9F8280001322A70C3E62A78AA
:10DED000C9F8200001322A705AE72A78C9F8880068
:10DEE00001322A70DCE62A78C4F8800001322A70F8
:10DEF0008EE72A78C9F8680001322A70C3E62A78CA
:10DF0000C8F8600001322A7014E72A78C9F848007E
:10DF100001322A70ABE62A78C8F8400001322A7034
:10DF20001FE740298E4628BF4FF0400E02EB0E033C
:10DF300002930123CEEB01014FEA0E480025019325
:10DF4000BCE600BF88004000C8004000F8B500F003
:10DF50008FFD294B29482A4C2A4F2B4DDFF8BCC096
:10DF6000DFF8BCE0294E00221A605A609A60DA603D
:10DF70001A615A619A61DA611A625A629A62DA62C5
:10DF80001A635A639A63DA631A645A649A64DA64A5
:10DF90001A655A659A65DA651A665A669A66DA6685
:10DFA0001A675A679A67DA67C3F880200168C3F86E
:10DFB000842041F480210160C3F307212170C3F361
:10DFC0000740134938701B0E2B70FF238CF800306C
:10DFD000104D8EF8003010480B700123337084F818
:10DFE000642070264FF40074102207F82C3C2E7029
:10DFF000046081F8F820F8BD0080FF1F34800440E1
:10E000009C200740B0200740B420074094200740E0
:10E010001020074049E400E008E100E080200740CC
:10E0200088200740704700BF72B60D480268B2FAF8
:10E0300082F30F2B10DC4FF00041D94022EA01029D
:10E04000026062B6074803EBC303DB00C21800217D
:10E05000C15010465160704762B60020704700BF43
:10E060001092FF1FBC83FF1F0D4B0E4AC31AA2FB69
:10E0700003231B090F2B0CD80B4A127852B972B626
:10E080000A484FF00041026821FA03F31A43026084
:10E0900062B67047064A1278002AF0D0FFF768B9D6
:10E0A000BC83FF1F398EE33821A0FF1F1092FF1F92
:10E0B0002CA0FF1F38B50E4B0E4C1B68218805465F
:10E0C0008BB1B1F5917F05D20B4A4B1C55549BB2D5
:10E0D000238038BD0022084898470021064A55543D
:10E0E0000123238038BDB1F5917FEDD338BD00BF4A
:10E0F00058A0FF1FF2A1FF1FF8A1FF1F2DE9F84351
:10E10000214E224F3168012380463B70B1B1204D32
:10E110004B8801EB8302013300240F2BC2F80880E7
:10E120002C7004D84B8000233B70BDE8F88340235B
:10E130000B800320FFF780F93460F4E7DFF8549098
:10E1400099F80030002BF0D0114D45F6215408E02D
:10E15000013C12D02B7883B900F00AFB99F800300B
:10E160007BB10320FFF7EEF80528F1D8FFF75CFF3D
:10E17000014630600028EBD0CAE701232B70BDE8D0
:10E18000F883BDE8F88300BF74A0FF1F48A0FF1FFD
:10E1900078A0FF1F2CA0FF1F1201F8B5D5B2A1B3C4
:10E1A000012943D04378044600781B0643EA004027
:10E1B00040F4704045F004068F1E3043FFF79EFF89
:10E1C000022F04F1020314D9053414F8023C14F8A8
:10E1D000032C14F8010C1B0443EA0223334343EAE3
:10E1E0000060033FFFF78AFF022F234604F1030478
:10E1F000EBD8022F23D0012F0DD045F4774040F00B
:10E200000500BDE8F840FFF779BF14482843BDE892
:10E21000F840FFF773BF187845F4770545F0060519
:10E2200045EA0020BDE8F840FFF768BF03780C48D6
:10E2300045EA03452843BDE8F840FFF75FBF1A7879
:10E24000587845F0774545F0070545EA022545EA47
:10E250000040BDE8F840FFF751BF00BF06F0F700EF
:10E2600007F000F738B5084B1C7824B9074D29682A
:10E2700009B14B8803B938BD9B000B800320FFF721
:10E28000DBF82C6038BD00BF48A0FF1F74A0FF1F43
:10E290002DE9F041AD4E33680746002B00F0928027
:10E2A0001D885A88910803EB81010432AA428C68C8
:10E2B00042D25A8004F00F064FEA1428A449A6F16E
:10E2C000080208F00F00C4F30313062A00F1010549
:10E2D0000B701AD9B31E012B5FFA88F04ED9052EA8
:10E2E00048D0042E00F0A481731F022B7FD90F2E7B
:10E2F0000ED1F72842D8F02802D0964B1B883BB1AC
:10E30000FFF7D8FE0020BDE8F08127B1BD4202D062
:10E310000020BDE8F081082EC4F3033300F08780AD
:10E32000092E11D00A2E40F094800A2BF0D18A4B8E
:10E330008A4A1B68A02181E01846FFF795FE042059
:10E34000FEF7E2FF3060B5E7092BE1D1270E00F0C0
:10E350007B81834B814A1B689021C4F3074611706F
:10E36000EDB2FCB2002B00F09D80224631462846DB
:10E37000984797E0F02843D9F72841D0F1380E2884
:10E38000C6D801A353F820F03FE5000023E50000C4
:10E3900011E5000011E3000011E3000003E50000B7
:10E3A00011E30000E3E5000011E30000ADE500002B
:10E3B000C7E50000EBE4000011E30000D3E4000037
:10E3C000B7E40000674B1B78002BA1D00420FEF7B8
:10E3D0009BFF0346306000289AD00588002D7FF40B
:10E3E00060AFFFF741FE35602846BDE8F081FFF7DA
:10E3F00061FEC4F30740FFF75DFE072E02D1200E39
:10E40000FFF758FE534B584A198858481468584D1E
:10E41000524A017000270E0AF0201F802E701070E3
:10E420000CB301225348A0470120BDE8F081082B1E
:10E430007FF46EAF504B494A1B688021C4F30746F6
:10E440001170EDB2240E6BB3284622463146984730
:10E4500028E00B2E11D10B2B7FF45AAF474B3F4ACC
:10E460001B68B021EAE7464B1B68002B00F0FB80DD
:10E47000404898470120BDE8F0810C2E40F0008113
:10E480000C2B7FF445AF3F4B344A1B68C021117001
:10E49000EDB2C4F30746002B00F0C8802846314691
:10E4A000240E98473849314A314B0D7016701C7054
:10E4B0000120BDE8F081354B1B68002B00F0D680B1
:10E4C0009847C4F30746254BEDB2240E83F800802D
:10E4D000E8E72F4B1B68002BF2D12E4B1B68A3B132
:10E4E000FE209847C4F30746EDE72B4B1B68002B33
:10E4F000E6D1284B1B6843B1FC209847C4F307467C
:10E50000E1E7264B1B68002BDAD1C4F30746DAE7B4
:10E51000234B1B68C4F30746002BD4D030469847E2
:10E52000D1E7204B1A68002AEFD0260C630C06F0C6
:10E530007F0003F47E531843F6B29047C3E71A4BAB
:10E540001B68C4F30746002BE8D1BCE780A0FF1F7F
:10E55000F6A1FF1FF2A1FF1F5CA0FF1FF0A1FF1F8C
:10E5600090A0FF1F2CA0FF1F58A0FF1FF4A1FF1FAA
:10E57000F5A1FF1FF8A1FF1F88A0FF1F8CA0FF1FA0
:10E5800070A0FF1F4CA0FF1FF7A1FF1F38A0FF1FA7
:10E590003CA0FF1F40A0FF1F7CA0FF1F6CA0FF1F1F
:10E5A00084A0FF1F54A0FF1F68A0FF1F3F4B1B68E4
:10E5B000002B85D13E4B1B68002BA6D0FA20984734
:10E5C000C4F307467FE73B4B1B68002B7FF478AF13
:10E5D000374B1B68002B98D0FB209847C4F30746A5
:10E5E00071E7354B1B68002B7FF46AAF304B1B681B
:10E5F000002B8AD0F8209847C4F3074663E70E2B18
:10E600007FF486AE2D4A2E4B1268E0211970002A45
:10E6100047D0260C610C06F07F0301F47E511943AC
:10E62000EDB2A1F5005128469047F6B2240E39E725
:10E63000FFF740FDC4F30740FFF73CFD200EFFF756
:10E6400039FD0020BDE8F0811E4B1D4A1B6880216A
:10E650001170EDB2C4F3074683B1314628463A46FD
:10E6600098473C461EE70120BDE8F081104B1B682F
:10E67000002B3FF44AAFFF20984746E71C4611E7BE
:10E680000D2EBCD10D2B7FF443AE0F4B0C4A1B68F3
:10E69000D0211170EDB2C4F30746002B7FF4FEAE1B
:10E6A000C4E7C4F30746EDB2240EFBE664A0FF1FE7
:10E6B00040A0FF1F44A0FF1F34A0FF1F50A0FF1F5A
:10E6C000F0A1FF1F88A0FF1F60A0FF1F38B5164DE7
:10E6D0002868E0B101884488A14213DD03191B7A40
:10E6E00083B104F10803C2180C1B002302E012F8E6
:10E6F000011F21B10133A342F9D1204638BD1C4688
:10E70000204638BDFFF7B0FC0020286038BD074B1D
:10E710001B780BB9002038BD0220FEF7F5FD2860FC
:10E720000028D7D1F6E700BF9CA0FF1F2CA0FF1F39
:10E730000D4B1B78BBB910B50C4C216803F0FF02E0
:10E740004B883F2B07DC07330B4401F1470003F8EC
:10E75000012F8342FBD140230B800120FEF76CFE8A
:10E760000023236010BD704794A0FF1F98A0FF1FD7
:10E7700038B5224C237803B138BD01232370FFF74D
:10E78000A5FF70BB00F048F840BB00F0DBF810BB01
:10E79000FEF7F8FCE0B900232370EFF30583002BAC
:10E7A000EAD1EFF3108172B6154B1868E0B1154C41
:10E7B0002278CAB945691D6001232370C5B1AA61D9
:10E7C00001B962B600254577836898472570D3E77D
:10E7D00000F020F8DFE700F01BF8D9E700F016F8AA
:10E7E000D3E7FFF71FFCCDE70029C5D162B638BDDE
:10E7F000054B1D600029E5D1E3E700BFA1A0FF1F85
:10E80000B89EFF1FBC9EFF1FB49EFF1F704700BF36
:10E81000704700BF704700BF054A064B10781B7851
:10E82000C0B2DBB2984238BF4030C01A704700BF58
:10E83000A8A0FF1FA9A0FF1FF0B4384B1A7912F04F
:10E84000300F2CD072B6997D01F0FF0200293DD027
:10E8500062B6334F334938780D78334E1C46C0B218
:10E86000EDB2431C402BE17928BF0023AB4202F1FB
:10E87000FF32C9B21CBFF154184612F0FF02F0D1AA
:10E880002A4B1B68C2B23A704BB1A84236BFC5F1E1
:10E890004005401B40192728C4BF01221A701F4998
:10E8A000CA78D2B2150616D452060DD51B4B1B7969
:10E8B0005B0609D51E4B1F491B6800220A7003B175
:10E8C0001A70164B3C22DA70F0BC70474022D9799E
:10E8D0005A7462B6E3E70B791C06E5D5164B174E62
:10E8E0001C783378E4B2DBB29C420ED0144D01E0C8
:10E8F000A3420AD00133402B28BF00230879E85CEB
:10E90000C0B2C871087D0728F2D9DBB20349337061
:10E910000B79180644BF7C23CB70C5E700A00640E6
:10E92000A8A0FF1FA9A0FF1FECA0FF1FA4A0FF1F0E
:10E9300030A1FF1F2CA1FF1F34A1FF1F2DA1FF1F1E
:10E94000ACA0FF1F054A064B10781B78C0B2DBB2A3
:10E95000984238BF4030C01A704700BFA8A1FF1FBF
:10E960003DA1FF1FF0B4384B1A7912F0300F2CD0B4
:10E9700072B6997D01F0FF0200293DD062B6334F97
:10E98000334938780D78334E1C46C0B2EDB2431C83
:10E99000402BE17928BF0023AB4202F1FF32C9B21C
:10E9A0001CBFF154184612F0FF02F0D12A4B1B682D
:10E9B000C2B23A704BB1A84236BFC5F14005401B08
:10E9C00040192728C4BF01221A701F49CA78D2B241
:10E9D000150616D452060DD51B4B1B795B0609D5BF
:10E9E0001E4B1F491B6800220A7003B11A70164B98
:10E9F0003C22DA70F0BC70474022D9795A7462B672
:10EA0000E3E70B791C06E5D5164B174E1C783378D7
:10EA1000E4B2DBB29C420ED0144D01E0A3420AD016
:10EA20000133282B28BF00230879E85CC0B2C871E5
:10EA3000087D0728F2D9DBB2034933700B79180639
:10EA400044BF7C23CB70C5E700B00640A8A1FF1FE0
:10EA50003DA1FF1F68A1FF1F38A1FF1FACA1FF1F31
:10EA60003CA1FF1FB0A1FF1FA9A1FF1F40A1FF1FD5
:10EA700070B584B072B6194B194D1A4870224126F0
:10EA80000F2480211A702E701A46047019701378A2
:10EA90001B06FCD5144B186862B6144B144C9842F4
:10EAA00098BF00EB800001A998BF40000A22FDF743
:10EAB000CFFE01A92046002311F8012B01333AB102
:10EAC0000A2B20F8022FF7D11623237004B070BD53
:10EAD0005B00DBB2237004B070BD00BF00000240D9
:10EAE0000700024006000240080002407F9698009E
:10EAF000DC92FF1FFFFFFFFF2DE9F043DFF8EC8002
:10EB00008BB006460F4600F073F898F900300133D9
:10EB100004460D4637D03046394600F0DFF900286C
:10EB200031D02BA3D3E900233046394600F026FE2E
:10EB3000814668BB28A3D3E900233046394600F05C
:10EB4000FFFD00B398F90030254ACDF82090042449
:10EB500000200021022BCDE90467CDE90267009473
:10EB60000192CDE906012CD0684600F0BDF940B312
:10EB7000089B1BB101F0AAF9089B0360DDE90601BF
:10EB80000BB0BDE8F083204629460BB0BDE8F0830A
:10EB9000134A98F90030019203210022CDE904675D
:10EBA000CDE90267009108922BB90E4B4FF06042FD
:10EBB000CDE90623D8E70C490020022BCDE9060158
:10EBC000D2D101F083F922230360D1E7AFF30080B3
:10EBD000EF39FAFE422E864051302DD5104987C0BC
:10EBE0007C360100FFFFEF470000F07FF292FF1F2D
:10EBF0002DE9F04FB04F21F00042BA4283B00C46ED
:10EC00004FEAD17605460DD9AC4FBA4225D9C1F3AA
:10EC10001303034340F0EF800EB10020014603B020
:10EC2000BDE8F08FA64B9A4200F2CC80A54B9A42E9
:10EC300000F2DE808AA3D3E9002300F05DF9002210
:10EC4000A14B00F09BFD002800F0058128462146DD
:10EC500000229D4B00F050F9E1E783A3D3E90023A4
:10EC600000F08CFD002840F0CB802846214680A390
:10EC7000D3E9002300F064FD0028CED1934B284651
:10EC800003EBC60821467CA3D3E9002300F0E6FA93
:10EC9000D8E9002300F030F900F07AFD804600F05A
:10ECA00077FA77A3D3E9002306460F4600F0D6FA99
:10ECB00002460B462846214600F01CF972A3D3E910
:10ECC0000023CDE900013046394600F0C7FA8246FC
:10ECD0008B4652465B46DDE9000100F00BF9054624
:10ECE0000C462A4623462846214600F0B7FA68A378
:10ECF000D3E9002306460F4600F0B0FA66A3D3E935
:10ED0000002300F0F7F832463B4600F0A7FA64A370
:10ED1000D3E9002300F0F0F832463B4600F09EFABB
:10ED200061A3D3E9002300F0E5F832463B4600F04A
:10ED300095FA5FA3D3E9002300F0DEF832463B46A4
:10ED400000F08CFA02460B462846214600F0D2F825
:10ED500006460F462846214632463B46B8F1000F8C
:10ED600056D000F07BFA324604460D463B46002062
:10ED70004FF0804100F0BEF802460B46204629467F
:10ED800000F096FB02460B465046594600F0B2F89A
:10ED9000DDE9002300F0AEF80B4602464A490020A8
:10EDA00000F0A8F86FF47F7398454FDA08F57A7889
:10EDB00001EB085100224FF0B87300F04FFA03B096
:10EDC000BDE8F08F424B9A423FF658AF414BF400FA
:10EDD0002344D3E9002300F08DF83F4BC6F101082E
:10EDE0001C44CDE90001D4E900ABC6EB080870E78C
:10EDF0004FF0000875E702460B4600F07DF80EE77D
:10EE000017A3D3E900231046194600F027FA06E7B6
:10EE100000F024FA0022804689464FF080433046B5
:10EE2000394600F067F802460B464046494600F076
:10EE30003FFB2A46234600F05DF802460B460020C1
:10EE4000214900F057F803B0BDE8F08F01EB0851FD
:10EE500003B0BDE8F08F804643E700BFAFF300800A
:10EE60009C7500883CE4377EEF39FAFE422E8640DE
:10EE700051302DD5104987C0FE822B654715F73FCD
:10EE80000000E0FE422EE63F763C7935EF39EA3D60
:10EE9000D0A4BE726937663EF16BD2C541BDBB3EA0
:10EEA0002CDE25AF6A56113F93BDBE166CC1663F7E
:10EEB0003E5555555555C53F412E8640FFFFEF7FC6
:10EEC000422ED63FFFFF2F3E0000F03F803601006C
:10EED000B1A2F03FA03601009036010041F00041A0
:10EEE00001F58010C00F70470020704781F000418D
:10EEF00002E000BF83F0004330B54FEA41044FEA1F
:10EF0000430594EA050F08BF90EA020F1FBF54EAB9
:10EF1000000C55EA020C7FEA645C7FEA655C00F055
:10EF2000E2804FEA5454D4EB5555B8BF6D420CDD26
:10EF30002C4480EA020281EA030382EA000083EAA9
:10EF4000010180EA020281EA0303362D88BF30BD49
:10EF500011F0004F4FEA01314FF4801C4CEA11319F
:10EF600002D0404261EB410113F0004F4FEA0333FE
:10EF70004CEA133302D0524263EB430394EA050F89
:10EF800000F0A780A4F10104D5F1200E0DDB02FAF8
:10EF90000EFC22FA05F2801841F1000103FA0EF28C
:10EFA000801843FA05F359410EE0A5F120050EF152
:10EFB000200E012A03FA0EFC28BF4CF0020C43FA83
:10EFC00005F3C01851EBE37101F0004507D54FF090
:10EFD000000EDCF1000C7EEB00006EEB0101B1F5E0
:10EFE000801F1BD3B1F5001F0CD349085FEA300026
:10EFF0004FEA3C0C04F101044FEA445212F5800F31
:10F0000080F09A80BCF1004F08BF5FEA500C50F1CD
:10F01000000041EB045141EA050130BD5FEA4C0CB0
:10F02000404141EB010111F4801FA4F10104E9D139
:10F0300091F0000F04BF01460020B1FA81F308BF30
:10F040002033A3F10B03B3F120020CDA0C3208DDFC
:10F0500002F1140CC2F10C0201FA0CF021FA02F1D7
:10F060000CE002F11402D8BFC2F1200C01FA02F147
:10F0700020FA0CFCDCBF41EA0C019040E41AA2BF6C
:10F0800001EB0451294330BD6FEA04041F3C1CDA34
:10F090000C340EDC04F11404C4F1200220FA04F054
:10F0A00001FA02F340EA030021FA04F345EA0301FE
:10F0B00030BDC4F10C04C4F1200220FA02F001FAC0
:10F0C00004F340EA0300294630BD21FA04F0294642
:10F0D00030BD94F0000F83F4801306BF81F48011DB
:10F0E0000134013D4EE77FEA645C18BF7FEA655C4E
:10F0F00029D094EA050F08BF90EA020F05D054EA20
:10F10000000C04BF1946104630BD91EA030F1EBF24
:10F110000021002030BD5FEA545C05D14000494128
:10F1200028BF41F0004130BD14F580043CBF01F51B
:10F13000801130BD01F0004545F0FE4141F4700101
:10F140004FF0000030BD7FEA645C1ABF19461046DC
:10F150007FEA655C1CBF0B46024650EA013406BFDD
:10F1600052EA033591EA030F41F4002130BD00BF9C
:10F1700090F0000F04BF0021704730B54FF4806459
:10F1800004F132044FF000054FF0000150E700BFDA
:10F1900090F0000F04BF0021704730B54FF4806439
:10F1A00004F1320410F0004548BF40424FF0000126
:10F1B0003EE700BF42004FEAE2014FEA31014FEA69
:10F1C00002701FBF12F07F4393F07F4F81F06051B8
:10F1D000704792F0000F14BF93F07F4F704730B527
:10F1E0004FF4607401F0004521F0004120E700BFBA
:10F1F00050EA010208BF704730B54FF000050AE041
:10F2000050EA010208BF704730B511F0004502D541
:10F21000404261EB41014FF4806404F132045FEA43
:10F22000915C3FF4DCAE4FF003025FEADC0C18BFE8
:10F2300003325FEADC0C18BF033202EBDC02C2F1DE
:10F24000200300FA03FC20FA02F001FA03FE40EA70
:10F250000E0021FA02F11444C1E600BF70B54FF070
:10F26000FF0C4CF4E06C1CEA11541DBF1CEA135552
:10F2700094EA0C0F95EA0C0F00F0DEF82C4481EABA
:10F28000030621EA4C5123EA4C5350EA013518BFDA
:10F2900052EA033541F4801143F4801338D0A0FBC7
:10F2A00002CE4FF00005E1FB02E506F00042E0FB74
:10F2B00003E54FF00006E1FB03569CF0000F18BF7A
:10F2C0004EF0010EA4F1FF04B6F5007F64F5407422
:10F2D00004D25FEA4E0E6D4146EB060642EAC621B5
:10F2E00041EA55514FEAC52040EA5E504FEACE2E22
:10F2F000B4F1FD0C88BFBCF5E06F1ED8BEF1004F25
:10F3000008BF5FEA500E50F1000041EB045170BDA0
:10F3100006F0004646EA010140EA020081EA0301E4
:10F32000B4EB5C04C2BFD4EB0C0541EA045170BDE0
:10F3300041F480114FF0000E013C00F3AB8014F15A
:10F34000360FDEBF002001F0004170BDC4F10004A3
:10F35000203C35DA0C341BDC04F11404C4F1200524
:10F3600000FA05F320FA04F001FA05F240EA02007F
:10F3700001F0004221F0004110EBD37021FA04F6B5
:10F3800042EB06015EEA430E08BF20EAD37070BD6F
:10F39000C4F10C04C4F1200500FA04F320FA05F0CE
:10F3A00001FA04F240EA020001F0004110EBD370D0
:10F3B00041F100015EEA430E08BF20EAD37070BD40
:10F3C000C4F1200500FA05F24EEA020E20FA04F319
:10F3D00001FA05F243EA020321FA04F001F00041C8
:10F3E00021FA04F220EA020000EBD3705EEA430E39
:10F3F00008BF20EAD37070BD94F0000F0FD101F068
:10F400000046400041EB010111F4801F08BF013CA0
:10F41000F7D041EA060195F0000F18BF704703F0DE
:10F420000046520043EB030313F4801F08BF013D65
:10F43000F7D043EA0603704794EA0C0F0CEA135521
:10F4400018BF95EA0C0F0CD050EA410618BF52EADB
:10F450004306D1D181EA030101F000414FF00000E1
:10F4600070BD50EA410606BF1046194652EA4306EF
:10F4700019D094EA0C0F02D150EA013613D195EA63
:10F480000C0F05D152EA03361CBF104619460AD1AB
:10F4900081EA030101F0004141F0FE4141F47001B5
:10F4A0004FF0000070BD41F0FE4141F4780170BDA5
:10F4B00070B54FF0FF0C4CF4E06C1CEA11541DBF0A
:10F4C0001CEA135594EA0C0F95EA0C0F00F0A7F80C
:10F4D000A4EB050481EA030E52EA03354FEA013139
:10F4E00000F088804FEA03334FF0805545EA13134C
:10F4F00043EA12634FEA022245EA111545EA106514
:10F500004FEA00260EF000419D4208BF964244F1AA
:10F51000FD0404F5407402D25B084FEA3202B61AC9
:10F5200065EB03055B084FEA32024FF480104FF49D
:10F53000002CB6EB020E75EB030E22BFB61A754611
:10F5400040EA0C005B084FEA3202B6EB020E75EBA4
:10F55000030E22BFB61A754640EA5C005B084FEA0C
:10F560003202B6EB020E75EB030E22BFB61A7546D9
:10F5700040EA9C005B084FEA3202B6EB020E75EBE4
:10F58000030E22BFB61A754640EADC0055EA060EA5
:10F5900018D04FEA051545EA16754FEA06164FEAE8
:10F5A000C30343EA52734FEAC2025FEA1C1CC0D194
:10F5B00011F4801F0BD141EA00014FF000004FF021
:10F5C000004CB6E711F4801F04BF01430020B4F1E2
:10F5D000FD0C88BFBCF5E06F3FF6AFAEB5EB030C9A
:10F5E00004BFB6EB020C5FEA500C50F1000041EB97
:10F5F000045170BD0EF0004E4EEA113114EB5C0464
:10F60000C2BFD4EB0C0541EA045170BD41F4801136
:10F610004FF0000E013C90E645EA060E8DE60CEA3E
:10F62000135594EA0C0F08BF95EA0C0F3FF43BAF5B
:10F6300094EA0C0F0AD150EA01347FF434AF95EA12
:10F640000C0F7FF425AF104619462CE795EA0C0FF6
:10F6500006D152EA03353FF4FDAE1046194622E7C3
:10F6600050EA410618BF52EA43067FF4C5AE50EA9D
:10F6700041047FF40DAF52EA43057FF4EBAE12E78D
:10F680004FF0FF3C06E000BF4FF0010C02E000BF6E
:10F690004FF0010C4DF804CD4FEA410C7FEA6C5C51
:10F6A0004FEA430C18BF7FEA6C5C1BD001B050EAF4
:10F6B000410C0CBF52EA430C91EA030F02BF90EADF
:10F6C000020F0020704710F1000F91EA030F58BF9E
:10F6D000994208BF90422CBFD8176FEAE37040F000
:10F6E000010070474FEA410C7FEA6C5C02D150EA9E
:10F6F000013C07D14FEA430C7FEA6C5CD6D152EA59
:10F70000033CD3D05DF8040B704700BF844610461D
:10F7100062468C461946634600E000BF01B5FFF71C
:10F72000B7FF002848BF10F1000F01BD4DF808EDEC
:10F73000FFF7F4FF0CBF012000205DF808FB00BFBD
:10F740004DF808EDFFF7EAFF34BF012000205DF817
:10F7500008FB00BF4DF808EDFFF7E0FF94BF012064
:10F7600000205DF808FB00BF4DF808EDFFF7CEFF65
:10F7700094BF012000205DF808FB00BF4DF808EDA4
:10F78000FFF7C4FF34BF012000205DF808FB00BF75
:10F790004FEA410212F5001215D211D56FF47873B9
:10F7A000B3EB625212D94FEAC12343F0004343EA5C
:10F7B000505311F0004F23FA02F018BF4042704737
:10F7C0004FF00000704750EA013005D111F00040C1
:10F7D00008BF6FF0004070474FF00000704700BF57
:10F7E0004FEA4102B2F1E04324BFB3F5001CDCF163
:10F7F000FE5C0DD901F0004C4FEAC0024CEA50709B
:10F80000B2F1004F40EB830008BF20F001007047C9
:10F8100011F0804F21D113F13872BCBF01F00040CC
:10F82000704741F480114FEA5252C2F11802C2F1FE
:10F83000200C10FA0CF320FA02F018BF40F001007F
:10F840004FEAC1234FEAD32303FA0CFC40EA0C0031
:10F8500023FA02F34FEA4303CCE77FEA625307D16E
:10F8600050EA01331EBF4FF0FE4040F440007047A5
:10F8700001F0004040F0FE4040F40000704700BF3F
:10F8800080F0004002E000BF81F0004142001FBF55
:10F890005FEA410392EA030F7FEA226C7FEA236C5E
:10F8A0006AD04FEA1262D2EB1363C1BFD218414053
:10F8B00048404140B8BF5B42192B88BF704710F0E9
:10F8C000004F40F4000020F07F4018BF404211F08C
:10F8D000004F41F4000121F07F4118BF494292EAF4
:10F8E000030F3FD0A2F1010241FA03FC10EB0C0020
:10F8F000C3F1200301FA03F100F0004302D54942AD
:10F9000060EB4000B0F5000F13D3B0F1807F06D359
:10F9100040084FEA310102F10102FE2A51D2B1F151
:10F92000004F40EBC25008BF20F0010040EA030046
:10F930007047490040EB000010F4000FA2F10102F3
:10F94000EDD1B0FA80FCACF1080CB2EB0C0200FA7D
:10F950000CF0AABF00EBC25052421843BCBFD040CB
:10F960001843704792F0000F81F4000106BF80F445
:10F9700000000132013BB5E74FEA41037FEA226C08
:10F9800018BF7FEA236C21D092EA030F04D092F0D3
:10F99000000F08BF0846704790EA010F1CBF002007
:10F9A000704712F07F4F04D1400028BF40F0004064
:10F9B000704712F100723CBF00F50000704700F084
:10F9C000004343F0FE4040F4000070477FEA2262AB
:10F9D00016BF08467FEA23630146420206BF5FEA7C
:10F9E000412390EA010F40F4800070474FF000037C
:10F9F00004E000BF10F0004348BF40425FEA000C43
:10FA000008BF704743F0964301464FF000001CE0EA
:10FA100050EA010208BF70474FF000030AE000BF40
:10FA200050EA010208BF704711F0004302D540427E
:10FA300061EB41015FEA010C02BF844601460020F0
:10FA400043F0B64308BFA3F18053A3F50003BCFA0B
:10FA50008CF2083AA3EBC25310DB01FA02FC6344B8
:10FA600000FA02FCC2F12002BCF1004F20FA02F2BF
:10FA700043EB020008BF20F00100704702F12002B2
:10FA800001FA02FCC2F1200250EA4C0021FA02F213
:10FA900043EB020008BF20EADC7070474FF0FF0C18
:10FAA0001CEAD0521EBF1CEAD15392EA0C0F93EA13
:10FAB0000C0F6FD01A4480EA010C400218BF5FEAB5
:10FAC00041211ED04FF0006343EA501043EA511128
:10FAD000A0FB01310CF00040B1F5000F3EBF490022
:10FAE00041EAD3715B0040EA010062F17F02FD2A26
:10FAF0001DD8B3F1004F40EBC25008BF20F0010009
:10FB0000704790F0000F0CF0004C08BF49024CEA1F
:10FB1000502040EA51207F3AC2BFD2F1FF0340EAB1
:10FB2000C250704740F400004FF00003013A5DDC22
:10FB300012F1190FDCBF00F000407047C2F1000263
:10FB4000410021FA02F1C2F1200200FA02FC5FEA50
:10FB5000310040F1000053EA4C0308BF20EADC709A
:10FB6000704792F0000F00F0004C02BF400010F40C
:10FB7000000F013AF9D040EA0C0093F0000F01F0B9
:10FB8000004C02BF490011F4000F013BF9D041EADB
:10FB90000C018FE70CEAD15392EA0C0F18BF93EADD
:10FBA0000C0F0AD030F0004C18BF31F0004CD8D107
:10FBB00080EA010000F00040704790F0000F17BF8E
:10FBC00090F0004F084691F0000F91F0004F14D0D4
:10FBD00092EA0C0F01D142020FD193EA0C0F03D12C
:10FBE0004B0218BF084608D180EA010000F000402F
:10FBF00040F0FE4040F40000704740F0FE4040F40A
:10FC0000400070474FF0FF0C1CEAD0521EBF1CEAA8
:10FC1000D15392EA0C0F93EA0C0F69D0A2EB0302C6
:10FC200080EA010C49024FEA402037D04FF0805360
:10FC300043EA111143EA10130CF000408B4238BF25
:10FC40005B0042F17D024FF4000C8B4224BF5B1A33
:10FC500040EA0C00B3EB510F24BFA3EB510340EA81
:10FC60005C00B3EB910F24BFA3EB910340EA9C002F
:10FC7000B3EBD10F24BFA3EBD10340EADC001B019F
:10FC800018BF5FEA1C1CE0D1FD2A3FF650AF8B4243
:10FC900040EBC25008BF20F0010070470CF0004C50
:10FCA0004CEA50207F32C2BFD2F1FF0340EAC2507B
:10FCB000704740F400004FF00003013A37E792F03C
:10FCC000000F00F0004C02BF400010F4000F013A9A
:10FCD000F9D040EA0C0093F0000F01F0004C02BF95
:10FCE000490011F4000F013BF9D041EA0C0195E7FE
:10FCF0000CEAD15392EA0C0F08D142027FF47DAF97
:10FD000093EA0C0F7FF470AF084676E793EA0C0F86
:10FD100004D14B023FF44CAF08466EE730F0004C84
:10FD200018BF31F0004CCAD130F000427FF45CAF14
:10FD300031F000437FF43CAF5FE700BF4FF0FF3C82
:10FD400006E000BF4FF0010C02E000BF4FF0010CD5
:10FD50004DF804CD4FEA40024FEA41037FEA226C9E
:10FD600018BF7FEA236C11D001B052EA530C18BFC0
:10FD700090EA010F58BFB2EB030088BFC81738BF25
:10FD80006FEAE17018BF40F0010070477FEA226C13
:10FD900002D15FEA402C05D17FEA236CE4D15FEA0F
:10FDA000412CE1D05DF8040B704700BF8446084643
:10FDB0006146FFE70FB5FFF7C9FF002848BF10F104
:10FDC000000F0FBD4DF808EDFFF7F4FF0CBF012049
:10FDD00000205DF808FB00BF4DF808EDFFF7EAFFD3
:10FDE00034BF012000205DF808FB00BF4DF808ED8E
:10FDF000FFF7E0FF94BF012000205DF808FB00BF83
:10FE00004DF808EDFFF7D2FF94BF012000205DF808
:10FE100008FB00BF4DF808EDFFF7C8FF34BF012015
:10FE200000205DF808FB00BF4FEA4002B2F1FE4F30
:10FE30000FD34FF09E03B3EB12620DD94FEA0023AC
:10FE400043F0004310F0004F23FA02F018BF404285
:10FE500070474FF00000704712F1610F01D142026C
:10FE600005D110F0004008BF6FF0004070474FF020
:10FE70000000704742000ED2B2F1FE4F0BD34FF09C
:10FE80009E03B3EB126209D44FEA002343F0004310
:10FE900023FA02F070474FF00000704712F1610F33
:10FEA00001D1420202D14FF0FF3070474FF0000005
:10FEB000704700BF0B460146184600F001B800BF6E
:10FEC00013460A460146022000F0ACBE014B1868FA
:10FED000704700BF2097FF1F70B50F4E0F4D761B68
:10FEE000B61018BF002405D0013455F8043B9847DC
:10FEF000A642F9D10A4E0B4D761B03F0DBFBB61080
:10FF000018BF002406D0013455F8043B9847A64298
:10FF1000F9D170BD70BD00BFC0360100C036010010
:10FF2000D4360100C0360100024B0146186800F0CB
:10FF30000BB800BF2097FF1F024B0146186800F066
:10FF400035BF00BF2097FF1F2DE9F04F01F10B05D2
:10FF5000162D83B0064640F29F8035F0070500F16C
:10FF6000BF80A94200F2BC8000F058FBB5F5FC7FD1
:10FF7000C0F09C826B0A00F0BA80042B00F28381EF
:10FF8000A80900F1390E4FEA4E033830C44F07EB91
:10FF90008303A3F108015C68A14207D1ACE0002A09
:10FFA00080F2AC80E468A14200F0A680636823F090
:10FFB00003035A1B0F2AF2DDB9493C6901F1080E0F
:10FFC000744500F0B381636823F003035A1B0F2AC2
:10FFD00000F39981002AC1F814E0C1F810E080F222
:10FFE0009E80B3F5007F80F06781DB0803F1010C90
:10FFF00001229B1002FA03F34A6851F83C80C4F8CE
:020000021000EC
:10000000088001EBCC091A43A9F10803E3604A60B8
:1000100041F83C40C8F80C40831001249C409442B5
:1000200000F28A80144206D120F0030064001442DA
:1000300000F10400FAD007EBC009CC468046DCF89A
:100040000C108C4507D173E1002A80F28181C968C8
:100050008C4500F06D814B6823F003035A1B0F2A77
:10006000F2DD0C46D1F80CC054F8088F4B1945F05E
:1000700001054D6042F00101C8F80CC03046CCF8D3
:1000800008807B613B61C3F80CE0C3F808E059606D
:100090009A5000F0C5FA1FE0102921D800F0BEFAEE
:1000A0001025062302207E4F07EB8303A3F10802ED
:1000B0005C68944200F045816368E168A56823F0BC
:1000C0000303234430465A68E96042F001028D6020
:1000D0005A6000F0A5FA0834204603B0BDE8F08F5E
:1000E00000240C232046336003B0BDE8F08F80234A
:1000F0004FF0400E3F2049E770465DE72344E1683A
:100100005A68A56842F00102E96030468D605A6085
:1001100000F086FA0834204603B0BDE8F08F23448F
:1001200030465A6842F001025A6000F079FA083409
:10013000204603B0BDE8F08FBC68636823F0030875
:10014000A84504D3C5EB08030F2B00F38C80554B57
:10015000DFF860911A68D9F8003001332A4404EBC3
:10016000080A00F0608102F580520F3222F47F62AB
:1001700022F00F0211463046019200F04BFCB0F124
:10018000FF3F8346019A00F05881824500F2FC80CF
:10019000454B1968DA451144196000F05381D9F8CC
:1001A0000000DFF810E101301BBFCAEB0B0A51441D
:1001B000CEF800B019601BF0070100F01781C1F103
:1001C0000800C1F58051834408315A44C2F30B0240
:1001D000C2EB010949463046019300F01BFC431C69
:1001E000019B00F03F81CBEB00024A4442F0010248
:1001F0001968C7F808B04944BC42CBF8042019601C
:10020000DFF8A49016D0B8F10F0F40F2FD806268BD
:10021000A8F10C0323F00703E01802F001024FF0ED
:10022000050E1A430F2B6260C0F804E0C0F808E026
:1002300000F21C811D4BBC681A68914288BF19608E
:100240001B4B1A689142626888BF196022F0030252
:100250009542A2EB050301D80F2B04DC304600F0D9
:10026000DFF9002438E7621943F0010345F0010586
:1002700065603046BA60536000F0D2F90834204619
:1002800003B0BDE8F08F142B71D9542B00F2A48079
:10029000280B00F16F0E4FEA4E036E3076E600BF7A
:1002A0002497FF1FBCA1FF1FC0A1FF1FB8A1FF1F04
:1002B000B4A1FF1F309BFF1F5A0A042A5ED9142ADB
:1002C00000F2B38002F15C0149005B3207EB810C64
:1002D00057F82110DFF8DC81ACF1080C8C4500F0F8
:1002E00088804A6822F00302934202D289688C45D2
:1002F000F7D1D1F80CC07A68C4F80CC0A160CCF872
:100300000840CC6088E6631942F0010745F001051A
:10031000656030464B610B61C3F80CE0C3F808E040
:100320005F609A50083400F07BF9D5E64A6873E6BE
:1003300008F1010818F0030F0CF1080C7FF47FAEF0
:1003400030E0DC68A34208BF02303FF435AEB3E6CC
:100350000B440C465A68C96854F8085F42F0010221
:100360005A603046E9608D6000F05AF9B4E603F156
:100370005C0E03F15B004FEA4E0307E69A0902F1B7
:10038000390149003832A1E7BC424A4B3FF400AF83
:100390009C68626822F003025AE759F808399945C7
:1003A00040F0828010F0030F00F1FF30F5D17B6840
:1003B00023EA04037B6064009C423FF6BDAE002C40
:1003C0003FF4BAAE1C4240467FF435AE64001C4296
:1003D00000F10400FAD02EE6B3F5AA7F18D8E80B96
:1003E00000F1780E4FEA4E037730CFE54FF480519D
:1003F000EBE60121D8F80430921001FA02F21A4318
:10040000C8F80420614677E70123CBF8043025E7DC
:1004100040F25452934220D8A80C00F17D0E4FEACE
:100420004E037C30B2E51032A4E6542A26D81A0BCB
:1004300002F16F0149006E3248E7BC68626822F041
:10044000030205E7CAF30B0000287FF4A8AE42447C
:10045000BB6842F001025A60ECE6FE234FF07F0ECB
:100460007E2093E501224FF00009C1E604F1080166
:10047000304600F09BFCD9F80010DBE6B2F5AA7F0D
:1004800005D8DA0B02F17801490077321EE740F215
:1004900054518A4205D89A0C02F17D0149007C3200
:1004A00014E7FE217E2211E77B6884E7E808431CFD
:1004B0005B00F8E52497FF1F8842F0B50DD98B1833
:1004C00098420AD28118002A51D09A1A13F8014D85
:1004D00001F8014D9342F9D1F0BD0F2A48D941EA04
:1004E00000039B0746D100F1100401F110031546EB
:1004F00053F8106C44F8106C53F80C6C44F80C6C06
:1005000053F8086C44F8086C103D53F8046C44F838
:10051000046C0F2D03F1100304F11004E8D8A2F1CC
:10052000100323F00F0302F00F0E1033BEF1030F80
:100530001944034421D91E1F0D467446043C55F846
:10054000047B46F8047F032CF8D8AEF1040424F0B1
:10055000030404342344214402F0030262B1013B4A
:100560000A4411F8014B03F8014F8A42F9D1F0BD5A
:100570000346F3E70346F2E7F0BD7246EEE700BF3D
:1005800070B4840746D0541E002A41D0CDB2034631
:1005900002E0621EE4B3144603F8015B9A07F8D147
:1005A000032C2ED9CDB245EA05250F2C45EA054589
:1005B00019D903F110022646103E0F2E42F8105CA6
:1005C00042F80C5C42F8085C42F8045C02F110024C
:1005D000F2D8A4F1100222F00F0204F00F0410323E
:1005E000032C13440DD91E462246043A032A46F82A
:1005F000045BFAD8221F22F003020432134404F0F1
:1006000003042CB1C9B21C4403F8011BA342FBD163
:1006100070BC704714460346C2E700BF704700BF76
:10062000704700BF024B0A460146186800F002B846
:100630002097FF1F2DE9F04F174683B0002900F0E7
:10064000C1800E46814607F10B05FFF7E7FF56F81C
:1006500004EC162D2EF00304A6F1080840D8102251
:100660001546AF4241D8944275DAC94B996808EBF8
:1006700004008842416800F0D98021F0010303445E
:100680005B68DB077DD51EF0010F35D03946484643
:10069000FFF75AFC0746E0B156F8043C23F001038B
:1006A0004344A0F108029A4200F04481221F242A08
:1006B00000F23181132A00F20481034632461168A8
:1006C00019605168596092689A603146484600F056
:1006D0006DFB4846FFF7A4FF384603B0BDE8F08F36
:1006E00025F00705002D2A46BBDA0C230020C9F8A7
:1006F000003003B0BDE8F08F56F8083CC3EB080AA1
:10070000DAF8043023F0030C04EB0C039342BDDB56
:100710005746DAF80C1057F8080F221F242AC16038
:10072000886000F21781132A40F212813168CAF8FA
:1007300008107168CAF80C101B2A00F22B810836C9
:100740000AF110023168116071685160B1689160FE
:100750003E461C46D046631B0F2B1DD8D8F80430EC
:1007600003F0010323434444C8F80430636843F0B2
:10077000010363604846FFF753FF304603B0BDE80E
:10078000F08F21F003012144914221DBC36882688C
:100790000C46D3609A60DEE7D8F8042008EB050128
:1007A00002F00102154343F001020B44C8F8045063
:1007B0004A605A6842F0010208315A60484600F027
:1007C000F5FAD7E7114603B0BDE8F04FFFF7BCBB21
:1007D0001EF0010F7FF45AAF56F8083CC3EB080A2D
:1007E000DAF8043023F0030C01EB0C0E96458BDB9A
:1007F000C36882685746D3609A6057F8081FDAF8D2
:100800000C30CB60221F242A996000F29980132AB1
:1008100062D93368CAF808307368CAF80C301B2AEA
:1008200000F2A08008360AF1100356E021F0030B15
:10083000A34405F11000834559DA1EF0010F7FF43F
:1008400025AF56F8081CC1EB080ADAF8041021F0AD
:10085000030CE34458453FF757AF5746DAF80C10FE
:1008600057F8080F221F242AC160886000F2B48064
:10087000132A40F2A5803168CAF808107168CAF8D6
:100880000C101B2A00F2AF8008360AF11002316802
:10089000116071685160B16891600AEB0501C5EBA8
:1008A0000B0242F0010299604A60DAF8043003F06A
:1008B00001031D434846CAF80450FFF7B1FE38460D
:1008C0005CE733680360736843601B2A27D800F134
:1008D000080306F10802F2E63B4632681A607268C5
:1008E0005A60B2689A603E467446D04633E708EBD9
:1008F0000501C5EB0B0B4BF0010299604A6056F8FD
:10090000043C03F001031D43484646F8045CFFF72E
:1009100087FE304632E73146FFF7CEFDD5E6B368B5
:100920008360F368C360242A28D000F1100306F125
:100930001002C4E650F8043C23F003031C440AE709
:10094000314638467446D046FFF7B6FD3E4602E7CC
:100950003A46F7E6314638461C46D046FFF7ACFD2E
:100960003E46F8E6B368CAF81030F368CAF81430A7
:10097000242A1BD010360AF11803AEE7336903614D
:100980007369436106F1180200F1180397E600BF8E
:100990002497FF1FB168CAF81010F168CAF8141044
:1009A000242A0FD010360AF11802CBE63369CAF8B0
:1009B00018307369CAF81C3018360AF120038CE726
:1009C0003A4664E73269CAF818207269CAF81C20EE
:1009D00018360AF12002B5E6314638460193FFF792
:1009E0006BFD019B59E7B168CAF81010F168CAF8AD
:1009F0001410242A03D010360AF1180247E732698E
:100A0000CAF818207269CAF81C2018360AF12002A8
:100A10003DE700BF38B5074C002305460846236074
:100A2000FBF7E0FE431C00D038BD2368002BFBD051
:100A30002B6038BD1CA3FF1FFFFFFFFFFFFFFFFF61
:100A400090F800F06DE9024520F007016FF0000C0E
:100A500010F0070491F820F040F049804FF00004B6
:100A60006FF00700D1E9002391F840F000F1080091
:100A700082FA4CF2A4FA8CF283FA4CF3A2FA8CF3C9
:100A80004BBBD1E9022382FA4CF200F10800A4FA30
:100A90008CF283FA4CF3A2FA8CF3E3B9D1E9042384
:100AA00082FA4CF200F10800A4FA8CF283FA4CF3BB
:100AB000A2FA8CF37BB9D1E9062301F1200182FA75
:100AC0004CF200F10800A4FA8CF283FA4CF3A2FA7B
:100AD0008CF3002BC6D0002A04BF04301A4612BA89
:100AE000B2FA82F2FDE8024500EBD2007047D1E98C
:100AF000002304F00305C4F100004FEAC50514F01B
:100B0000040F91F840F00CFA05F562EA05021CBFEB
:100B100063EA050362464FF00004A9E7002A41D0CA
:100B200040EA010313F00303F0B425D1032A23D9CB
:100B300004680D68AC421FD1043A35D0A4F10135E8
:100B400025EA040414F0803F31D1071D0D1D0DE08E
:100B500057F8043B0E68A3F10134B34224EA0304BE
:100B60000AD1043A20D014F0803F23D1032A294629
:100B7000384605F10405EBD803780C789C4202F165
:100B8000FF320CD182B114B916E06AB17BB110F812
:100B9000013F11F8014FA34202F1FF32F5D0181BBB
:100BA000F0BC7047104670471046F0BC70471846BE
:100BB000F0BC70470020F3E72046F1E740EA01036C
:100BC0009B0770B42BD1032A29D90C460346214632
:100BD00054F8046BA6F1013525EA060515F0803FAF
:100BE00006D1043A032A43F8046B2146EFD8A2B198
:100BF0000C781C70013A013301313CB16AB111F833
:100C0000014B03F8014B013A002CF7D12AB11A44E9
:100C1000002103F8011B9A42FBD170BC70470346C8
:100C2000E5E700BF2DE9F047254C2568D5F8484198
:100C30000646884692469946C4B360681F2817DC6A
:100C4000431C76B104EB80050122C5F888A0D4F8D6
:100C5000881182401143022EC4F88811C5F808910A
:100C60001ED00230636044F820800020BDE8F08789
:100C7000144B03B34FF4C870FFF756F90446D0B1D4
:100C8000D5F84831002780E88800C5F84841384643
:100C90000123C4F88871C4F88C71002EE1D0D1E72B
:100CA000D4F88C110A43C4F88C21DAE705F5A67450
:100CB000C5F84841C1E74FF0FF30BDE8F08700BFFD
:100CC000B036010029FF0000024B13B1024800F0CA
:100CD00005B8704700000000E90C01000023014640
:100CE0001A461846FFF79EBF38B5074D074C2C1B18
:100CF000A41005D0013C55F8043D9847002CF9D1CB
:100D0000BDE8384002F0E6BC000000000000000032
:100D1000F8B5234F0C460646FFF780FCBB685D68BC
:100D200025F00305291B01F6EF7121F47F6121F005
:100D30000F01A1F58054B4F5805F07DB0021304638
:100D4000FFF768FEBB682B44984204D03046FFF79B
:100D500067FC0020F8BD61423046FFF75BFE0130C2
:100D60000DD0104BBA6819682D1B45F001053046AF
:100D7000091B55601960FFF753FC0120F8BD0021E5
:100D80003046FFF747FEBA68831A0F2BDEDD064CAC
:100D90000449246843F00103001B53600860D5E751
:100DA0002497FF1FC0A1FF1F309BFF1F002945D0C4
:100DB0002DE9F0410D468046FFF730FC55F8047CE4
:100DC0006A4927F00103A5F10804E2188E6850680B
:100DD000B24220F0030062D0FE0750600BD455F8F9
:100DE000087CE41B01F1080EA56875453B446FD0F3
:100DF000E768EF60BD6015186D68ED0742D543F0F8
:100E000001026260E350B3F5007F18D2DB085A1C80
:100E10004D6851F83270A76001209B1000FA03F36F
:100E200001EBC2001D430838E0604D6041F83240DC
:100E3000FC604046BDE8F041FFF7F2BB70475A0A3C
:100E4000042A53D89A0902F139077F0002F13805C4
:100E500001EB870051F827204449083890424DD0D3
:100E6000516821F003018B4202D292689042F7D17F
:100E7000D068E060A2608460D4604046BDE8F04184
:100E8000FFF7CEBB95683A4FBD4203443FD0D068D0
:100E9000E86043F0010285606260E350B3E7FF075A
:100EA000034407D455F8082CA41A1344A068E26838
:100EB000C26090602F4A126843F001009342606064
:100EC0008C60B6D32C4B40461968FFF721FFB0E782
:100ED00011184968C90744D49168D268CA600344AC
:100EE00043F0010091606060E350A2E7142A17D834
:100EF00002F15C077F0002F15B05A9E7AA104B68CD
:100F0000012505FA02F213434B600246B1E743F0B4
:100F100001024C610C61E560A5606260E35088E706
:100F2000542A06D81A0B02F16F077F0002F16E05F2
:100F30008EE7B2F5AA7F06D8DA0B02F178077F00B8
:100F400002F1770584E740F25450824206D89A0CA9
:100F500002F17D077F0002F17C0579E7FE277E25FF
:100F600076E743F001026260E35062E72497FF1FD7
:100F70002C97FF1F2C9BFF1FBCA1FF1F00007805B3
:100F80003408540B800C3C0F5C12E015FA19141E47
:100F90006022AC265C2B0C30BC34023AFF3FFFFFD2
:100FA000FDFFFFFFFBFFFFFFF8FFFFFFFDFFFFFF60
:100FB000FBFFFFFFF8FFFFFFFDFFFFFFFAFFFFFF53
:100FC000F7FFFFFFFDFFFFFFFBFFFFFFF7FFFFFF47
:100FD000FCFFFFFFFBFFFFFFF7FFFFFFFDFFFFFF32
:100FE000FAFFFFFFF7FFFFFFFDFFFFFFFBFFFFFF24
:100FF000F8FFFFFFFDFFFFFFFBFFFFFFF8FFFFFF15
:10100000FDFFFFFFFAFFFFFFF7FFFFFFFCFFFFFF02
:10101000FBFFFFFFF7FFFFFFFDFFFFFFFBFFFFFFF2
:10102000F7FFFFFFFDFFFFFFFAFFFFFFF7FFFFFFE7
:10103000FDFFFFFFFBFFFFFFF7FFFFFFFDFFFFFFD0
:10104000FBFFFFFFF7FFFFFFFDFFFFFFFAFFFFFFC3
:10105000F7FFFFFFFDFFFFFFFAFFFFFFF8FFFFFFB6
:10106000FDFFFFFFFAFFFFFFF7FFFFFFFDFFFFFFA1
:10107000FAFFFFFFF7FFFFFFFDFFFFFFFAFFFFFF94
:10108000F8FFFFFFFDFFFFFFFAFFFFFFF8FFFFFF85
:10109000FDFFFFFFFAFFFFFFF7FFFFFFFCFFFFFF72
:1010A000FBFFFFFFF7FFFFFFFDFFFFFFFAFFFFFF63
:1010B000F7FFFFFFFDFFFFFFFAFFFFFFF7FFFFFF57
:1010C000FEFFFFFFFBFFFFFFF8FFFFFFFEFFFFFF3D
:1010D000FBFFFFFFF8FFFFFFFDFFFFFFFAFFFFFF32
:1010E000F7FFFFFFFCFFFFFFFAFFFFFFF7FFFFFF28
:1010F000FCFFFFFFFAFFFFFFF7FFFFFFFDFFFFFF12
:10110000FAFFFFFFF7FFFFFFFDFFFFFFF9FFFFFF04
:10111000F7FFFFFFFDFFFFFFF9FFFFFFF7FFFFFFF7
:10112000FDFFFFFFFAFFFFFFF7FFFFFFFDFFFFFFE0
:10113000FAFFFFFFF7FFFFFFFDFFFFFFFAFFFFFFD3
:10114000F6FFFFFFFDFFFFFFFAFFFFFFF7FFFFFFC7
:10115000FEFFFFFFFBFFFFFFF7FFFFFFFEFFFFFFAD
:10116000FBFFFFFFF7FFFFFFFDFFFFFFFAFFFFFFA2
:10117000F7FFFFFFFDFFFFFFFBFFFFFFF8FFFFFF94
:10118000FDFFFFFFFBFFFFFFF8FFFFFFFDFFFFFF7E
:10119000FAFFFFFFF7FFFFFFFCFFFFFFF9FFFFFF75
:1011A000F7FFFFFFFCFFFFFFF9FFFFFFF7FFFFFF68
:1011B000FDFFFFFFFAFFFFFFF7FFFFFFFDFFFFFF50
:1011C000FAFFFFFFF7FFFFFFFDFFFFFFF9FFFFFF44
:1011D000F6FFFFFFFDFFFFFFFAFFFFFFF7FFFFFF37
:1011E0009817010074170100501701002C17010017
:1011F000E4130100A0120100C4120100E812010072
:101200000C1301004C150100701501007C0F01004A
:101210000814010000000000070000000C0000009E
:101220001000000013000000180000001C00000067
:1012300000000000070000000C0000001300000088
:10124000180000001F000000240000000000000043
:101250000C00000018000000240000003000000016
:101260003C0000004800000000000000FBFFFFFF02
:10127000F4FFFFFFEFFFFFFFE8FFFFFFE3FFFFFFCC
:10128000DCFFFFFF00000000F4FFFFFFE8FFFFFFAF
:10129000DCFFFFFFD0FFFFFFC4FFFFFFB8FFFFFF32
:1012A0000000580246056608540BD80E5C12E01583
:1012B000FA19141E6022AC265C2B0C30BC34023AA6
:1012C000FF3FFFFF0000900120031405D0075A0ADA
:1012D000AC0DCC10B4146A18E81C342180252A2BDC
:1012E00070301437FF3FFFFF0000C800F401840393
:1012F000140508072E091C0CD80EF811AE15961906
:10130000401F1C25F22B5834FF3FFFFF00006400F4
:10131000C8009001BC021A04DC059E07F609800C87
:10132000A00F2413A2174C1D5424442FFF3FFFFF8E
:10133000FBFFFFFFF8FFFFFFF4FFFFFFFAFFFFFFD8
:10134000F7FFFFFFF4FFFFFFFDFFFFFFF9FFFFFFC8
:10135000F4FFFFFFFAFFFFFFF7FFFFFFF4FFFFFFC0
:10136000FCFFFFFFF7FFFFFFF4FFFFFFFBFFFFFFA7
:10137000F8FFFFFFF4FFFFFFFDFFFFFFFAFFFFFF96
:10138000F4FFFFFFFDFFFFFFF9FFFFFFF4FFFFFF8B
:10139000FDFFFFFFF8FFFFFFF4FFFFFFFCFFFFFF74
:1013A000F7FFFFFFF4FFFFFFFBFFFFFFF8FFFFFF6B
:1013B000F4FFFFFFFCFFFFFFF7FFFFFFF4FFFFFF5E
:1013C00040067805B004E80384032003BC025802F9
:1013D000F40190012C01FA00C8009600640032006C
:1013E0001900FFFF0000FF03FF07FF0BFF0FFF13B4
:1013F000FF17FF1BFF1FFF23FF27FF2BFF2FFF33CD
:10140000FF37FF3BFF3FFFFF0000D007800CD80EE7
:101410000010C012EC130C17FA19141E6022AC262F
:101420005C2B0C30BC34023AFF3FFFFFFBFFFFFF99
:10143000F8FFFFFFF4FFFFFFFAFFFFFFF7FFFFFFDB
:10144000F4FFFFFFFDFFFFFFF9FFFFFFF4FFFFFFCA
:10145000FAFFFFFFF7FFFFFFF4FFFFFFFCFFFFFFB7
:10146000F7FFFFFFF4FFFFFFFBFFFFFFF8FFFFFFAA
:10147000F4FFFFFFFDFFFFFFFAFFFFFFF4FFFFFF99
:10148000FBFFFFFFF8FFFFFFF4FFFFFFFDFFFFFF84
:10149000F8FFFFFFF4FFFFFFFCFFFFFFF7FFFFFF79
:1014A000F4FFFFFFFBFFFFFFF8FFFFFFF4FFFFFF6D
:1014B000FCFFFFFFF7FFFFFFF4FFFFFFFBFFFFFF56
:1014C000F8FFFFFFF6FFFFFFFAFFFFFFF8FFFFFF48
:1014D000F6FFFFFFFDFFFFFFFBFFFFFFF9FFFFFF31
:1014E000FDFFFFFFF9FFFFFFF7FFFFFFFEFFFFFF1D
:1014F000FCFFFFFFF7FFFFFFFBFFFFFFF8FFFFFF12
:10150000F6FFFFFFFCFFFFFFFAFFFFFFF6FFFFFF05
:10151000FDFFFFFFFBFFFFFFF9FFFFFFFCFFFFFFEA
:10152000FAFFFFFFF6FFFFFFFEFFFFFFFCFFFFFFDD
:10153000F7FFFFFFFBFFFFFFF8FFFFFFF6FFFFFFD7
:10154000FEFFFFFFFCFFFFFFF7FFFFFF0000580259
:1015500046056608540BD80E5C127017FC21F82A59
:1015600070305834DC37663A8C3C803EFF3FFFFFDA
:101570000000580246056608540BA00FD417282314
:10158000F82A442F643284354038663A8C3C803ED9
:10159000FF3FFFFF00000000070000000C000000FC
:1015A00010000000130000001A0000001F000000DF
:1015B00000000000070000000C0000001000000008
:1015C00013000000180000001C0000002C01130193
:1015D000FA00E100C800AF0096007D0064004B00F7
:1015E0003200190000000000CDCC4C3DCDCCCC3DEC
:1015F0009A99193ECDCC4C3E0000803E9A99993E76
:101600003333B33ECDCCCC3E6666E63EFBFFFFFFF8
:10161000F7FFFFFFF6FFFFFFFBFFFFFFF7FFFFFFF7
:10162000F6FFFFFFFBFFFFFFF7FFFFFFF6FFFFFFE8
:10163000FDFFFFFFFCFFFFFFF8FFFFFFFDFFFFFFC8
:10164000FCFFFFFFF8FFFFFFFDFFFFFFFCFFFFFFB9
:10165000F8FFFFFFFBFFFFFFF7FFFFFFF6FFFFFFB6
:10166000FBFFFFFFF7FFFFFFF6FFFFFFFBFFFFFFA3
:10167000FAFFFFFFF8FFFFFFFCFFFFFFF9FFFFFF8F
:10168000F8FFFFFFFDFFFFFFFCFFFFFFF8FFFFFF7D
:10169000FCFFFFFFFAFFFFFFF7FFFFFFFBFFFFFF6E
:1016A000F7FFFFFFF4FFFFFFFBFFFFFFF7FFFFFF69
:1016B000F4FFFFFFFBFFFFFFF7FFFFFFF4FFFFFF5C
:1016C000FDFFFFFFF8FFFFFFF4FFFFFFFDFFFFFF40
:1016D000F8FFFFFFF4FFFFFFFDFFFFFFF8FFFFFF35
:1016E000F4FFFFFFFBFFFFFFF7FFFFFFF4FFFFFF2C
:1016F000FBFFFFFFF7FFFFFFF4FFFFFFFBFFFFFF15
:10170000F8FFFFFFF4FFFFFFFCFFFFFFF9FFFFFF04
:10171000F4FFFFFFFDFFFFFFF8FFFFFFF4FFFFFFF8
:10172000FCFFFFFFF7FFFFFFF4FFFFFF000078055E
:10173000220B0410B4143219B01DFC214826FE29D6
:10174000822D383126344637663A223DFF3FFFFF6F
:101750000000D007100E88133219AA1E2823742700
:101760005C2B442F643284354038663A8C3C803E92
:10177000FF3FFFFF0000540BEC13FA1908201C2553
:101780003629EC2C0C302C33E8357238663AF63BAF
:10179000863D163FFF3FFFFF0000CC10581BFC2189
:1017A000AC26C62A7C2E3831F4334C36A438983A0D
:1017B0005A3C543D803E7A3FFF3FFFFF000000004F
:1017C000070000000C0000001000000013000000E3
:1017D000180000001A000000070000000C000000C4
:1017E0001000000013000000180000001A000000A4
:1017F0001F000000FBFFFFFFF7FFFFFFF4FFFFFFED
:10180000FBFFFFFFF7FFFFFFF4FFFFFFFDFFFFFF01
:10181000F7FFFFFFF4FFFFFFFDFFFFFFF8FFFFFFF4
:10182000F4FFFFFFFAFFFFFFF7FFFFFFF4FFFFFFEB
:10183000FBFFFFFFF7FFFFFFF4FFFFFFFBFFFFFFD3
:10184000F7FFFFFFF4FFFFFFFBFFFFFFF7FFFFFFC7
:10185000F4FFFFFFFDFFFFFFF8FFFFFFF4FFFFFFB7
:10186000FDFFFFFFF8FFFFFFF4FFFFFFFDFFFFFF9E
:10187000F8FFFFFFF4FFFFFFFAFFFFFFF8FFFFFF96
:10188000F4FFFFFFF4180100009CFF1F0000FF0F92
:10189000B89DFF1F0000FF0FF9530000C0180100A2
:1018A000B09DFF1F32005E0100000000000000003C
:1018B0009953000054485200534E53004D41580074
:1018C000544F5543482053454E53450045585452B4
:1018D0004120434F4E54524F4C4C455200000000A3
:1018E00050495443482042454E4400004249544523
:1018F0000000000042524541544800FFCC1801004E
:101900000C9DFF1FF401A00F089DFF1FF401A00F05
:10191000A5530000EC180100789DFF1FBC025C126B
:10192000909DFF1FBC025C12DD530000E018010017
:101930005A9DFF1FF401A00F989BFF1FF401A00FF9
:10194000C153000068220100702201005C220100E6
:101950006022010064220100D02001002022010049
:101960003C220100402201004422010048220100E3
:101970004C220100502201005422010028220100C3
:1019800058220100D0200100CC20010030220100AB
:101990003422010038220100D02001002022010061
:1019A00024220100282201002C2201000C22010027
:1019B0001022010014220100182201001C22010043
:1019C0009829010004220100082201007822010068
:1019D0007C22010080220100842201008822010073
:1019E0008C22010090220100942201009822010023
:1019F0009C220100A0220100A4220100A8220100D3
:101A000001000000AC2201000700000000000000FF
:101A100000000000000000000000000000000000C6
:101A200000000000000000000000000000000000B6
:101A300000000000000000000000000000000000A6
:101A40000000000000000000000000000000000096
:101A50000000000000000000000000000000000086
:101A60000000000000000000000000000000000076
:101A70000000000000000000000000000000000066
:101A80000000000000000000000000000000000056
:101A90000000000000000000000000000000000046
:101AA0000000000000000000000000000000000036
:101AB0000000000000000000000000000000000026
:101AC0000000000000000000000000000000000016
:101AD0000000000000000000000000000000000006
:101AE00000000000000000000000000000000000F6
:101AF00000000000000000000000000000000000E6
:101B000000000000000000000000000000000000D5
:101B100000000000000000000000000000000000C5
:101B200000000000000000000000000000000000B5
:101B30000001FFFFFFE3600007736000000000008A
:101B40000001FFFFFFE360000EE360000000000003
:101B500000018000000360001DC360000000000061
:101B60000001BFFFFFE360003B8360000000000056
:101B70000001BFFFFFE3600077036000000000008A
:101B80000001B00000036000EE03600000000000F0
:101B90000001B00000036001DC03600000000000F1
:101BA0000001B00000036003B803600000000020E3
:101BB0000001B000000360077003600000000060D7
:101BC0000001BFFFFFE3600EE00360000000006063
:101BD0000001BFFFFFE3601DC00360000003006061
:101BE000000180000003603B80036000000300E010
:101BF0000001BFFFFFE3607700036000000300C047
:101C00000001BFFFFFE360EE00036000000380C03F
